:020000022000DC
:1060000000000120756302005D6302005F6302000F
:106010006163020063630200656302000000000028
:1060200000000000000000000000000067630200A4
:1060300069630200000000006B6302006D630200F0
:10604000F99C02006F630200FDA002006F63020072
:106050006F6302006F630200B19F02006F63020072
:106060006F6302006F6302006F6302006F630200E0
:106070006F6302006F6302006F6302006F630200D0
:106080006F630200097902006F6302006F63020010
:106090006F6302006F63020075F602006F63020017
:1060A0006F6302006F6302006F6302006F630200A0
:1060B0006F6302006F630200000000000000000038
:1060C0006F6302006F6302006F6302006F63020080
:1060D0006F6302006F6302006F6302000000000044
:1060E00000000000000000000000000000000000B0
:1060F00000000000000000000000000000000000A0
:10610000000000000000000000000000000000008F
:10611000000000000000000000000000000000007F
:10612000000000000000000000000000000000006F
:10613000000000000000000000000000000000005F
:10614000000000000000000000000000000000004F
:10615000000000000000000000000000000000003F
:10616000000000000000000000000000000000002F
:10617000000000000000000000000000000000001F
:10618000000000000000000000000000000000000F
:1061900000000000000000000000000000000000FF
:1061A00000000000000000000000000000000000EF
:1061B00000000000000000000000000000000000DF
:1061C00000000000000000000000000000000000CF
:1061D00000000000000000000000000000000000BF
:1061E00000000000000000000000000000000000AF
:1061F000000000000000000000000000000000009F
:10620000354936480A1A02D0072291438D4634494F
:1062100034480A1A06D00722914381F309880222E2
:1062200082F3148830483149314A00F044F831484B
:106230003149324A00F03FF831483249324A00F0E1
:106240003AF832483249334A00F035F83248334997
:10625000334A00F030F833483349344A00F02BF821
:1062600033483449344A00F026F83448344900228F
:1062700000F02CF833483449002200F027F8334866
:106280003349091A082902DB002202604160314AC1
:1062900090471F481F49884205D00268043003B464
:1062A000904703BCF7E700208646EC46002000211B
:1062B000294A9047FEE7884207D0521A05D0037852
:1062C00001300B700131013AF9D17047884202D098
:1062D00002700130FAE770470000012000E0002062
:1062E0000000012000000120142F03003C2A0020A0
:1062F0006C300020D0630200D0630200040603006B
:10630000142F03003C2A00203C2A002078070300B9
:106310007807030078070300780703007807030075
:10632000780703007807030078070300132F0300A2
:10633000443503006C3000206C3000206C300020AD
:10634000D8440020D8440020DC440020DC44002055
:10635000DC6400209D63020099BA0200FEE7FEE7BC
:10636000FEE7FEE7FEE7FEE7FEE7FEE7FEE7FEE705
:1063700000F002B8FFF7FCBF0F484FF00701884359
:1063800085460E4880470E48016841F4700101605F
:10639000BFF34F8FBFF36F8FFFF732BF09480A4932
:1063A0000A4A884207D0521A05D0037801300B7090
:1063B0000131013AF9D17047000001202197020014
:1063C00088ED00E064070300282A00203C2A002012
:1063D00000487047D04400207047000007B5044BC8
:1063E0000093044A402300F032F803B05DF804FB48
:1063F000F96302006D3000202DE9F8438846144609
:10640000B2B10F4B0F4E0325002743F0010922467E
:1064100008EB0701002007F057FB0744241A48B98E
:1064200033782BB14FF47A40C847013D02D1357023
:10643000BDE8F88301233370002CE8D1F8E700BFF2
:10644000800703006C300020704707F06DBBF0B58B
:1064500095B01D46164608460C4601F019FE1A9BDB
:106460000D93CDE9086500252B46082205A9204695
:106470000A958DF82C500C9501F026FE079B02938F
:10648000069B03939DF814308DF8115003F003021E
:10649000012A1DD1BDF81420059DC3F3C203C2F328
:1064A00083168DF81030B20008230EA9204601F0A3
:1064B0000BFEC5F3952508AB0093324602AB0EA93F
:1064C000284600F05BFB204601F0E6FD15B0F0BD6C
:1064D000022AF8D1BDF81650C3F3C203C5F38915DB
:1064E0008DF810300827082D2E4628BF08263B4679
:1064F00032460EA9204601F0E7FDAD1B08AB02AA0B
:1065000031460EA8374400F09DFB002DEBD1DAE7B1
:1065100008B5FFF79AFF0448042100F099FA034BED
:1065200001225A7108BD00BF540703003C2A002015
:10653000037813F0040216D003F00303012B03D0F9
:10654000022B09D0012070470A6800880232C0F38C
:10655000831002440A60F5E70B684288023303EBBC
:1065600092130B60EEE71046704700002DE9F04FE4
:10657000DFF81CA187B00F4600230446861C0DF1EE
:10658000070015468DF8073001F050F8DAF80420BE
:106590003A60DAF8083003F580739B1A0AF21C4758
:1065A0000AF583690AF21448B3421AD30020002D79
:1065B00069D004F00F039B0143F0050363F30F0060
:1065C000DAF80430DAB2033233444AF822009DF894
:1065D0000700CAF8043001F04DF8012007B0BDE80B
:1065E000F08F0121384601F07EFA484601F096FA14
:1065F000404601F093FADAF808000290C0B2033086
:106600000AEB800002A9FFF793FF029B30BBDAB2CE
:106610000AEB8202D16803919A1C0133DBB20AEBC8
:1066200083030292D3F80CB001F00303012B22D0B4
:10663000022B15D08346404601F073FA10B1029B3D
:10664000CAF808305946384601F04DFADAF80830F1
:10665000DAF8042003F580739B1AA5E7D8B2CEE7D9
:10666000BDF80E30C3F3891303334FEA1B4B02EB23
:1066700093030293DFE7BDF80C30C3F383134FEAB3
:106680001B4B1344F5E7A40544F0060098E700BF50
:1066900080310020064B074810B500221A7001F027
:1066A000B0FC044610B9044801F011FE204610BDAC
:1066B00080310020B8060300BC07030030B50A4C47
:1066C00071B10A4A0A49121BD20800239A4201D129
:1066D000002030BD31F82350854202D00133F5E768
:1066E000034654F83300F4E718060300B806030025
:1066F000282A0020094B013903EBC000032909D8DF
:10670000DFE801F00A0204060420704700797047B0
:106710004079704700207047022070471806030038
:10672000034BD3E90130C31A58425841704700BFA8
:10673000803100202DE9F04186B0FFF7F1FF0546DA
:10674000002840F0ED80774CC4F81804BFF34F8F59
:10675000A3680293DBB2033304EB830002A9FFF7C3
:10676000E7FE029B18B1D4F81824002A5AD0DAB2F6
:10677000991C013304EB8202DBB204EB8303D26881
:10678000DB68049302F00303022B0392029154D1BD
:10679000BDF80E306448C3F38917502F3E4628BF1A
:1067A000502606F1080166F38F13C1F30901ADF815
:1067B0000E3001F03EFC0546002800F09C8001F000
:1067C00067FC0023082203A9284601F073FC029904
:1067D000CB43DBB20133C9B20331B6EB830F4FEACF
:1067E000830204EB810125D95FFA82F80823A6EB26
:1067F0000806284601F05EFCF6B208F108034B4992
:1068000003F0FC033246284601F054FC029B033798
:1068100003EB97070297D4F81834002B43D1D4F830
:10682000106453E062689A4294D8A260284606B089
:10683000BDE8F08108233246E5E7012B5BD1BDF8C6
:106840000C303948C3F38311062928BF062161F3B0
:106850008913023101F00F018900ADF80C3001F00D
:10686000E8FB0546002846D001F012FC0023082270
:1068700003A9284601F01EFC0026BDF80C20C2F337
:106880008312B300964203F10803C4D202994A1C52
:10689000C9B20331029204EB81010422284601F0BF
:1068A00009FC0136E9E7284601F0F6FBFFF738FF5F
:1068B00080F00100C5B2B9E7F3685B7923B13368B2
:1068C00029461B6830469847F3681E68002EF3D1AE
:1068D000284601F0E1FB0DF107008DF8076000F09C
:1068E000A5FED4F818340BB9029BA3609DF80700ED
:1068F00000F0C0FEDAE7D4F8104454B90C4B0D4850
:106900000D49C01AC008000440F0020000F05CF815
:10691000CCE7236820469B689847E3681C68ECE74F
:10692000002583E780310020B80603008C31002069
:106930001806030040060300A40703002DE9F347EF
:1069400004460E46924601A9012218469946FFF7D1
:106950000DFE1B4F10B3019D4FF00008AA1CC84547
:1069600008EB020123D11748002101F081F880F3E0
:106970001000000440EA1440E4006B1C04F03804EA
:10698000DBB2EDB244F0010407EB8303033544EAC4
:10699000881444EA8624D86047F825403B781BB128
:1069A000FFF7C8FE0028FBD102B0BDE8F087C9B2EE
:1069B00007EB81015AF82830CB6008F10108CEE7D7
:1069C000803100209C35002000231A46FFF7B6BF17
:1069D00007B50123019201AAFFF7B0FF03B05DF8EC
:1069E00004FB07B5CDE9002302236A46FFF7A6FFA3
:1069F00003B05DF804FB1FB5CDE90123069B0393AB
:106A000001AA0323FFF79AFF05B05DF804FB1FB549
:106A1000CDE90023069B0293079B03936A46042358
:106A2000FFF78CFF05B05DF804FB7FB5CDE90023CF
:106A3000089B0293099B03930A9B04930B9B05936A
:106A40006A460623FFF77AFF07B05DF804FB0000F3
:106A500030B50F4CD4F8102403460020114631B94C
:106A6000D96808714AB9C4F810340A6030BDC968E1
:106A70000D79854206D00968F1E7D26814680C6088
:106A80001360F3E701300A28E8D14FF0FF30EDE75B
:106A90008031002038B5084B0125D3F810441D7013
:106AA00004B938BDE3685D71236820465B68984788
:106AB000E3681C68F4E700BF8031002030B5C3886C
:106AC00085B004460D4633B1144A00921449154A64
:106AD000284601F089F8217A05291DD0637A4BB147
:106AE000A088FFF707FE104B104953F820202846D6
:106AF00001F07AF8227A0E4BA08853F822200392F4
:106B00000021FFF7DBFD039A0A490346284605B03A
:106B1000BDE8304001F068B805B030BDE8070300BB
:106B2000D0070300C807030054080300ED07030063
:106B300078080300F007030007B503460846197AF2
:106B4000052911D05B7A2BB1094A0A49019001F05D
:106B50004BF801980849019001F046F8019803B0FC
:106B60005DF804EB01F035B8002AF8D0F2E700BF79
:106B7000E8070300ED0703003B1403002DE9F04391
:106B800085B01F460C9D002395F80C902B7306468C
:106B90000C46904629463846FFF790FFB8F1060F9D
:106BA00009D8DFE808F00412181F283340003146E6
:106BB000284601F019F8002229463846FFF7BCFFA5
:106BC00085F80C9005B0BDE8F08322683146284670
:106BD00001F00AF8EFE7D4E900233146284601F036
:106BE00003F8E8E7A36800933146D4E90023284678
:106BF00000F0FAFFDFE7E3680193A36800933146F2
:106C0000D4E90023284600F0EFFFD4E7236902937C
:106C1000E3680193A36800933146D4E90023284632
:106C200000F0E2FFC7E76369039323690293E36817
:106C30000193A36800933146D4E90023284600F06D
:106C4000D3FFB8E708292DE9F74F80460E461746CF
:106C50001C463DD800251B7B257321461046019319
:106C6000FFF72CFFDFF88CA0DFF88CB0AE4232D9F2
:106C700018F805205946204600F0B6FF0135082DCA
:106C8000F4D11B49DFF874A0DFF874B0204600F09F
:106C9000ABFF4FF000094E4524D918F809507E2D5E
:106CA0001ED8284608F076FF002814BF2A462E2258
:106CB0005946204600F098FF09F10109B9F1080F83
:106CC000E9D1012221463846FFF736FF019B2373A5
:106CD00003B0BDE8F08F5146204600F085FFCDE7B8
:106CE0002E22E5E75146204600F07EFFE4E700BF94
:106CF0000408030000080300FA0703000208030069
:106D000006080300C30710B507D4F023054A40085E
:106D1000145C23401943115410BD0901C9B20F235B
:106D2000F4E700BF6836002030B5094B1C78094BEA
:106D3000196800239C4202DC0022104630BD11F885
:106D40003350854201EBC302F7D00133F2E700BFB5
:106D5000383600207836002013B504460191FFF73D
:106D6000E3FF38B143682BB10199204602B0BDE87A
:106D70001040184702B010BD034B044819680022A8
:106D8000490800F058BA00BF3C36002040360020C9
:106D900010B5C0B2FFF7C8FF0446007803F0FEF854
:106DA00063785A1E53425341834208D1044BD3E9BE
:106DB0000023134303D1BDE81040FFF7DDBF10BD32
:106DC0006036002037B54308374AD35CC2074CBF52
:106DD0001B0903F00F0304460D46042B25D8DFE8FA
:106DE00003F003262F3C4000F9B10121FFF78AFF91
:106DF00000230DF107008DF8073000F017FC01208B
:106E0000A4F12003C4F12001284A20FA01F100FA7C
:106E100003F30B43A040D2E9004120430B43C2E9F6
:106E200000039DF8070000F025FC03B030BD0029E9
:106E300018BF0221204603B0BDE83040FFF762BF13
:106E400049B10321FFF75EFF0121204603B0BDE8F1
:106E50003040FFF781BF0121ECE70029E5D1042193
:106E6000E8E709B10321E5E7FFF74CFF2946204693
:106E7000FFF772FF0DF107008DF8075000F0D6FB09
:106E80000120A4F12003C4F12001084A20FA01F1F5
:106E900000FA03F30B43A040D2E9004124EA0000CA
:106EA00021EA0303BBE700BF6836002060360020FC
:106EB0002DE9F041124E134F00243378A34208DC31
:106EC000114BD3E90023134318D0BDE8F041FFF77D
:106ED00053BF3D6805EBC40815F8340003F05EF8B5
:106EE00098F801305A1E53425341181A4142414109
:106EF00015F83400FFF766FF0134DEE7BDE8F081E6
:106F0000383600207836002060360020092AF7B590
:106F100005460C4616463ED902F078FFE8B11F4BF5
:106F20001F481D601F4B204F1C70204B002110225A
:106F30001E6008F0C5FF1E4B00200021C3E90001C0
:106F4000013CE4B20326FF2C0DD11A4A1A48002155
:106F500003B0BDE8F04000F063B902F01FFF002865
:106F6000DDD003B0F0BD9DF8063015F834008DF883
:106F7000046005EBC40223F007038DF8063001A975
:106F800093788DF805303A4602F04AFF013CE4B2AE
:106F90000028D8D0E5E70720E3E700BF78360020D7
:106FA0006836002038360020916D02003C36002003
:106FB00060360020B16E02009808030070B5084DDD
:106FC000084E00242B789C4201D3002070BD33680A
:106FD000012113F8340002F09BFF0134F2E700BFF7
:106FE00038360020783600201FB50021039001AA12
:106FF00044F20100CDE9011100F004F805B05DF89C
:1070000004FB000010B572B6FFF744FDFFF792FBDA
:107010000028FBD10D4B0E4C0E49E41AE408240461
:1070200044F00100FFF7D0FC0B4944F00200FFF7E9
:10703000CBFCBFF34F8F0949094BCA6802F4E062E9
:107040001343CB60BFF34F8F00BFFDE7180603006B
:10705000400603009C080300A808030000ED00E0C0
:107060000400FA0549B152B1531E1A4007D182609B
:1070700001608380C260104670470E20704709206F
:10708000704710B58468C2688388121B934208D386
:10709000C26813400268D154C3680133C360002042
:1070A00010BD0420FCE78268C3689A420AD0826857
:1070B000838813400268D35C0B708368013383605C
:1070C000002070470520704710B5D0E90243D1E990
:1070D0000202A04272EB03032CBF0120002010BD6E
:1070E00008B50A4800F0F9FB094AD2E90031C01896
:1070F000084BD3E9002341F10001904271EB0303F7
:1071000003D210F1807041F1000108BD442A002033
:1071100080360020F836002037B505460C460A4870
:1071200001A900F030FC60B10570446001A9064877
:1071300000F053FC18B1054800F0D4FB002003B068
:1071400030BD0420FBE700BFE4360020442A0020C5
:1071500038B5184B1B78044613B90025284638BDAE
:107160000028FAD0037F03F0FF05002BF5D0FFF7CE
:10717000B7FFD4E90223904271EB030314D32369D0
:1071800003B92377D4E90530984721690029E4D071
:10719000237F03F0FF05002BDFD0D4E902325B1818
:1071A00042F10002C4E902320348214601F0AEF880
:1071B000D4E700BF88360020C408030013B5114B84
:1071C00011491868019008231048582200F0A6FBC6
:1071D000044698B90E4A0F4801A900F06FFA044618
:1071E00060B90C48012100F05BFB01230A4A094801
:1071F000194600F0BDFA094B01221A70204602B070
:1072000010BD00BFC00803008C360020E43600200B
:1072100081720200442A0020FFFF7F008836002090
:107220003AB103685A614A1E514251411961002026
:1072300070470720704738B5037F04460D4683B971
:107240008261FFF74DFF2369281841F10001C4E96D
:10725000020103B1256121460020BDE83840FFF757
:107260005BBF002038BD0023014603770120FFF7F4
:1072700053BF0000014800F030BB00BF442A00208B
:107280002DE9F347064600F013FB40B1584AD2E916
:10729000003113F1807341F10001C2E90031002196
:1072A000304600F014FB38B1524C236823B12068FB
:1072B000FFF74EFF002323600121304600F007FB5B
:1072C00020B1FFF70DFF4C4BC3E900014B48494D7E
:1072D0004B4C4C4F01A900F090FB002842D1DFF845
:1072E0002081444CDFF82491404601F025F82368C2
:1072F000002872D07BB12368D0E90252D3E902138F
:107300008D4272EB03032AD223681B7F1BB12168D5
:10731000404600F0FBFF404601F008F8D0E9027A51
:107320000546FFF7DDFE381A6AEB010A01287AF1FB
:10733000000345DBB0F5350F40D3FFF79BFF324A22
:1073400002444FF496030021484600F031FA002829
:107350003ED1236813B9304600F002FA256002B02E
:10736000BDE8F0870378012B1DD0022B09D14FF027
:107370000008204600F0DAFF002836D080F81C8094
:10738000F7E73BB941680B7F23B901230B77204610
:1073900000F0BCFF01A9194800F05AFB01A91748E9
:1073A00000F02BFB99E741682B68994202D100233A
:1073B0002B60EFE7204600F0C2FFEBE7AA68C0E7CA
:1073C0000021484600F079FA2846FFF7C1FE01E0A7
:1073D0000D28F9D00023236086E7002BBFD130466B
:1073E00002B0BDE8F04700F0BFB901233B70D1E720
:1073F0008036002000370020F8360020E4360020D8
:10740000C408030088360020FFFFB400442A00208F
:107410000648074A03780749D35C012213B10430B8
:1074200003F0CCBA0C3003F08FB800BF4C2A002018
:107430004C3900202C3700200648074A03780749BA
:10744000D35C012213B1043003F06ABA0C3003F0AC
:107450002BB800BF4C2A00204C3900202D370020CB
:1074600037B50578012D0DD0022D30D075B91F49E3
:107470001F48FFF718FE002834D103B0BDE83040A4
:10748000FFF7DABF037A1BB9FFF7C2FF03B030BDC5
:107490004368184C19782046FFF7F3FD80B18DF84A
:1074A00000500190144B68461B689847A168E36838
:1074B000A2885B1A9A42E7D2104B01221A70E5E7C4
:1074C000A268E3689A42F1D08DF80000EAE7C36849
:1074D0008DF800500193FFF79BFF074B68461B6830
:1074E0009847D3E703238DF80030F6E72D370020C7
:1074F0001C370020083700200437002018370020F0
:10750000F0B51F46234B89B004461A600D4600298A
:107510003DD08A8820480968FFF7A4FD002834D1AF
:10752000AA89A9681D48FFF79DFD00282DD11C4E92
:107530000FCE6D460FC596E80F0085E80F00636912
:107540000693237C174A18488DF81C70003B18BF1F
:1075500001238DF81430637C002B14BF0E2300230D
:107560008DF81530E3680293A368039323680193B1
:1075700069466368009302F047FB30B90B4B187003
:107580002368013301D0FFF743FF09B0F0BD0720A6
:10759000FBE700BF04370020083700201C3700201D
:1075A000D0080300617402004C2A00201837002024
:1075B00070B5084D014608482E78FFF774FD044663
:1075C00036B100232B70FFF723FF08B1FFF70CFD46
:1075D000204670BD183700200837002010B501463E
:1075E0000E48FFF74EFD0446A8B90D480D4A037832
:1075F000D35C63B1043003F087F960B90A490748E6
:10760000FFF751FD38B9BDE81040FFF715BF0C304A
:1076100002F03EFFF1E7204610BD00BF1C370020FE
:107620004C2A00204C3900202D37002070B5EFF394
:10763000108672B60C4A946801239CB993600B4B78
:107640000B4DD3F8801029401160C3F88050D3F857
:10765000841051604FF0FF32C3F88420047006B9E3
:1076600062B670BD0370FAE73037002000E100E039
:10767000FC06FFBD084B9A6810B55AB150B9EFF33C
:10768000108172B6054A1C6814605C68546098608A
:1076900001B962B610BD00BF3037002000E100E044
:1076A000435882B03BB10023435043580193019BA0
:1076B000012002B070471846FBE70000F8B5204BE8
:1076C0004479204E43F824201F4A204B06EBC40483
:1076D0009B1A2279DB081B0432B143F002001C49DB
:1076E000FFF772F90820F8BD02680C88C2F8084557
:1076F00090F904508A7804795201002DD2B219DB36
:1077000014494F1987F8002301226D0904F01F0462
:1077100002FA04F441F82540427906EBC201012443
:1077200046F832000C7143F003000B49FFF74CF9A7
:107730000020D8E7094904F00F040A55ECE700BF20
:10774000443700203C370020180603005006030091
:10775000F008030000E100E01209030014ED00E06E
:10776000036801221A607047036801225A6070475B
:1077700073B501F15005AD000068ADB24FF480342F
:107780008C400026C0F80843C0F84843465101F534
:10779000A8714559019522F07F42019D40F82120B2
:1077A000C0F844430BB1C0F8044302B070BD000000
:1077B0002DE9F74F0D4622F07F4402684FF48037E1
:1077C00005F150068F408046B60002EB8500C2F8F6
:1077D0004873B6B2C2F80873D2F8041599464FF050
:1077E000000BD0F84035C0F8401542F806B05B1ADF
:1077F0009259009223F07F43012B009A4FEA850AA9
:107800000CD1264B4FF4806043F001039847D8F821
:10781000003043F806B09B590193019BD8F8001043
:10782000D1F80465C1F84473A31B23F07F43012BF7
:107830001CD11A4B05F5A875013443F0010341F83A
:1078400025404FF480609847D8F80030D3F80435CD
:107850009E4209D1D8F800300020C3F84473C3F821
:10786000047303B0BDE8F08F0D20FAE78A44C9F134
:10787000FF13CAF84045D1F80405221A013A22F054
:107880007F4203F57F439342EED3002AE2D10134D5
:10789000CAF84045D1F804359842DAE730090300C8
:1078A00003680222C3F8442309B1C3F804237047D4
:1078B00000684FF48271FFF7F3BE4FF4803303FA90
:1078C00001F10368C3F84813C3F808137047503137
:1078D0008900006889B2FFF7E3BE0368D3F80405A6
:1078E0007047000090F90430002B09DB5A09012190
:1078F00003F01F0301FA03F34032024941F822303A
:10790000704700BF00E100E0024B034A1B681068AB
:10791000184700BF443700203C37002010B561B144
:10792000B2FBF3F403FB1424A4B244B9C0E900147D
:1079300084608281C381204610BD0E20FCE70920AF
:10794000FAE782B050E8022FC188B2EB324F4FF015
:10795000000317BF92B241EA014142EA014104E04B
:107960004268B2EB324F08BF012340E80212002AFE
:10797000E8D18DF807309DF80730002B0CBF11209F
:10798000002002B0704737B550E8013F9DB2C4896E
:1079900025448489A54228BF2D1B0489A54202BF26
:1079A000BFF32F8F002207E0C5EA030540E801542A
:1079B000002CE9D14FF001028DF803200193019AC8
:1079C0000A609DF8031001F0FF0321B1006810FA6E
:1079D00082F003B030BD1846FBE70A884B889A4214
:1079E00009D150E8012FC2EA024240E80123002BEE
:1079F000F7D1012070470020704737B550E8023FAB
:107A00001FFAA3F5C488A54202BFBFF32F8F00223F
:107A10000DE0C48925448489A54228BF2D1BC3EAF3
:107A2000054540E80254002CE8D14FF001028DF8E2
:107A300003200193019A0A609DF8031001F0FF03EF
:107A400021B1006800EB124003B030BD1846FBE7DF
:107A50000A884B889A4209D150E8022FC2EA224292
:107A600040E80223002BF7D1012070470020704727
:107A700010B5034653E8000F0A4643E8002494F08B
:107A8000000FF7D110BD10B5034653E8000F40EAD0
:107A9000010243E8002494F0000FF6D110BD10B5A8
:107AA000034653E8002F42EA010043E8000494F043
:107AB000000FF6D110BD10B5034653E8000F00EAE1
:107AC000010243E8002494F0000FF6D110BD10B578
:107AD000034653E8000F00EB010243E8002494F052
:107AE000000FF6D110BD10B5034653E8002F02EB8E
:107AF000010043E8000494F0000FF6D110BD10B56A
:107B0000034653E8002FA2EB010043E8000494F081
:107B1000000FF6D110BD0121FFF7B5BF0121FFF71E
:107B2000BEBF0021FFF7C7BF10B590B1D0E9012358
:107B300001689B1ADBB20A60013BDBB2FF2B0268D3
:107B400002D10020107110BD11684C1C14600B7024
:107B5000F2E70E20F7E737B5054600240DF10700E0
:107B60008DF80740FFF762FD2A686B68116899423B
:107B70000ED9481E106011F8013CEC68298A01FBFF
:107B80000344AB6811791B1ADBB2994238BF1371F9
:107B90009DF80700FFF76EFD204603B030BD37B5F6
:107BA000054600230DF107000C468DF80730FFF75E
:107BB0003DFD2A681368591C1160E968641A298A16
:107BC000B4FBF1F41C709DF80700FFF753FD03B000
:107BD00030BD826810B504462AB143690168006966
:107BE00098470023A36010BD0EB403B5039921B1DB
:107BF00004AB01AA019300F077F802B05DF804EB42
:107C000003B070470A2938B504460D4602D10D214C
:107C1000FFF7F8FFA3682268591CA160D554D4E986
:107C200001329A4204D32046BDE83840FFF7D1BF65
:107C300038BD00002DE9F84F9846DDE90A431546A6
:107C400082460F460A464FF00109AA420FD2C145AB
:107C500038BFC14613F0010B01D16CB900240126D5
:107C6000B8F1010F1BD908F1FF386E43F8E709F1AD
:107C70000109B2FBF5F2E8E79B070ED5B8F1000F5A
:107C80000CBF30262026A145E9D2013C31465046A2
:107C9000FFF7B8FF002CF6D1E0E72026F3E7B7FBAB
:107CA000F6F39D42E1D9DFF83C80B7FBF6F350468E
:107CB00018F8031006FB1377FFF7A4FF3346AB4217
:107CC000B6FBF5F6F1D2BBF1000F02D00CB1A14525
:107CD00001D3BDE8F88F20215046013CFFF792FF09
:107CE000F4E700BF360903002DE9F74F05461746B4
:107CF0008846002900F03E8118F8011B49B92B7B0A
:107D0000002B00F03781284603B0BDE8F04FFFF7A5
:107D100060BF252940F0B780002698F800302D2B51
:107D2000424608F1010823D0302B24D02B2B25D03C
:107D300000242A2B02F1010123D13B681A1D1B6884
:107D40003A601C440A4613782E2B26D101324FF09C
:107D5000000A104610F8011BA1F1300CBCF1090F0C
:107D60001DD80A2303FB0A13A3F1300A0246F0E7E9
:107D700046F00106D1E746F00206CEE746F00406DB
:107D8000CBE711F8013CA3F130000928DBD80A2227
:107D900002FB0434303C0A46CBE74FF0000A12F8ED
:107DA000011B01F0FB0068289046F8D0782909D81B
:107DB0006F290CD8632962D022D8252963D058298D
:107DC00000F0888098F80030002B95D197E7703943
:107DD0000829F7D801A353F821F000BF4F7F020014
:107DE000C57D0200C57D0200E57E0200C57D020062
:107DF000C37E0200C57D0200C57D0200D57E020063
:107E0000642901D06929DDD13A68D2F80090111DAA
:107E100089EAE9723960A2EBE9724FF0010B092A95
:107E200035DCD34538BFD3462CB1B9F1000F01DBA7
:107E3000720700D5013CB30702D5BAF1000F03D099
:107E4000F00701D44CBB0024B9F1000F2DDAC9F1C1
:107E500000092D212846FFF7D5FE06F00302022A6D
:107E600004D1BAF1000F01D11CBB0024CDE90046BA
:107E700053460A2249462846FFF7DCFEA2E73B6844
:107E80001A1D19783A602846FFF7BCFE9AE70A23C4
:107E90000BF1010BB2FBF3F2C1E7A345D4D22021D1
:107EA0002846013CFFF7AEFECCE77107D5D52B2164
:107EB000D0E7A345DAD230212846013CFFF7A2FEE5
:107EC000D2E73968CDE900460A1D3A6053460A22D6
:107ED0000968D0E739680A1D3A60CDE90046534683
:107EE0001022F5E73B681A1D3A6016F00106D3F838
:107EF000009024D1B9F1000F03D0484608F035F8BE
:107F00000646B4421DD809F1FF3919F8011F0029AE
:107F10003FF458AF2846FFF775FEF6E728460136CE
:107F2000FFF770FE19F806100029F7D1A642BFF43A
:107F300049AF20212846013CFFF764FEF6E7002602
:107F4000F0E720212846013CFFF75CFED9E73B68BB
:107F50001A1D3A60302128461C68FFF753FE78212D
:107F60002846FFF74FFE00220823CDE900322146C4
:107F7000102280E703B0BDE8F08F00BF2DE9F84F75
:107F8000B0F806A04579D2F800B09DF828900AFB19
:107F900005F5043D88460BEB0301A94203F10404F7
:107FA00088BFA5EB030BB4FBFAF607460AFB1644A1
:107FB000C2F800B04EB9AAEB04055D4528BF5D4686
:107FC000BBF1000F04D1BDE8F88F3F68013EF1E737
:107FD000043408EB06003C442A46B9F1000F0DD0EA
:107FE0002146ABEB050B07F042FFDA452E443F6814
:107FF00055464FF0000428BF5D46E1E701462046A4
:10800000EFE7FFF791BDF8B546790146721E0546C8
:10801000002393422D6803D30024A64202D8F8BD62
:108020000133F6E70F682846FFF7B9FD01343946FA
:10803000F3E72DE9F843068ACD1C0746FFF78BFDD1
:10804000043E35440446B5FBF6F5F0B14FF48073B9
:10805000EDB28380C680013D076081464FF0000885
:10806000A84512D23846FFF776FD064648B1637937
:108070000133637108F10108C9F800000760814607
:10808000EEE72046FFF7BFFF34462046BDE8F88301
:1080900001210430FFF727BD10B50121044604304B
:1080A000FFF72DFDC0B220B92046BDE81040FFF714
:1080B000AABF10BD1FB503920022009203AAFFF7CA
:1080C0005DFF05B05DF804FB1FB50392012200922D
:1080D00003AAFFF753FF05B05DF804FB41DF7047CB
:1080E000064B10B500241C70054B1C60BFF35F8F5E
:1080F0000449054800F0F4F8204610BD5037002030
:1081000054370020500903004837002007B50023EA
:108110000DF107008DF80730FFF788FAF1EE103AFD
:1081200023F09F03E1EE103ABFF35F8F0A4B40222A
:10813000C3F884219DF80700FFF79CFA07F080FA46
:1081400020B103B05DF804EBFFF7C8BF20BF40BF0C
:1081500020BF03B05DF804FB00E100E00268136893
:108160005268934291BFD01A80680130801888BF4E
:10817000C01A7047036881681A685B688B4234BF15
:1081800001330023D31A58425841704773B5002376
:1081900004460DF107000D468DF80730FFF746FA4B
:1081A0002046FFF7E7FF10B1237C002B3BD123686B
:1081B000A1685E685A688A4234BF013200225A6060
:1081C00028B11A688A4234BF013200221A60E2687C
:1081D0006368511E072920D8DFE801F004101F143E
:1081E0001F1F1F182A789A552046FFF7B7FF2368EC
:1081F0009A68824200D29860002415E02A8823F809
:108200001620F1E72A6843F82620EDE7D5E90001BA
:1082100003EBC603C3E90001E6E7294602FB06308B
:1082200007F025FEE0E704249DF80700FFF722FA97
:10823000204602B070BD036818685B68C31A5842D4
:108240005841704773B5002305460DF107000C46F1
:1082500016468DF80730FFF7E9F92846FFF7EBFFE0
:10826000002832D12B6819682EB91A68A868824292
:1082700038BF561C1E60EA686B68501E07281ED85F
:10828000DFE800F0040E1D121D1D1D165B5C23703F
:1082900000249DF80700FFF7EDF9204602B070BDFD
:1082A00033F811302380F3E753F821302360EFE7F0
:1082B00003EBC103D3E90023C4E90023E8E701FB92
:1082C0000231204607F0D3FDE2E70524E1E78368A9
:1082D00000225A60C3E904229A60DA601A6070478B
:1082E0000B684A684360934208BF0023016008BFDF
:1082F00043607047436843B10268916852680B4419
:108300009342436004BF00234360704770B54468E4
:1083100006460D46206818B1B3682946984718B933
:1083200023682B60256070BD2468F3E743681868F4
:1083300008B102681A60704743681868704743685C
:10834000186800B97047884203D102681A6001209A
:10835000704703460068F4E710B50D49A1F5947223
:10836000914201D800200FE08C1AE30F03EBE403E5
:108370005B1002EBC30452F83330834205D802D2BB
:1083800004F10802ECE7606810BD2146E8E700BF91
:108390005C0E030008B5FFF7DFFF024B002808BFA3
:1083A000184608BD1F0D030003462AB110881A465F
:1083B00019448A4203D170474FF6FF70F7E712F86D
:1083C000013B40BA80B25840C0F30313584080EAE2
:1083D0000033580100F4FF509BB25840E9E7000019
:1083E00070B5064D0646002455F8043B0BB13046E7
:1083F00098470134042CF7D170BD00BF64370020CA
:108400004388033300EB830399420BD382884FF6F2
:10841000FF739A4208D0038833B18068431C5842E6
:10842000584170470220704701207047033080B2E6
:1084300040F2FE33984230B51FD8134B1A783AB940
:108440001C895D892C440444A4B2B4F5806F0AD918
:108450001A7DAAB99A8BDC8B2244024492B2B2F5FF
:10846000806F0DD801220A801446142202FB0433C7
:108470005A8910445881002030BD48F20860FBE75B
:1084800048F20660F8E700BF983700200B4A0C4915
:108490005388142000FB0311CB6833B904204968CA
:1084A00010700122074800F025BF0749052313700B
:1084B00002238B80012209680023F3E77C37002028
:1084C00098370020282A00206038002007B50023B4
:1084D00005490093054A09680548082300F070FE25
:1084E00003B05DF804FB00BF60380020680E030095
:1084F000282A002007B5002301460093034A0448B8
:10850000082300F05DFE03B05DF804FB600E03007D
:10851000282A002013B500230C4600930146084A80
:108520000848042300F04CFE38B9074B142101FB26
:10853000043101230B7402B010BD48F20D60FAE75C
:108540005C0E0300282A00209837002037B50A481F
:108550000A4B42689C8819685388032503330570C9
:108560009BB2002000909B0001EB8401044800F0C6
:1085700027FE03B030BD00BF7C37002060380020EC
:10858000282A002010B501460448FFF7FCF91C22F8
:108590000446002107F094FC204610BD4C38002012
:1085A00068B10268084B9A4209D14068074B98426B
:1085B00007D00133984214BF0320012070470320E5
:1085C00070470020704700BFDEC0ADDEFE011EF127
:1085D0002DE9F0410D460223154F2B80164600F57C
:1085E000805100F108044FF001088C420ED223683C
:1085F00001330BD02046FFF703FF48B10EB186F8D8
:108600000080022809D14FF480632B80BDE8F081FF
:10861000A3683A68934200D93B602B886288033391
:1086200013442B806388033304EB8304DDE700BF2E
:108630009037002038B5144B14220D4602FB003051
:108640002B68446804F58051A3B15C88033403EBC4
:1086500084048C4215D22368013312D02046FFF7E0
:10866000CFFE012808D002280BD00028F1D12C60C1
:10867000012038BD0834ECE76388033304EB83043E
:10868000E7E70020F5E700BF98370020426873B5A0
:1086900004460D466AB3234BD9688A4229D31B6925
:1086A0009A4226D812F0030323D11F490089098971
:1086B00088421ED12068916888421AD11B484168BF
:1086C0008A4203D901F580518A420DD381698A42D9
:1086D0000CD901F580518A4208D201222A80B3FACE
:1086E00083F0400902B070BD1A46F7E748F209630B
:1086F000F5E700262E800196288801A9FFF79AFF4A
:1087000030B92B8801339BB2012B2B80F3D9E9E7D9
:10871000019B226899689142EED16360024B1B89EC
:108720002381DFE7282A00207C37002098370020AB
:108730002DE9F8431C461D4B1B7806460F4615468F
:1087400073B382B37CB3DFF86C804FF01409A38855
:10875000012B02D948F2096020E009FB03F318F865
:1087600003302BB9A0882146FFF764FF20B92060B1
:10877000A3880133A380EAE723681EB19988328871
:108780009142EFD11FB119883A889142EAD19A6893
:10879000C5E90023064B1B892B810020BDE8F88327
:1087A00048F20160FAE748F20460F7E77437002006
:1087B0007C3700209837002008B5074B5888191DD2
:1087C000FFF738FF18B1BDE80840FFF7BFBEBDE8AE
:1087D0000840FFF75BBE00BF7C3700202DE9F04763
:1087E000A24FDFF8AC8288B006463B6823B9A048A8
:1087F0004146FFF702F938603D6829784B1E052B8A
:1088000007D8DFE813F020007A007A000C010C0191
:10881000630148F20E641422002103A807F050FB04
:1088200041F61D539C4208BF00243B6804941A780B
:10883000023A042A00F20282DFE812F0E301EF01BB
:108840001102190220022EB18A4B00225A604FF405
:108850000644E0E72B79032B1CD8DFE803F0140271
:108860002A35854A1378022B1AD0137D022B4FF03C
:10887000010317D114214B43D1180020D05448686C
:10888000FFF738FE03E001232B71FFF71FFE0028DE
:1088900000F0BF80774B00225A6048F20D64BAE7BF
:1088A0000023E7E7734A13700023536041F61D5419
:1088B000B1E772497248002302222B718A8009684D
:1088C000012200F017FDE2E76C4C00262E712068B3
:1088D000FFF710FE6B4BDFF8A0C15B882568142200
:1088E00053430CEB03020CF8036051685560A588F4
:1088F000158102222160A280C9E7B5F814A0AA7DE3
:10890000DFF87491AEB1022AEB8806D9142101FB7D
:108910000A91DA1C088902440A81142202FB0A998E
:10892000C3F57F43B9F80A20FD331344A9F80A3090
:108930008DE7142303FB0A9318895C6804EB800419
:10894000062A69D8DFE802F0274E36441D5A040093
:1089500041F61D54AA7DEB88022A06D9142101FB99
:108960000A91DA1C088902440A81142202FB0A993E
:10897000C3F57F43B9F80A20FD331344A9F80A3040
:1089800049E74148414900234360AB690360FFF771
:108990007DFE00285BD00223AB75002300930423E7
:1089A000EA182146364800F00BFC002831D048F286
:1089B0000D64CFE72B69002B14BF03230123AB7594
:1089C0000023009305F10C02042304F10801E9E7F8
:1089D0000123AB750022EB8800922A699B0004F109
:1089E0000C01DFE703290CBF05230623AB75002329
:1089F0000093042305F10802E118D3E70623AB75C1
:108A0000224B1988204B5868FFF784FD0446002844
:108A1000A0D108B0BDE8F08748F20E649AE7002EB6
:108A20007FF415AF2B79012B34D0022B3FF43EAFEE
:108A3000002B7FF4EEAE02232B710DF10A01EB68DF
:108A4000039303A8CDE90466FFF720FE10B948F2AE
:108A50000964E0E60498BDF80A108388EB80038877
:108A60002B81FFF757FD044629E000BF9437002013
:108A70004C380020743700209837002060380020E0
:108A8000282A00207C370020583700206C3800202E
:108A90008C370020DFF8009203AA4B463146A81D10
:108AA000FFF746FE044670B9B9F804100498FFF7C2
:108AB00031FD044648F209639C423FF4F7AE002CB6
:108AC0007FF4A9AEA5E7C9E90066F3E7002E7FF4BD
:108AD000BEAE6C4B1A7BBAB11E731A78013A062AE5
:108AE0003FF697AE01A151F822F000BF978B02002C
:108AF000BD8B0200DB8B0200E18B020013880200B9
:108B0000E78B0200F98B02001A78072AE5D801A149
:108B100051F822F0358B0200DB8A0200DB8A02006A
:108B20005B8B02006F8B0200938B0200938B020021
:108B3000578B02001A89544901321A8100225A8047
:108B40001A730A78B2FA82F252099A720A7DB2FA5C
:108B500082F25209DA72012207E04C4958688A8889
:108B60004088033202448A8002221A70B5E75C888A
:108B7000454A4649142505FB04220868546850609C
:108B80008888108102200C608880002111740622E0
:108B9000EBE70722E9E79A7A32B9DA7A8AB9002252
:108BA0001A705A805A6081E6374900229A72CA6860
:108BB000002AF2D1097C0029EFD05A80FFF7FCFD92
:108BC00051E70022DA72304A116A0029E7D192F89F
:108BD0002420002AE3D00122EFE7FFF7B7FC42E7A9
:108BE000FFF754FC3FE75A88274B142101FB02335F
:108BF0005868FFF77FFC36E700225A60FFF766FCF3
:108C000031E701228DF80C201A89ADF818209A88D6
:108C1000DB68ADF81A20059310E002228DF80C20D5
:108C20001A89ADF818209A88ADF81A20DA689B7D69
:108C300005929A1F534253418DF81C3003A8FFF749
:108C4000CFFB0026414612483E60FEF701FF114867
:108C50000121FEF754FF00287FF4C7ADD9E60322B7
:108C60008DF80C20DA88ADF818201A89D0E7042294
:108C70008DF80C20DB88ADF81830DFE705238DF880
:108C80000C30DBE77C37002098370020603800206C
:108C90004C3800205C380020703800204068FFF716
:108CA0009DBD000008B505480121FEF710FF18B969
:108CB000BDE80840FFF792BD08BD00BF5C3800204A
:108CC0002DE9F34198460023ADF80230414B1B7863
:108CD00006460D46002B71D0002972D009884FF648
:108CE000FF73994270D06B88002B6DD06B689B0727
:108CF0006DD142B92F8969463846FFF797FB30B1ED
:108D000002B0BDE8F08113885788ADF8003001A8A3
:108D1000FFF738FC044660B9BDF800202E4B142143
:108D200001FB023358890338C01B588148F20760A1
:108D3000E6E780F8008000238375BDF80030838269
:108D40006B68036101212548FEF7CDFE2B88238146
:108D5000B8F1030F6B88A38001BF0423A3753368A8
:108D6000A361E06000220621E780201DFFF71CFBC5
:108D70000DF10202ADF80200042104F10C00FFF72E
:108D800013FBA968ADF80200890068680DF10202C2
:108D9000FFF70AFB01A9ADF8020060811048FEF759
:108DA0001CFE3EB10023E2687360B3720D4B32606B
:108DB0001B893381FFF776FF0020A1E748F20160AD
:108DC0009EE748F204609BE748F2036098E748F2A8
:108DD000026095E774370020983700209037002014
:108DE0004C3800207C37002008B50346074802684D
:108DF000042A08D00168064A42F821300121FEF712
:108E000072FE002008BD48F20B60FBE768380020C6
:108E1000643700202DE9F04F89B01422002103A807
:108E200007F04EF87A4B1B7803F0FF0B3BB103A819
:108E3000FFF7D6FA0027384609B0BDE8F08F744B2B
:108E4000181DFEF768FE0028F4D1DBF8F83FDFF8C4
:108E5000E0A15C1C08BF4FF010234FF0805208BF08
:108E60005B6911695269581C08BF02FB01F3CAF81B
:108E700010306849A3F5405300225046CAF80C3020
:108E800000F06CF907460028D5D11C2362496348DD
:108E9000DFF8A0918C22FEF741FD0323B8463D4642
:108EA00001933C46DAF80C6046443046FFF778FB05
:108EB000012862D0032817D000283DD158494FF02F
:108EC000140C0CFB04FC01EB0C0201F80C005660C6
:108ED0000CF110020CF1080C0A4430466144FFF713
:108EE00077FB45F0020545E03268531C02D04D4B3C
:108EF0009A4234D1321D06F58051106801302ED1CE
:108F000004329142F9D1D9F800203AB90222C9F8C5
:108F10000060A9F804204FF0010B0BE0142262431B
:108F20003F4B0220991898543F4A4E6054800134B8
:108F30000881A4B245F0010508F58058B8F5405FF6
:108F4000B0D1019B012B98BF0025EDB2022D03D0BB
:108F5000062D32D0002D39D148F20A676BE7019B0C
:108F60002F495A1E93B21422624388180193466017
:108F7000032088540134A4B2DEE7BBF1000F0DD00A
:108F8000274B14226243991802209854D9F80020E4
:108F90004A60254A088154800134A4B20022234942
:108FA000C9F800603046FFF713FBB9F80420022A25
:108FB0000CBF042208221543BEE7154A0123137093
:108FC00003A800235360FFF70BFA34E702A8FFF76A
:108FD000D9FAC8B10123013D03700A2D09D8DFE891
:108FE00005F006080608070807080F110F00002300
:108FF000037102A90948FEF7F0FCFFF753FE1AE7D8
:109000000323F5E70223F3E748F2076713E700BFFE
:10901000743700204C100300C03700204C3800206B
:1090200098370020DEC0ADDE7C3700206438002099
:10903000282A0020603800202DE9F3410D4604461F
:1090400068B361B301A9FFF721FB58B3666800223A
:1090500006213046B6F806807788FFF7A5F9791C17
:10906000ADF806000DF10602890006F10800FFF7D1
:109070009BF9804519D1BDF804300D48142202FB3C
:10908000030001210C30FEF72EFD63682E600C33C7
:109090006B600123A372002002B0BDE8F08148F2AA
:1090A0000460F9E748F20960F6E748F20C60F3E77C
:1090B0009837002013B50446A8B10DF10601FFF75B
:1090C000E5FA98B1BDF806200B4B142101FB0233E1
:1090D000DA6872B1A27A62B1DA680020013ADA6025
:1090E000A07202B010BD48F20460FAE748F20960CD
:1090F000F7E748F20560F4E79837002002230022E2
:10910000FFF7DEBD104B1B7837B505469BB1A8B104
:1091100001A8FFF737FAA0B1042303702B68C360DE
:109120000024047101A90948FEF757FCFFF7BAFDB6
:10913000204603B030BD48F20160FAE748F204600F
:10914000F7E748F20760F4E7743700204C38002056
:109150000B46002102460846FFF7EABA13B50B4654
:10916000114680B9104B1148114AC01A0E23C0088D
:109170000093104B0004104940F00100FDF73BFC48
:109180000E2002B010BD4BB9074B08480B4AC01A5D
:10919000C0080E2300930004064BECE703601B6835
:1091A00002B0BDE810401847180603008806030007
:1091B000700E03002C100300750E0300A40E0300B4
:1091C0002DE9F743DDF8288088B93E4B3E483F4AF9
:1091D000C01AC0080E243E4B009400043D4940F0E4
:1091E0000100FDF708FC204603B0BDE8F0834AB952
:1091F000344B3548384AC01AC0080E24344B00940A
:109200000004EBE7D0F800E0BEF1000F09D12D4BD0
:109210002D48324AC01AC00808242D4B009400047F
:10922000DCE74BB9274B28482D4AC01AC00809244F
:10923000274B00940004D1E74568D5F80490B3FBB0
:10924000F9F509FB15354DB11E4B1F48254AC01ACB
:10925000C00809241E4B00940004BFE78D0709D005
:10926000184B1948204AC01AC0081024184B009403
:109270000004B3E712F0030F09D0124B12481B4A47
:10928000C01AC0081024124B00940004A6E7C56859
:10929000A9420DD34D1EEC180569AC4208D8CDF893
:1092A0002880DEF80C40A44603B0BDE8F0436047D8
:1092B000044B05480E4AC01AC0081024044B009401
:1092C00000048BE71806030088060300700E0300F5
:1092D00019100300750E0300F20E03009E0E03002A
:1092E000B10E0300F80E0300220F03003A0F030033
:1092F0005D0F0300F7B580B92A4B2B482B4AC01AE3
:10930000C0080E242A4B009400042A4940F00100B2
:10931000FDF771FB204603B0F0BDD0F800C0BCF1F2
:10932000000F09D11F4B2048234AC01AC008082447
:109330001F4B00940004E8E74AB91A4B1A481F4A29
:10934000C01AC00809241A4B00940004DDE74568E0
:10935000D5F800E00EF1FF350D4209D0114B12484F
:10936000174AC01AC0081024114B00940004CCE71F
:10937000C568A9420CD34D1E0EFB02540569AC42D0
:1093800006D8DCF81040A44603B0BDE8F0406047C2
:10939000044B05480B4AC01AC0081024044B009423
:1093A0000004B2E71806030088060300700E0300ED
:1093B00006100300750E03009E0E0300B10E03009D
:1093C000840F0300AA0F030029DF704728DF7047CE
:1093D00070B503689E6886B004460D466EB11422CF
:1093E0000021684606F06CFDA3680593237901957A
:1093F0002BB1012B0DD06846B04706B070BD0123DC
:109400008DF8003023690293E36803936369049342
:10941000F1E702238DF80030E3681B030293F5E7C0
:109420000846704700207047024B187A003818BF72
:109430000120704714390020034B187A0122B0FA3A
:1094400080F05A74400970471439002008B510465E
:109450001A4606F00CFD002008BD000008B51422D5
:109460000021044806F02CFD0348FEF76AFA0020AC
:1094700008BD00BF143900200439002010B5094C84
:10948000094B43602046FEF746FB40B906F0D8F88A
:10949000064920741C2306488C22FEF73FFA002060
:1094A00010BD00BF143900204010030078380020A0
:1094B0000439002038B5234D234C2B7A3BB923497E
:1094C0002348FEF79AFA206008B9686038BD022385
:1094D00024682B72237973B1012B24D020460321F9
:1094E000FFF776FF00232B726B6018491848BDE820
:1094F0003840FEF7ADBAD4E90523D21AB2F5805F41
:10950000D4E9031028BF4FF480529208012A38BFD3
:10951000012219441844FFF757FF50B11128DDD13B
:1095200001232B72D2E7D4E903031844FFF74EFF5F
:10953000F3E72B7C002BC9D1BDE83840022000F0B6
:1095400009B800BF143900202C3900202839002028
:109550000439002038B5234C237A002B41D0022B4C
:1095600009D1032830D0204B00221B68E2601A7911
:109570003AB1012A22D0637C7BBBBDE83840FFF7BB
:1095800099BFD3E905128D1AB5F5805F94BF5219C2
:1095900002F580529A619142EDD102284FF000030A
:1095A00008BF19462372104B18BF0D211868FFF72A
:1095B0000FFF0E490E48FEF74BFADCE71A6901323D
:1095C0001A615B699A42E7E7E3680133082B01D827
:1095D000E360D0E70023E360DFE7BDE8384006F052
:1095E0001FB838BD143900202C390020283900203C
:1095F00004390020831E012B01D8FFF7ABBF704751
:1096000000F0FD03012B08D1044B00225A74421EC6
:10961000504250411874FFF74DBF70471439002075
:1096200010B5064C201DFEF776FA28B9637C1BB9ED
:10963000BDE81040FFF73EBF10BD00BF1439002049
:109640002DE9F34180460D46104801A916461F46F4
:10965000FEF799F90446B0B118220021043006F053
:109660002FFC2D0B0123237101A90848C4F80080A9
:10967000A760E5606661FEF7B0F9FFF7D1FF002053
:1096800002B0BDE8F0810420FAE700BF04390020F1
:109690002DE9F34180460F460F4801A916461D46A5
:1096A000FEF771F90446A8B118220021043006F033
:1096B00007FC089BA36001A9C4E903670648C4F836
:1096C00000806561FEF789F9FFF7AAFF002002B06C
:1096D000BDE8F0810420FAE7043900204FF0805300
:1096E000D3F83001421C04BF4FF0704393F8E00FF1
:1096F000831F5842584170474FF0704393F8E02F52
:10970000062A09D1D3F8E83FC3F30313033B032B25
:1097100002D8024AD05C70470020704774100300E2
:1097200008B5FFF7DBFF40B14FF080538F4AD3F805
:109730002433C3F30423C2F84035FFF7DDFF10B133
:109740008B4B8C4A5A67FFF7C9FF48B14FF08053E3
:109750004FF08042D3F84432C3F34233C2F83C3571
:10976000FFF7CAFF30B1844AD2F8FC3023F080738F
:10977000C2F8FC30FFF7B2FF40B14FF08043002247
:10978000C3F80C21C3F81021C3F83825FFF7B4FF44
:1097900020B14FF080430322C3F8A025FFF7ACFFB0
:1097A00060B1764B0522C3F810260122C3F8882643
:1097B0000022C3F818263F22C3F814264FF0805326
:1097C000D3F83021511C09BF4FF07043D3F8343126
:1097D00093F8E02FD3F8E83F08BFC3F30313062A3A
:1097E0004DD1033B032B03D8654AD35C002B46D0F5
:1097F0004FF08052634BD2F80414C3F82015D2F80E
:109800000814C3F82415D2F80C14C3F82815D2F89C
:109810001014C3F82C15D2F81414C3F83015D2F86C
:109820001814C3F83415D2F81C14C3F84015D2F834
:109830002014C3F84415D2F82414C3F84815D2F8FC
:109840002814C3F84C15D2F82C14C3F85015D2F8CC
:109850003014C3F85415D2F83414C3F86015D2F894
:109860003814C3F86415D2F83C14C3F86815D2F85C
:109870004014C3F86C15D2F84424C3F87025FFF7E0
:109880002DFF48B14FF080534FF08042D3F858324B
:1098900003F04F03C2F8E43EFFF720FF48B14FF05A
:1098A0008043D3F80024D20744BF6FF00102C3F80D
:1098B00000244FF08053D3F83021062A0ED1D3F87C
:1098C0003431033B032B02D82F4AD35C33B12F4AE8
:1098D000D2F83C3743F48063C2F83C37264AD2F8CA
:1098E000883043F47003C2F88830BFF34F8FBFF362
:1098F0006F8F4FF01023D3F80022002A03DBD3F838
:109900000432002B2EDA224B0122C3F80425D3F8AF
:109910000024002AFBD04FF010221521C2F80012BB
:10992000D3F80024002AFBD04FF010231522C3F8EF
:109930000422174BD3F80024002AFBD00022C3F8DE
:109940000425D3F80024002AFBD0BFF34F8F0A4927
:10995000104BCA6802F4E0621343CB60BFF34F8F31
:1099600000BFFDE70C4B0D4A1A6008BD00300140F6
:1099700000C007400DF0ADBA00ED00E0005000401F
:109980006C10030000C00040701003000010004085
:1099900000E001400400FA05602A00200090D00396
:1099A000054A4FF0A043105CD3F8043523FA00F0C9
:1099B00000F00100704700BF7C100300044B1A5CEC
:1099C000012393404FF0A042C2F80835704700BF12
:1099D0007C100300044B1A5C012393404FF0A0421B
:1099E000C2F80C35704700BF7C10030008B500209A
:1099F000FFF7F0FF0120FFF7EDFF0220FFF7EAFF7E
:109A00000320FFF7E7FF4FF0A0438022C3F80C25A7
:109A100008BD08B50020FFF7D1FF0120FFF7CEFFFA
:109A20000220FFF7CBFFBDE808400320FFF7C6BFC9
:109A3000074A4FF0A041105CD1F804350122824062
:109A400022EA03001340C1F80805C1F80C3570473D
:109A50007C100300014B185C704700BF78100300B6
:109A600038B5074C051E04F1080318BF1C462368CF
:109A70002BB11A6822605B6828469847F7E738BD23
:109A80003839002020B9054B01225A70FFF7E8BF92
:109A9000012802D1014A9070F8E770473039002060
:109AA00020B9034B01225A70FFF7DABF704700BF9D
:109AB0003039002038B50E4C2378B3B90D486360B7
:109AC000A3602361E36000F0E7F8054605F0B8FD08
:109AD00008B900F0EDF801232370074BD3F80034E8
:109AE0000BB10123A370284638BD8525F5E700BFDB
:109AF00030390020859A02000000014037B50D4C36
:109B000000230DF107008DF80730FDF78FFDE368A6
:109B1000013BE360E36833B9074BD3F8005415B950
:109B200000F0D8F8A5709DF80700FDF7A3FD03B07D
:109B300030BD00BF3039002000000140012813B5BE
:109B40000CD0032820D038B9134B0122C3F8802051
:109B5000BFF34F8FBFF36F8F02B010BD0F4C0023C8
:109B60000DF107008DF80730FDF760FD23780BB984
:109B7000FFF7A0FFE3689DF807000133E3600123CE
:109B8000A370FDF777FDE7E700F092F802B0BDE8BB
:109B90001040FFF7B3BF00BF00E100E03039002004
:109BA0001FB503788DF800304368019383688DF802
:109BB0000830C368054A0393054B684653F82130C3
:109BC00052F82110984705B05DF804FB4439002095
:109BD000483900201FB503788DF8003043680193A1
:109BE00083688DF80830C368054A0393054B6846BF
:109BF00053F8213052F82110984705B05DF804FB66
:109C00004439002048390020F0B5194B90F800C0C5
:109C100091F81DE043F82C20164B16460A6943F8CC
:109C20002C20154B03F80CE00C4607460FCC89B0EE
:109C30006D460FC594E80F0085E80F00CDF810C001
:109C4000BEF1000F09D0002E0C4A694608BF32460B
:109C5000381D00F097FD09B0F0BD002E084A694696
:109C600008BF324607F10C0000F05EFBF3E700BFCF
:109C700048390020443900204C390020A19B0200C3
:109C8000D59B020000F18040002382B0036003688E
:109C90000193019B02B07047044A137923B9012153
:109CA0001060918018467047852070475039002019
:109CB000074B1A68D20704D4C02283F8002301227C
:109CC0001A604FF080430122C3F81825704700BF87
:109CD00000E100E04FF0804208B50223C2F80833EB
:109CE0004FF48270FFF7CEFF0123D360D2F818340F
:109CF000DB03FBD408BD00004FF0804110B5D1F864
:109D0000003163B14FF48070FFF7BCFF0D4B587901
:109D10000122C1F8082310B95A711B6898474FF007
:109D20008042D2F8043163B14FF48270FFF7AAFF8A
:109D30000223C2F80833034BBDE810401B68012022
:109D4000184710BD5039002000F1804000F5C04098
:109D5000002382B0036003680193019B02B0704747
:109D6000800000F1A040D0F8002722F44032C0F873
:109D70000027D0F8003743EA0141C0F800177047C8
:109D8000054B4FF0FF32072843F8202084BFC0184E
:109D900080F84820704700BF5839002010B5184996
:109DA00091F8583053BB4FF0FF3222FA03F0C0074E
:109DB00048BFC81803F1010348BF80F83020202BAA
:109DC000F3D10024E0B20134FFF7DAFF0C2CF9D113
:109DD0000C4B0022C0204A6583F80603402018601F
:109DE0004FF4BE70FFF7B0FF074B4FF00040C3F8D1
:109DF0000403012381F85830104610BD0820FCE709
:109E00005839002000E100E000600040034B93F867
:109E10005800003818BF0120704700BF5839002093
:109E2000F0B5394E331893F93030002B69DA8D785C
:109E3000C5F34005002D0BBF082300230C24082484
:109E4000A34201D10420F0BD56F82370013743D15D
:109E500037185CB246F8232087F8304015B9F2185D
:109E600082F848008A78550716D4D70736D582007D
:109E700002F1A042D2F8005725F00205C2F80057BF
:109E8000224FC50800F0070C012202FA0CF217F865
:109E900005C042EA0C027A558A780D7812F0020267
:109EA00025D09B0003F1804303F5C0430002D3F8A3
:109EB000102522F4473222F44072C3F810252D04F5
:109EC000D3F8102500F4F85005F44035284310432A
:109ED000C3F810050020B6E70133B1E74D7800F56F
:109EE000E0724FF0A047AD0047F82250C8E7083CA9
:109EF00046FA84F494F8500040EA851584F85050EE
:109F0000E8E708209FE700BF58390020AC3900205F
:109F100038B5204C251895F93020072A18DD083A65
:109F200044FA82F494F850309B09032B0BD14FF084
:109F3000A043D3F81015C14001F001010231BDE882
:109F40003840FFF70DBF012B0CBF02210321F6E7BC
:109F5000D3B2072B1DD8930003F1804303F5C04310
:109F6000D3F8100540F00100C3F8100502F14000DD
:109F700040B2800080B2FFF7E7FE51B195F9303072
:109F800054F823302BB1012303FA02F2024BC3F839
:109F9000042338BD58390020006000404FF0A04332
:109FA000D3F8103523FA00F000F0010070470000EC
:109FB0002DE9F74F00244E4D01944FF4807201219A
:109FC00002F1804303F5C04390B21B68012B06D118
:109FD000D5F804330B4202D0FFF7B6FE0C4304322F
:109FE000B2F5907F4FEA4101EAD1414BD3F87C3181
:109FF000012B0CD14FF4BE70FFF7A6FE4FF0A0432B
:10A0000044F00044D3F820250192C3F82025E3B2A0
:10A01000D3B1384F00250126344210D0AB0003F1F4
:10A02000804303F5C043D3F81005D3F8101557F853
:10A03000253023B1C1F30141C0F304209847013515
:10A04000082D4FEA4606E7D1002C48DA294D4FF09B
:10A05000A048294E4FF00009012716F9013B5A1C70
:10A0600031D0C3F3C20202A90A44DCB212F8042CB4
:10A0700003F03F0A03F0070307FA03F31A4222D062
:10A080000AF5E073504658F82330C3F3014BBBF197
:10A09000020F0CBF03210221FFF762FE07FA0AF349
:10A0A000C8F8203505EB0A0393F9303055F8233012
:10A0B0004BB1A109032904D0BBF1020F12D1012930
:10A0C00001D15046984709F10109B9F1040FC4D1F3
:10A0D000D8F820350193C8F82035002BB9D103B04A
:10A0E000BDE8F08FBBF1030FEDD10229E8E700BF17
:10A0F0000060004058390020A8390020014B1B683F
:10A10000184700BFB43900200E4B984237B50C46B3
:10A1100002D0002003B030BD00230DF107008DF800
:10A120000730FDF783FA084B1D7915B901221C6031
:10A130001A719DF80700FDF79DFA002DE9D0112056
:10A14000E8E700BF00200040B4390020002343505E
:10A1500082B043580193019B02B070470A4610B584
:10A160004FF48E71FFF7F2FF136A9168C95C136AAE
:10A1700001331362C0F81C1510BD024608B5006813
:10A180004FF49271FFF7E2FF10684FF48471FFF70C
:10A19000DDFF136801221A6008BD8B690A4610B5FD
:10A1A0004FF4847123B9FFF7D1FFD0F8183510BDF3
:10A1B000FFF7CCFF536AD168D0F81805C854536A2A
:10A1C00001335362F3E700001FB501238DF800301F
:10A1D000044BCDE90110D3E900126846904705B061
:10A1E0005DF804FBBC39002030B54D4DD5F8043383
:10A1F0009A0585B051D5D5F82431002B4DD04FF4B8
:10A2000092712846FFF7A2FF4FF40173C5F8083397
:10A21000444B93F829200AB901226A60404902227E
:10A220008DF80020D1F88024C1F8802403929A6927
:10A230000292DA6801920022C3E906226846D3E955
:10A24000001290473648D0F81C315BB1354A51694D
:10A25000136A99424DD992F82830002B49D1114602
:10A26000FFF77CFF2E48D0F84431002B56D04FF436
:10A27000A271FFF76BFF2B4B93F829200AB1012243
:10A2800002609A69002A49D0586AD96800229A6106
:10A2900005B0BDE83040FFF797BFD5F804335B0742
:10A2A000D0D5D5F80831002BCCD01E4C1C48214607
:10A2B000FFF773FF636AA2699A42C3D1E369E16859
:10A2C0004BB1A3612369E3600023606AE3616362C9
:10A2D000FFF77AFFB6E794F829300BB901236B60DA
:10A2E0000F4B4FF40172C3F808230023606AA36187
:10A2F000EEE70B484FF48E71FFF728FF5369002BF0
:10A30000B0D051690291002391688DF8003001911D
:10A3100053616846D2E900139847A3E705B030BD02
:10A3200000200040BC3900202DE9F843534D90F83F
:10A3300004802C2303FB0853064693F82A300C466E
:10A340009146002B40F096804D490068FFF7DCFEF7
:10A350000746002840F0908022683068511C0BD0DE
:10A360004FF0A04101239340C1F8083502F5E07396
:10A370004FF0030C41F823C061684B1C1FBF01F56F
:10A38000E0734FF0A04C4FF0000E4CF823E0A369AF
:10A39000C0F8243594F814C0637DBCF1010F4CEA79
:10A3A0000303C0F86C35C0F81415C0F80C251DD196
:10A3B000A268531C1FBF02F5E0734FF0A0414FF09D
:10A3C000000C41F823C0E368591C0BD04FF0A04C9F
:10A3D00001219940CCF8081503F5E0714FF0030E08
:10A3E0004CF821E0C0F80835C0F810252C2202FBFB
:10A3F00008F2AB18C3F804902369AB50B9F1000F11
:10A4000020D04FF48E71247FFFF7A0FE4FF4A2718D
:10A410003068FFF79BFE32681A4BC2F80433130B07
:10A4200042F307326101002AC9B21EDB16488418C4
:10A4300084F800130121520903F01F0301FA03F30A
:10A4400040F8223033680422C3F800252C2303FB94
:10A4500008530022C3E9062283F829205A61012209
:10A4600083F82A203846BDE8F883084A03F00F0332
:10A47000D154E7E70827F5E71127F3E7BC390020B7
:10A48000E9A102008000020000E100E014ED00E01C
:10A490000279044B2C2101FB02335869003818BFA4
:10A4A00001207047BC3900202DE9F84F064690F88E
:10A4B000048089469246FFF7EBFF044600283CD112
:10A4C000204F2C2508FB057B4FF48E71CBF814A090
:10A4D000CBF80890CBF820008BF828003068FFF705
:10A4E00035FE3068012383605946FFF737FEDBF8FD
:10A4F00004305D461BBB3068DBF814402B6A9C427D
:10A5000011D83368D3F81C21002AFBD00122DA606D
:10A5100000202C2303FB087700237B61BDE8F88F24
:10A5200095F828303BB9D0F81C31002BF8D05946AB
:10A53000FFF714FEE2E70F20EBE71120EEE72046DD
:10A54000ECE700BFBC3900202DE9F0473A4D077910
:10A550002C2303FB075306465C6824B103684FF4C1
:10A560000170C3F808032C2303FB0753986950B10B
:10A57000D869002841D024B133684FF40172C3F880
:10A580000423112436E09A61D9605862D8612C23E3
:10A5900003FB075393F829301BB910B93046FFF776
:10A5A000ECFD4FF02C0808FB075A3068DAF804304D
:10A5B000002B37D14FF4A271D046FFF7C7FD3068AA
:10A5C000D0F82491D0F80831D0F84441CBB914B96F
:10A5D000B9F1000FF3D02C2303FB07550023AB6127
:10A5E000B9F1000F24D12CBB95F829103368012252
:10A5F000B1B11A602046BDE8F0871961DA61012027
:10A60000C5E7B9F1000FE6D1002CE4D14146FFF7D0
:10A61000C4FDDAF82430DAF818209A42CFD8DAE705
:10A620005A60E7E74FF40173C0F804330024E1E710
:10A630000324DFE70F24DDE7BC390020002343506B
:10A6400082B043580193019B02B070471FB50123AC
:10A650008DF80030044BCDE90110D3E900126846B3
:10A66000904705B05DF804FBE83900207FB5434A08
:10A67000D2F82461002E60D010464FF49271FFF79B
:10A68000DDFF02238DF80030D2F88034C2F8803428
:10A690000393D2F83C350293394BDA6801920022D9
:10A6A000C3E906226846D3E9001290473348D0F840
:10A6B000443173B14FF4A271FFF7C0FF304B9A6978
:10A6C0003AB10022C3E90622D968D0F83C05FFF769
:10A6D000BDFF2A48D0F82031ABB14FF49071FFF79D
:10A6E000ADFF0123C360264B5A6962B1D0F84C1507
:10A6F0000291002299688DF8002001915A61684604
:10A70000D3E9001290471D48D0F858319BB14FF45F
:10A71000AC71FFF793FF1A4B5A6962B1D0F84C1530
:10A720000291002299688DF8002001915A616846D3
:10A73000D3E90012904704B070BDD2F81031002B5D
:10A74000B4D04FF488711046FFF778FF0C4BD2F865
:10A750003C0599698842A9D1DC69D96864B1D2F80D
:10A76000005225F02005C2F800521A699C61DA6097
:10A77000DE61FFF76BFF99E79C61FAE7002000407C
:10A78000E83900202DE9F8435A4E90F8048024233C
:10A7900003FB0863044693F820300D469146002BD6
:10A7A00040F0A38054490068FFF7AEFC074600283C
:10A7B00040F09D802A682068511C0BD04FF0A041CA
:10A7C00001239340C1F8083502F5E0734FF0030C04
:10A7D00041F823C069684B1C1FBF01F5E0734FF0BF
:10A7E000A04C4FF0000E4CF823E0AB69C0F82435C4
:10A7F00095F814C06B7DBCF1010F4CEA0303C0F85F
:10A800006C35C0F80C25C0F814151DD1AA68531C6E
:10A810001FBF02F5E0734FF0A0414FF0000C41F86C
:10A8200023C0EB68591C0BD04FF0A04C012199407C
:10A83000CCF8081503F5E0714FF0030E4CF821E059
:10A84000C0F80835C0F81025242202FB08F2B3181E
:10A85000C3F804902B69B350B9F1000F2FD04FF417
:10A8600088712A7FFFF7EAFE20684FF49071FFF7A6
:10A87000E5FE20684FF49271FFF7E0FE20684FF488
:10A88000A271FFF7DBFE4FF4AC712068FFF7D6FE34
:10A8900023681A49C3F80413190B43F30733520111
:10A8A000002BD2B21CDB1648C51885F80023012204
:10A8B0005B0901F01F0102FA01F140F8231023683F
:10A8C0000822C3F80025242303FB08660023C6E9F9
:10A8D00006337361012386F820303846BDE8F883DB
:10A8E000084B01F00F015A54E9E70827F5E7112753
:10A8F000F3E700BFE83900206DA602001003420014
:10A9000000E100E014ED00E00279044B242101FB9A
:10A9100002335869003818BF01207047E839002019
:10A9200001F06043B3F1005F2DE9F0470646884629
:10A9300092463BD190F80490FFF7E6FF04460028CA
:10A9400036D11D4F3068242505FB09754FF49071F1
:10A95000C5F814A0C5F80880FFF770FE4FF4AC717D
:10A960003068FFF76BFE33686A69A968C3F844155D
:10A97000C3F8482501229A606A68DAB9D3F8202121
:10A98000D3F858011AB90028F8D00F2007E00028A2
:10A99000FBD10122DA60D3F85821002AFBD024230E
:10A9A00003FB097700237B61BDE8F0871020FBE7FC
:10A9B0001120F9E72046F7E7E8390020F8B501F063
:10A9C0006043B3F1005F04460F465ED10379304D1A
:10A9D000242101FB0351496821B100684FF404763A
:10A9E000C0F80863242000FB03539E6956B1D86960
:10A9F000002839D021B123684FF40472C3F804232E
:10AA0000112030E09A61DF60DE6120684FF48871C8
:10AA1000FFF714FE20684FF4A271FFF70FFE2368C2
:10AA2000C3F83475C3F8382516BB01221A6024799F
:10AA3000242202FB045252680ABBD3F81011D3F847
:10AA40004421D3F82401114302D10028F5D00A464D
:10AA5000242303FB04550023984218BF03209A4285
:10AA6000AB6118BF0F20F8BD1F61DA610126CCE78A
:10AA7000D3F8002242F02002C3F80022D7E74FF4B7
:10AA80000472C3F804230020EDE71020EBE700BFB9
:10AA9000E839002008B5094B1B7853B10020FEF7B8
:10AAA00099FF0120FEF796FFBDE808400320FEF75E
:10AAB00091BFBDE80840FEF799BF00BF0C3A0020E7
:10AAC000F8B57A4C237805461BB100232370FFF7B5
:10AAD000E1FF172D00F28780DFE805F00C17174221
:10AAE0005364757F878C878C949999999999C3C879
:10AAF000D0D8E3E3FFF7CEFF6D48FCF7B4FB6D4B16
:10AB0000002204461A702046F8BD0020FEF748FFD8
:10AB1000F0B10020FEF75EFF022D0CBF4FF4E164A0
:10AB20004FF47A64634B1D7000254FF400464FF4D8
:10AB30007A7029464FF4FA620023E4FB060104F020
:10AB400001FF2A460146BDE8F8405948FCF773BBAF
:10AB5000FEF734FF022D0CBFC8244FF4C874E1E7A0
:10AB60000020FEF71DFF40B10020FEF733FF4FF439
:10AB70004874504B03221A70D6E7FEF71FFFC82413
:10AB8000F7E70020FEF70CFF38B10020FEF722FFA8
:10AB90004FF47A64474B0422EDE7FEF70FFF4FF4C2
:10ABA000C874F7E70020FEF7FBFE48B10020FEF76F
:10ABB00011FF404B05221A7040F6CD410022C2E73A
:10ABC000FEF7FCFEF5E70020FEF732FF394B0622C8
:10ABD0001A70002240F26661B5E70020FEF7EEFE33
:10ABE000344B07221A7000248DE701202070FEF7F5
:10ABF0001FFFEEE701202070FEF71AFF00224FF43E
:10AC00000051A0E7FEF705FF2A4B0C22EAE72A488D
:10AC10002A4EFCF728FBD5F1110504461CD0D8B903
:10AC2000012D13D0C820454321464FF400474FF46F
:10AC30007A704FF4FA620023C5FB070104F082FE2C
:10AC4000224601461C48FCF7F6FA04460220FEF7AD
:10AC5000B5FE0123337056E70220FEF7BBFE00234A
:10AC6000F8E7FFF717FF134B1222BBE7FFF712FFBE
:10AC70000020FEF7A3FE0F4B1322B3E7FFF70AFFF6
:10AC80000120FEF79BFE0B4B1422ABE7FFF702FF00
:10AC90000020FEF793FE0120FEF790FE054B1522E3
:10ACA000A0E7FEF7B6FE034B1D709CE7603A00205C
:10ACB000303A0020613A0020103A00200C3A00207F
:10ACC00010B5002914BF03240024FEF7C3FE800042
:10ACD00000F1A040D0F8002722F44032C0F800274D
:10ACE000D0F8003743EA0443C0F80037002010BD15
:10ACF000044B1B6813F0010301D0FFF7E1BE1846B7
:10AD0000704700BF5C3A0020032811D8012A0AD1FD
:10AD100001290FD100F10E02D2B20D4B00EB400021
:10AD20001A54002070470129F7D0022904D049B1F4
:10AD3000072070470022F8E7054B00EB400018445D
:10AD40004270EEE7024B00EB400018448270E8E7E7
:10AD5000503A0020032802D80121FFF7B1BF062096
:10AD6000704708B5012202210020FFF7CDFF08B18E
:10AD7000072810D1072202210120FFF7C5FF08B1E3
:10AD8000072808D100210A220846FFF7BDFF10B1AD
:10AD9000072808BF002008BD0388102B10B502D07B
:10ADA000112B1ED010BD1A4C2168B1B901220846E2
:10ADB000FFF7AAFF08B1072824D1072202210120AA
:10ADC000FFF7A2FF08B107281CD1042202210020AE
:10ADD000FFF79AFF08B1072814D1236801332360D5
:10ADE000E0E70B4A1368013B1360002BDAD1FFF751
:10ADF000B8FF0028D6D0074B1B68002BD2D0BDE887
:10AE000010401847034B1B68002BE6D09847E4E737
:10AE1000683A0020643A002008B50020FFF79AFF46
:10AE200008B1062806D10120FFF794FF10B10628CB
:10AE300008BF002008BD6CDF70476DDF704775DF0D
:10AE4000704776DF70477FDF70478FDF7047000005
:10AE5000234A2449136801331360234B1A680132D3
:10AE60001A601A6901321A615A6901325A619A6983
:10AE700001329A611A6A01321A625A6A01325A62BE
:10AE80009A6A01329A62DA6A0132DA628A69013AAE
:10AE90008A611A680A2192FBF1F001FB10220AB9BB
:10AEA00001225A601A68642192FBF1F001FB102222
:10AEB0000AB901229A601A684FF47A7192FBF1F094
:10AEC00001FB10220AB90122DA601A6A42F21073F9
:10AED0009A4204D116214FF6FF70FFF7B2BF7047B8
:10AEE0006C3A0020A03F00207040002010B503788D
:10AEF0000446042B2AD8DFE803F0032213290700B5
:10AF0000BDE8104000F096BF1148124B1249C01A1C
:10AF1000C0080004BDE8104040F00300FBF754BD3A
:10AF20000B4B0C480D491B1ADB081B0443F00100B6
:10AF3000FBF74AFD6068BDE81040FCF755B8044BCC
:10AF4000044807491B1ADB081B04EFE710BD00BFCC
:10AF50004006030018060300A2100300B01003000F
:10AF6000E2100300FCF740B837B5294B294C0546E1
:10AF7000E41A2A78284B406853F82220E408240475
:10AF800044F0030480B925492046FBF721FD2B78C6
:10AF9000012B13D0032B26D023B96B6813B9204B98
:10AFA00001221A7003B030BD019201F03BFF019AFB
:10AFB0001C4903462046FBF714FDE8E76B68002BAD
:10AFC000F0D1AA6818492046FBF702FDAA89174963
:10AFD0002046FBF7FDFCEA891549204603B0BDE891
:10AFE0003040FBF7F5BC6B6873B9AA680E49204680
:10AFF000FBF7EEFCAA890D492046FBF7E9FCEA893C
:10B000000B492046FBF7E4FC0A4B00225A70C9E7C3
:10B010001806030040060300781603000E11030013
:10B02000163C00202F1103004711030059110300A3
:10B0300069110300143C00200146014804F0A4B843
:10B04000FC3B00200388212B13B504460FD80F2B9F
:10B0500011D9103B112B0ED8DFE803F01C3F0D581F
:10B060000D0D0D0D0D0D0D4E0D0D0D5F0F653B2BD7
:10B0700067D0562B65D002B010BD3448344B3549EB
:10B08000C01AC008000440F0030002B0BDE8104040
:10B09000FBF79ABC2E4B2D482F49C01AC00800045C
:10B0A00040F00300FBF790FCA1882C48002204F03C
:10B0B00099F908B1FBF798FF0720FFF719FE08B1CF
:10B0C000FBF792FFA188264802F000FF0028D2D0AB
:10B0D00002B0BDE81040FBF787BF1D4B1B48A2889C
:10B0E0002049C01AC008237A000440F0030002B0CF
:10B0F000BDE81040FBF775BC037A022BBBD11348A7
:10B10000134B1949C01AC0080004BCE700231A46B3
:10B1100085218088FFF797FED8E700F10801808835
:10B12000FFF78DFED2E7002380888DF8043001A957
:10B130008DF80530FFF789FE00289CD0FBF754FFFF
:10B1400099E7A0881321FFF77CFEBFE740060300C4
:10B15000180603007C11030098110300FC3B00203B
:10B16000842A0020AE110300DC11030008B5074853
:10B1700003F05EFD08B1FBF737FF0120FFF7B8FDD4
:10B1800018B1BDE80840FBF72FBF08BD503C0020B8
:10B190002DE9F0470B78012B80460D4638D0022B65
:10B1A00000F09982002B40F02A819F4E9F4C86F838
:10B1B00098309F4B9F49E41AE408240444F00304A8
:10B1C0002046FBF701FC698805F10E02404604F0B9
:10B1D00009F908B1FBF708FF404604F081F808B10F
:10B1E000FBF702FF20469449FBF7EEFB96F8990027
:10B1F000022804D0032802D0012840F0008101F089
:10B2000029FFBDE8F0478D498D48102204F09CB815
:10B21000874B864F844CFF1AFF088B6889491A7840
:10B220003F0447F005063046FBF7D2FB94F8983010
:10B23000002B40F0CF81A9680B78723B032B00F202
:10B24000DE80DFE813F07B0121010400A101AA895F
:10B250007D48DFF828A204F00AFE784901F11100C8
:10B2600001F096FF79493046FBF7AEFB4FF000093D
:10B2700004EB0903514693F83820304609F10109DF
:10B28000FBF7A6FBB9F1100FF2D1AB68DFF8ACC148
:10B29000013304F1480E624603CA724518605960D2
:10B2A000944603F10803F6D1AB681B7B013B032BEB
:10B2B00000F2A580DFE803F0024461A547F0030730
:10B2C00063493846FBF780FBAB685A7B84F8302033
:10B2D0009A7B84F83120DB7B84F832302378DBB131
:10B2E000032B40F08A805B4801F08CFE012840F07F
:10B2F00084800025062258495148257725752570F8
:10B3000004F022F855493846FBF75EFB657100F002
:10B3100028FD00F019FD09E00122227541F2883272
:10B32000A2614F4AA372936100F0D6FFB8F8020001
:10B330001321FFF786FD00285FD0FBF755FE5CE088
:10B3400047F0030747493846FBF73EFBAB685A7B9B
:10B3500084F830209A7B84F83120DB7B84F832300B
:10B3600023783BB1032B48D13A4801F04BFE01282A
:10B37000DCD1BEE701F096FCD8E747F003073A4975
:10B380003846FBF721FB3649AA6800238B62507BC5
:10B3900084F83000907B84F83100D27B84F832202E
:10B3A000227F52B309222275DFF8D480DFF8D490CF
:10B3B0008B614FF4FA62A2611D4618F8012B4946D1
:10B3C00038460135FBF704FB062DF6D1E26A274922
:10B3D0003046FBF7FDFA26493046FBF7F5FAE06AFE
:10B3E00001F0D0FD1C4916482A4603F0ADFF214963
:10B3F0003846FBF7E9FA01F041F80023A372BDE8F3
:10B40000F0871D4947F00300FBF7DEFAAB685A7B73
:10B4100084F830209A7B84F83120DB7B84F832304A
:10B4200000F0D4FF82E700BFA03F002040060300E9
:10B4300018060300FA1103000E120300D83F002083
:10B44000FC3B00203C120300E83F002045120300B3
:10B450004A120300BC440020E112030069120300F9
:10B4600070400020851203009F120300CF120300DA
:10B47000821C0300DC120300E81203005B190300C6
:10B48000BD3F0020C8120300AA899A499A4F30464E
:10B49000FBF79EFA012384F89830732384F89A30DE
:10B4A000AA89A968954804F0E2FC954901F11100C8
:10B4B00001F06EFE93493046FBF786FA00256319CA
:10B4C000394693F8382030460135FBF781FA102DC4
:10B4D000F5D18D493046FBF777FA94F83C3084F883
:10B4E0009B3094F83D3084F89C3094F83E3084F8DA
:10B4F0009D3094F83F3084F89E3094F8403084F8C2
:10B500009F3094F8413084F8A03094F8423084F8A9
:10B51000A13094F8433084F8A23094F8443084F891
:10B52000A33094F8453084F8A43094F8463084F879
:10B53000AD3094F8473084F8AE3060E7AA8973499B
:10B540006D4F3046FBF744FA012384F8983072239C
:10B5500084F89A30AA89A968684804F088FC684988
:10B5600001F1110001F014FE66493046FBF72CFA98
:10B5700000256319394693F8382030460135FBF72A
:10B5800027FA102DF5D1A4E7AA8961495A4F304610
:10B59000FBF71EFA012384F89830752384F89A305B
:10B5A000AA89A968554804F062FC554901F11100C7
:10B5B00001F0EEFD53493046FBF706FA002563190A
:10B5C000394693F8382030460135FBF701FA102D43
:10B5D000F5D17EE7012B7FF412AF002784F8987035
:10B5E000AA89A96804F1480004F041FC04F138017B
:10B5F00004F1480001F0CCFD46493046FBF7E4F980
:10B600003D463D4F6319394693F8382030460135A1
:10B61000FBF7DEF9102DF5D130463B49FBF7D4F9A5
:10B6200094F89A0073281FD0752838D072287FF4B8
:10B63000E6AE637A002B7FF4E2AE01F05BFD3049A9
:10B6400035482A4603F080FE23780BB900F0B0FCA1
:10B65000B8F802001321FFF7F4FB08B1FBF7C4FCB4
:10B66000002384F89930CAE6667A002E7FF4C7AECC
:10B6700001F040FD224928482A4603F065FE84F87F
:10B68000996000F043FDB8F802001321FFF7D9FBE1
:10B6900000283FF4B4AEBDE8F047FBF7A5BC677ADD
:10B6A000002F7FF4ACAE01F08DFD15491A482A46F3
:10B6B00003F04AFEA77200F013FCB8F80200132151
:10B6C000FFF7BFFB08B1FBF78FFC30461349BDE81D
:10B6D000F047FBF779B9124B12481349C01AC0085A
:10B6E000000440F00300FBF76FF9BDE8F047FFF7F7
:10B6F0003DBD00BF031303005B190300E83F0020BA
:10B70000D83F002014130300821C030027130300FA
:10B710003613030047130300FC3B00205D130300B6
:10B720001806030040060300731303001FB50378D7
:10B73000052B12D0062B17D0042B2AD1164B1748F5
:10B740001749C01AC008000440F00300FBF73CF999
:10B7500004B0BDE81040FFF709BD4068C8B104B0AF
:10B76000BDE81040FBF740BC41680B4C0B488B78A0
:10B770004A78001B8C7903944C7902940C790194DB
:10B78000C008C97800910004064940F00300FBF7A7
:10B790004CF904B010BD00BF1806030040060300BA
:10B7A000C41303009613030010B504460020FFF7EE
:10B7B0009FFA08B1FBF718FC24B9FFF72DFB08B17D
:10B7C000FBF712FC012010BD0A8840F677239A424D
:10B7D00013B50C4615D10C4B0C480D49C01AC008C6
:10B7E000000440F003000190FBF7EEF8A38809493C
:10B7F0000198033B9BB21A4602B0BDE81040FBF72C
:10B80000F0B802B010BD00BF1806030040060300E8
:10B81000D4130300F01303000B2837B52ED11A4BB5
:10B820001A481B49C01AC00800044FF0A04540F058
:10B8300003000190FBF7C8F8D5F8104501981549A9
:10B84000C4F3C0242246FBF7C3F801984FF4003339
:10B8500064B9C5F80C351049FBF7B6F80F4B012257
:10B860005A7103B0BDE8304001F0EAB90C49C5F89F
:10B87000083503B0BDE83040FBF7A6B803B0BDE81B
:10B880003040FBF7B1BB00BF1806030040060300C1
:10B89000181403002914030034140300A03F0020EF
:10B8A0003E14030038B5054D044645F001054FF43C
:10B8B0007A40A847013CFAD138BD00BF701603009A
:10B8C000014B01221A707047143C002038B5104D0E
:10B8D0006B78012B1AD02B78C3B10E4B0E4C0F494D
:10B8E000E41AE408240444F003042046FBF76CF84F
:10B8F00001F0A0FA002814BF012300232B7005D10A
:10B9000020460749BDE83840FBF75EB838BD00BFA8
:10B91000143C0020180603004006030049140300ED
:10B920005F14030008B50849084802F0ADFC08B1EF
:10B93000FBF75AFB0548F72102F0BAFC18B1BDE845
:10B940000840FBF751BB08BDC9B70200183C0020F6
:10B9500070B5494C2378042B0AD8DFE803F0030ABA
:10B9600039577100454B00221A635A639A63DA63B0
:10B9700070BD424D4248EB6B42490133EB63424B91
:10B98000EA6BC01AC00800044FF4167340F00500BB
:10B99000FBF727F8EB6BB3F5167F09DB0026EE63A8
:10B9A000267000F0D1F900F0DCF926756670DFE74B
:10B9B0006378002BDCD0A3780133DBB2092B01D8EC
:10B9C000A370D5E70023A370BDE8704000F008BC69
:10B9D0002A4D2B486B6B2D4901336B632A4B6A6BE5
:10B9E000C01AC0080004D22340F00500FAF7F9FF9E
:10B9F0006B6BD12BBCDD00266E63267000F0A4F9C2
:10BA000000F0BDF900F0C9F92675B1E71B4D1C48DF
:10BA10002B6B1F4901332B631B4B2A6BC01AC008C9
:10BA200000043C2340F00500FAF7DBFF2B6B3B2BB7
:10BA30009EDD00262E632677267000F085F9E3E769
:10BA40000E4D0F48AB6B13490133AB630E4BAA6B22
:10BA5000C01AC00800043C2340F00500FAF7C1FFFB
:10BA6000AB6B3B2B84DD0026AE632677267000F09F
:10BA70006BF900F076F9C7E7A03F00207040002086
:10BA8000400603007A14030018060300B5140300EF
:10BA9000EC1403002015030070B58EB000204FF4A5
:10BAA00080418DF80800FAF7F5FD08B1FBF79CFA24
:10BAB000FAF72EFD8748884CFDF796F9874B8849A1
:10BAC000E41AE408240444F005000190FAF77CFF2E
:10BAD00084490198FAF778FF81490198FAF774FFD1
:10BAE000FDF798F908B1FBF77FFAFBF767FB08B1A0
:10BAF000FBF77AFA7C4E7D4A7D480121FBF790FBEB
:10BB00000FCE08AD0FC596E803007A4B7A4A04932E
:10BB10004FF4807385E80300CDE906230593774A47
:10BB2000072304A908A8FBF7EBFC08B1FBF75CFAB4
:10BB3000734840F233320121FBF7E8F908B1FBF713
:10BB400053FA7049704E08784FF0A04300F5E0704A
:10BB5000032243F82020487800F5E07043F82020C5
:10BB60008878C97800F5E07001F5E07143F820208D
:10BB700043F8212008A8654B0893099602F068F95C
:10BB800008B1FBF731FAFCF7ABFA08B1FBF72CFA76
:10BB900003F098FC08B1FBF727FA002308A901205D
:10BBA000089303F0A1FD08B1FBF71EFA08A803F003
:10BBB0005BFE08B1FBF718FA554D2846FFF73DF933
:10BBC00044238DF8093033238DF80A30C0238DF8D3
:10BBD0000B302B798DF80C306B798DF80D3002A875
:10BBE000AB798DF80E30FFF726F94A48FFF725F9B3
:10BBF000FFF798FE484B0893484B494808A9CDE900
:10BC0000093603F007FB08B1FBF7EEF9102200211B
:10BC100008A804F055F90123424A43488DF824301E
:10BC200008A98DF82C3002F0A6FF08B1FBF7DCF96B
:10BC30003E4A3D48032102F071FE08B1FBF7D4F9FA
:10BC400039480022042102F089FE08B1FBF7CCF943
:10BC5000032500F073F86420FFF724FE013D00F097
:10BC600073F86420FFF71EFE15F0FF05F1D130498F
:10BC700044F00300FAF7A8FEFFF778FA2A461021ED
:10BC80002C48FBF7D8FAFBF799F908B1FBF7ACF9A8
:10BC900000F05AF801F0E6F800F0ACFD4FF47A70CD
:10BCA000FFF700FE00F0A6FD234C0025FAF742FD49
:10BCB00008B9FCF72BFA00F085F800F077FE01F0E8
:10BCC00015F8FFF703FEE368002BEFD0E560FFF700
:10BCD0003FFEEBE769AF02004006030018060300D1
:10BCE0005B1503009A1503005016030051AE0200C5
:10BCF000A8160300D23C0020D23D0020EDAE020089
:10BD0000642A0020AC1603006C2A002039B002001F
:10BD1000CB3C0020C43C002091B1020065AF020082
:10BD2000FC3B00202DB70200503C0020A41603006D
:10BD3000D3150300303C0020704000204FF0A0439A
:10BD40008022C3F8082570474FF0A0438022C3F833
:10BD50000C2570474FF0A0434FF40062C3F808254C
:10BD600070474FF0A0434FF40062C3F80C257047B2
:10BD70004FF0A0434FF48052C3F8082570474FF0AE
:10BD8000A0434FF48052C3F80C2570474FF0A043F6
:10BD90004FF40052C3F8082570474FF0A0434FF40A
:10BDA0000052C3F80C25704738B5054D044645F0E0
:10BDB00001054FF47A40A847013CFAD138BD00BFD5
:10BDC000D01A030038B5144C23690A2B18DD134B25
:10BDD000DA78AAB1124D13482A680021142A815436
:10BDE000D9700BD1012210481A71104B1049C01A9A
:10BDF000C008000440F00500FAF7E6FD00232B60C0
:10BE000023690A2B06DD064B1A681AB10349002282
:10BE1000CA701A6038BD00BF70400020A03F0020EB
:10BE2000383F0020D23E00204006030018060300E1
:10BE3000B016030013B50DF10700FBF7B9FB88B985
:10BE4000094B0A499DF807400122DA70084A136835
:10BE5000CC540133642193FBF1F401FB14331360E0
:10BE6000044B186102B010BDA03F0020D23E00205C
:10BE7000383F002070400020F7B5144B144F0646A1
:10BE800014481B1ADB081B0443F005000C4612493A
:10BE90000190FAF799FD0025A542019807DB0F49AB
:10BEA000FAF792FD0025A54208DB03B0F0BD725DF4
:10BEB00001903946FAF78CFD0135EDE7705DFBF72F
:10BEC0008DFB0028FAD10135EDE700BF40060300E5
:10BED000E516030018060300CE160300821C0300BB
:10BEE0002C4B2D482D49C01AC008000410B540F055
:10BEF00005002B4CFAF768FD222323754FF4966357
:10BF0000A361284B00219961274B617132221846A9
:10BF100003F0D6FF02222549027003220346427035
:10BF20000122C2700879D871487989795972122131
:10BF300099727421D97294F89B10197494F89C101A
:10BF4000597494F89D10997494F89E10D97494F8CB
:10BF50009F10197594F8A010597594F8A11099754F
:10BF600094F8A210D97594F8A310197694F8A41037
:10BF700018725976985C197F013201441C2A19778E
:10BF8000F8D103225A77BDE8104007481E21FFF779
:10BF900073BF00BF1806030040060300EB16030042
:10BFA000A03F0020704000203C3F0020C43C002007
:10BFB0002DE9FF414B4B4C4F4C4D4D494D4CFF1A19
:10BFC000FF083F0447F00500FAF7FEFC41F2883312
:10BFD000AB61494B00264FF001089E6140F20123FE
:10BFE0002B8085F81480AE7285F80580FFF7B2FECD
:10BFF00031463222204603F063FF404984F8038033
:10C00000022323706370D1F89830E3B1063101A8A0
:10C0100003F089FF1022314602A88DF80A6003F070
:10C02000DDFE1022A07131460DF106008DF808608A
:10C0300003F0D4FE10226071314601A88DF806602D
:10C0400003F0CCFE20712E4B1A79E2715A792272DC
:10C0500095F89B20227495F89C20627495F89D2099
:10C06000A27495F89E209B79E27495F89F206372E4
:10C070002275122395F8A020A3726275722395F899
:10C08000A120E372A275002395F8A22023736373A5
:10C09000A373E37323766376A376E376E2750123D5
:10C0A000E15C227F01330A441C2B2277F8D1032361
:10C0B0006377104B134A03F1300153F8040B42F835
:10C0C000040B8B42F9D11B88138047F003000E4903
:10C0D000FAF77AFC07481E21FFF7CEFE04B0BDE850
:10C0E000F08100BF1806030040060300A03F0020B7
:10C0F000021703003C3F002070400020B4400020A5
:10C10000C43C00206E3F00201C17030070B52C4B70
:10C110002C4E2D4C2D49F61AF608360446F0050033
:10C12000FAF752FC212323754FF49663A361284B41
:10C1300000259D61274BA57232222946184665715C
:10C1400003F0BEFE022202704270C270224A1179D0
:10C15000C171517992794272122282727322C27233
:10C1600094F89B20027494F89C20427494F89D20CB
:10C17000827494F89E20C27494F89F20027594F8FB
:10C18000A020427594F8A120827594F8A220C2756F
:10C19000034601720122995C01320D441C2AEDB262
:10C1A000F9D1032246EA02000C491D775A77FAF7C3
:10C1B0000BFCBDE8704007481E21FFF75DBE00BFC5
:10C1C0001806030040060300A03F002031170300BB
:10C1D000704000203C3F0020C43C00204917030071
:10C1E000154B164910B5164CE41AE408240444F023
:10C1F0000500FAF7E9FB134B134A03F1300153F83A
:10C20000040B42F8040B8B42F9D11B8813800F49B1
:10C2100044F00300FAF7D8FB0D4B5B78012B02D0FA
:10C22000022B06D010BD1421BDE810400648FFF7D0
:10C2300023BE1E21F8E700BF180603005D170300A8
:10C24000400603006E3F00203C3F002075170300AE
:10C25000A03F002010B51B4B1B4904461B481B1A6E
:10C26000DB081B0443F00500FAF7AEFB184B322243
:10C270000021184603F024FE1649C470022203462A
:10C280000270012242700879D8714879897959720F
:10C29000082199724121D972432119734B21597395
:10C2A00018720021985C01320144122AC9B2F9D1F6
:10C2B00003229974DA74BDE8104005481421FFF791
:10C2C000DBBD00BF4006030089170300180603000A
:10C2D0003C3F0020C43C002038B5334B334D344C38
:10C2E0003449ED1AED082D0445F00500FAF76CFB12
:10C2F0000123314A237541F28833A36100239361FE
:10C3000040F201122280227F012A08BF23772B4BA3
:10C3100032220021184603F0D3FD94F82010017159
:10C3200094F82110417194F822108171022224495D
:10C330000270034601224270C2700879D8714879B0
:10C34000897959720821997294F83110D97294F848
:10C350003210197394F83010597318720021985CD8
:10C3600001320144122AC9B2F9D103229974DA7454
:10C37000124B144A03F1300153F8040B42F8040B3A
:10C380008B42F9D11B88138045F003000E49FAF760
:10C390001BFB0A481421FFF76FFD01236371BDE801
:10C3A0003840FFF7D7BC00BF180603004006030063
:10C3B000A03F002099170300704000203C3F002060
:10C3C000C43C00206E3F00207717030038B5244B93
:10C3D000244C2549E41AE408240444F00500FAF743
:10C3E000F3FA224B32220021184603F069FD0621A0
:10C3F0000222C1701E49027003460122427091F868
:10C400002000187191F82100587191F8220098715C
:10C4100018480579DD71457980795872082098723D
:10C4200091F83100D87291F8320091F830105973B8
:10C430001D7218730021985C01320144122AC9B29E
:10C44000F9D10322997444EA02000B49DA74FAF72D
:10C45000BBFABDE8384005481421FFF70DBD00BF09
:10C460001806030040060300AF1703003C3F0020FE
:10C47000A03F0020C43C0020C11703001F4B2048F0
:10C480002049C01AC008000410B540F00500FAF7B2
:10C490009BFA1D4B00241C631C4B3222214618467C
:10C4A00003F00EFD0D210222C170194902700346EE
:10C4B0000122427091F82000187191F8210091F842
:10C4C00022109971134958710879D871487989797E
:10C4D0005972082118729972995C01320C44122A1F
:10C4E000E4B2F9D1032209489C74DA741421FFF7ED
:10C4F000C3FCBDE810403220FFF756BC180603000D
:10C5000040060300CF170300704000203C3F00208E
:10C51000A03F0020C43C00202DE9F04F6D4B6E4E33
:10C520006E4F6F49D7F89820F61AF608360487B090
:10C5300046F00500FAF74CFAD7F89850002D40F075
:10C54000C080684C32222946204603F0B9FC022301
:10C5500023704FF001080D23B91D03A8E37084F880
:10C56000018003F0E0FC102229460DEB02008DF85B
:10C57000125003F033FC1022A07129460DF10E0079
:10C580008DF8105003F02AFC10226071294603A890
:10C590008DF80E5003F022FC534B25711A79E2718D
:10C5A0005A799B7922726372A27C65710823A37207
:10C5B000A571E57225736573A573E57325746574BC
:10C5C0004346E15C01330A44122BD2B2F9D1032372
:10C5D000E37400234549A27400931A4646F0030011
:10C5E000FAF709FA3F481421FFF746FC3220FFF71B
:10C5F000DBFB07B0BDE8F08F32220021C5EB05154B
:10C60000384803F05DFC0223A91D23704FF0010B95
:10C610000D23394403A80025E37084F801B003F02A
:10C6200082FC102229460DEB02008DF8125003F017
:10C63000D5FB1022A07129460DF10E008DF8105087
:10C6400003F0CCFB29466071102203A88DF80E5030
:10C6500003F0C4FB99F80430E37199F805302372B4
:10C6600099F806306372A17C20710823A372E572E9
:10C6700025736573A573E573257465745B46E25C89
:10C6800001331144122BC9B2F9D10323E374A37906
:10C69000A174C2B200935146637946F00300FAF7E1
:10C6A000AAF914212046FFF7E7FBC820FFF77CFB1F
:10C6B00008F10108D7F898305FFA88F59D429BDBB6
:10C6C00097E7084CDFF82090DFF824A04FF000082F
:10C6D000F0E700BF1806030040060300B440002046
:10C6E000E91703003C3F0020C43C00200E18030063
:10C6F0002A1803007FB5374C32220021204603F070
:10C70000DFFB354B35483649C01AC008000440F0FD
:10C710000300FAF759F9334B5D7A04221A70002DA1
:10C7200052D141F288329A612F4A9D7201261E75BC
:10C730005E719561FFF70EFB02232C4923701323D2
:10C74000E370D1F898306670A570002B3ED00631AA
:10C7500001A803F0E8FB1022294602A88DF80A5030
:10C7600003F03CFB1022A07129460DF106008DF864
:10C77000085003F033FB10226071294601A88DF8A0
:10C78000065003F02BFB2071194B1A79E2715A798C
:10C790009B7963720823A3720023E372237363738C
:10C7A000A373E37323746374A37C22720122A15CDC
:10C7B00001320B44122ADBB2F9D1A37405480323DA
:10C7C0001421E374FFF758FB04B070BD237163714B
:10C7D000A371D9E73C3F0020180603004006030080
:10C7E00047180300A03F002070400020B440002004
:10C7F000C43C002038B52148214B2249224CC01AA4
:10C80000C008000440F00500FAF7DEF81F4B0021D5
:10C810001846322203F054FB617A034639BB1022DA
:10C82000227540F2DC52A261194AA1729161022282
:10C830000270012242701120D8701648DA72057910
:10C84000DD7145798079587208201D7298721A73CB
:10C85000985C01320144122AC9B2F9D103229974B9
:10C86000DA740A481421FFF707FB00236371BDE85F
:10C8700038404FF47A70FFF797BA00BF40060300C4
:10C88000180603005C180300A03F00203C3F002076
:10C8900070400020C43C002070B5394B394C3A49F7
:10C8A0003A4DE41AE408240444F005042046FAF75B
:10C8B0008BF8374B00211846322203F001FB697ACE
:10C8C000034639BB10222A7540F2DC52AA61314A74
:10C8D000A972916102220270012242700F20D87069
:10C8E0002D48DA720679DE7146798079587208200F
:10C8F0001E7298721A73985C01320144122AC9B2EE
:10C90000F9D103229974DA7421481421FFF7B4FA9B
:10C9100000236B7120462149FAF756F8204620493A
:10C92000FAF752F820461D49FAF74EF84FF47A709C
:10C93000FFF73AFA0524FFF701FA6420FFF734FA0B
:10C94000013CFFF701FA6420FFF72EFA14F0FF0410
:10C95000F1D140F6B830FFF727FA4FF08043B1220B
:10C96000C3F81C25BFF34F8F0E490F4BCA6802F462
:10C97000E0621343CB60BFF34F8F00BFFDE700BF02
:10C9800018060300400603007C180300A03F0020A7
:10C990003C3F002070400020C43C00209A18030057
:10C9A000EC18030000ED00E00400FA052DE9F74360
:10C9B000894E3379002B3BD08848894C8949DFF870
:10C9C0007882DFF87892241AE408240444F0050001
:10C9D000002501903571F9F7F7FF01988249F9F7C1
:10C9E000F3FF0198474618F8012B0190494601359D
:10C9F000F9F7EEFF142D0198F5D17A49F9F7E4FF24
:10CA00003B78022B14D17B78013B012B10D8FB78AB
:10CA1000013B112B0CD8DFE803F0090E1F2B313935
:10CA20003B6B0B870BB10BD70BCD0BC30023737084
:10CA300003B0BDE8F0836D4944F003000025357074
:10CA4000F9F7C2FFFFF780F9FFF78BF9FFF797F9C6
:10CA5000FFF7A3F97571EBE7654944F00300F9F7B7
:10CA6000B3FFFFF76BF9FFF77CF900237371DFE782
:10CA7000604944F00300F9F7A7FFF6E75E4944F088
:10CA8000030003B0BDE8F043F9F79EBF5B49F6E74A
:10CA9000022333705A4B5B4944F00300002201909B
:10CAA0005A63F9F791FFFC7A019884B95649F9F76E
:10CAB0008BFF56490198F9F787FFFFF76EF9FFF7EB
:10CAC00057F9FFF74EF9FFF739F97471B0E750499C
:10CAD0000190F9F779FF4F490198F9F775FFFFF7D2
:10CAE0004EF9FFF753F903B0BDE8F043FFF726B95D
:10CAF00044F0030048490190F9F766FF3578019842
:10CB00005DB903233370082333750920012333777C
:10CB1000FFF7A0FB3A4B9D628AE740492A4603B0E3
:10CB2000BDE8F043F9F754BF3D4944F00300F9F77D
:10CB30004BFF0B20FFF78EFB9C220021394803F0AE
:10CB4000BFF9FEF7BDFEFFF7F9F84FF49670FFF757
:10CB50002BF9FFF7F9F84FF49670FFF725F9FFF777
:10CB6000EDF84FF49670FFF71FF9FFF7EDF84FF46B
:10CB7000967003B0BDE8F043FFF716B92A4944F0B8
:10CB80000300F9F721FFFFF7C7FCFFF7D7F84FF4D1
:10CB90009670FFF709F903B0BDE8F043FFF7D4B88A
:10CBA000224944F00300F9F70FFF03B0BDE8F0435A
:10CBB000FFF7A0BD1E4944F00300F9F705FF03B0DD
:10CBC000BDE8F043FFF716BE1A4944F00300F9F739
:10CBD000FBFEFFF761FE00BFA03F00201806030028
:10CBE00040060300971503003E1903006119030076
:10CBF0006F1903007E190300901903009C190300AC
:10CC000070400020AE190300C0190300C7190300CB
:10CC1000D3190300DB190300E6190300071A030008
:10CC20001E1A0300B4400020401A0300621A0300D9
:10CC30007F1A03009B1A0300D23E002059190300FB
:10CC400008B5154B32220021184603F039F9134973
:10CC500002220346027001224270C2700879D87124
:10CC60004879897959720821997218720021985C63
:10CC700001320144122AC9B2F9D103229974DA743B
:10CC800005481421FFF7F8F8054B01225A71BDE859
:10CC90000840FFF75FB800BF3C3F0020C43C0020C5
:10CCA000A03F00200C4B0D480D49C01AC0080004DD
:10CCB00010B540F005000B4CF9F786FE01236371B7
:10CCC000FFF748F81423237540F6E443A361064BAD
:10CCD00000229A6110BD00BF180603004006030041
:10CCE000BB1A0300A03F00207040002038B5304C34
:10CCF000237D142B36D019D8082B13D0092B20D024
:10CD000063795BB3237D4BB32A4B9A69B2F5FA7F03
:10CD100024DB00229A61284A13780133DBB21370B6
:10CD2000DB0741D5BDE83840FFF708B8213B032BAE
:10CD3000E6D8A369002B32DA00252575FFF704F841
:10CD400019E0237F012B19D1A369002B16DA0823E0
:10CD50002375FEF7F3FF184B00221A7038BDFEF75B
:10CD6000F3FFCDE7A369002B08DA00252575FEF750
:10CD7000EBFFFEF7F6FF104B1D70EFE70D4B9A69C6
:10CD8000B2F5FA7FEADB00229A610B4A137801338D
:10CD9000DBB21370DA07E2D5FEF7D0FFB0E7054B40
:10CDA0009A69B2F5967FEDE7BDE83840FEF7CCBF53
:10CDB000A03F002070400020B040002010B586B099
:10CDC00003230593124C134BADF80E00E41AE4084C
:10CDD00024040C2344F00304CDE900130122049140
:10CDE00003460D49ADF80C202046F9F710FE03A9C3
:10CDF0000020FCF783F940B1A0F50640074B084935
:10CE000053F820202046F9F7E3FD06B010BD00BF1F
:10CE10004006030018060300701B0300681E030091
:10CE2000B71B0300024BA0F5064053F820007047E3
:10CE3000681E030010B586B0002401A903A8CDE93F
:10CE40000144CDE903440594FCF782F938B903A8FD
:10CE5000FCF758F9B0FA80F0400906B010BD204642
:10CE6000FBE700002DE9F04F8BB00023CDE9033341
:10CE7000CDE907330993384D384B3949DFF8F48051
:10CE8000DFF8F490DFF8F4A0ED1AED082D0445F07A
:10CE900003063046F9F798FD03A907A8FCF758F9EF
:10CEA00048F20967B84227D0002305A907A8CDE9B1
:10CEB0000533FCF7C1F8B842044625D048F20C63AC
:10CEC00098421CD010BB059ADFF8B4B05188938803
:10CED000890001911188009145F00507514692683B
:10CEE0003846F9F794FDDBF898300699042B17DDE6
:10CEF0001C493846F9F768FD0BB0BDE8F08F49468C
:10CF00003046F9F761FDC7E74146F9E7A0F5064469
:10CF1000154B164953F824203046F9F759FDBBE765
:10CF2000C3EB0310584401330C220473CBF8983040
:10CF300002F029FFDBF898200D49013AC2EB0212FA
:10CF400038465A44F9F744FD07A8FCF7B3F800281F
:10CF5000A2D0FAF749F89FE740060300180603003D
:10CF6000DF1B0300071C0300681E03002D1B0300CA
:10CF7000D8120300131B0300F91A0300491B030016
:10CF8000B4400020F7B51B4DD5F89840042C01465D
:10CF900017DC2F460026B44215DCC4EB0414281914
:10CFA000002303730C22019102F0EDFED5F89800E6
:10CFB00001990130FFF702FFD5F898300133C5F829
:10CFC000983003B0F0BD38460C22019102F0BDFE4E
:10CFD0000F37019960B9084B08480949C01AC008C1
:10CFE000000440F0050003B0BDE8F040F9F7ECBCE8
:10CFF0000136D0E7B44000201806030040060300C5
:10D00000161C0300F8B50F4CD4F89870064600259E
:10D01000AF4201DC002011E020460C22314602F034
:10D0200094FE0F3458B9084B08480949C01AC00883
:10D03000000440F00500F9F7C7FC0120F8BD0135F8
:10D04000E6E700BFB44000201806030040060300D6
:10D050002C1C0300F0B5214B89B06A46064603F14B
:10D060001007154618685968144603C40833BB42B4
:10D070002246F7D11A4B04AA03F1100C1746186880
:10D080005968144603C4083363452246F7D1022E7B
:10D0900008D145238DF810304D238DF811304723EA
:10D0A0008DF8123002F02CFE2946C0F30723044607
:10D0B0008DF813000B4A8DF81430384600F00CFC44
:10D0C00009480A4B0A491B1ADB081B04A2B243F0A9
:10D0D0000500F9F77DFC09B0F0BD00BF481C030056
:10D0E000591C0300D83F0020180603004006030027
:10D0F000371C0300F0B5204B89B06C46024603F1A3
:10D100001006274618685968254603C50833B342F8
:10D110002C46F7D1194B04AC03F1100C26461868C5
:10D120005968254603C5083363452C46F7D1722A52
:10D1300012D0752A1AD0124A3946304600F0CCFB7C
:10D14000104B11481149C01AC008000440F00500F6
:10D15000F9F73AFC09B0F0BD45238DF813304D23A3
:10D160008DF8143047238DF81530E4E750238DF8FF
:10D1700013304123F7E700BF481C0300731C030072
:10D18000D83F002018060300400603006A1C030075
:10D19000F0B50B4B85B06C4606460A4603F1100C01
:10D1A000274618685968254603C5083363452C4649
:10D1B000F7D13946304600F0A5FB05B0F0BD00BF01
:10D1C000481C0300FFF796BFF0B5134A8BB002ACC2
:10D1D00007460E4602F1100C23461068516825469A
:10D1E00003C5083262452C46F7D10C4A06AC02F161
:10D1F000100EA44610685168254603C508327245D2
:10D200002C46F7D1CDF800C010223946304600F048
:10D210008FFB0BB0F0BD00BF841C0300951C030006
:10D22000F7B504464D494E4E0C30FFF7CDFF4D4843
:10D230004D4B4E491B1ADB081B0443F005000190BF
:10D24000F9F7C2FB0198651E1B3415F8012F0190F8
:10D250003146F9F7BDFBA5420198F6D144493F4D4F
:10D260003F4EF9F7B1FB01984249F9F7ADFB019840
:10D27000102415F8012B01903146013CF9F7A8FB69
:10D2800014F0FF040198F4D13B4C39493B4DF9F7B8
:10D290009BFB94F8483094F84CC094F8A5E084F8CF
:10D2A0009B3094F8493084F89C3094F84A3094F8D4
:10D2B0004D7094F84E6094F84F0094F8501094F824
:10D2C000512084F89D30E64594F84B3084F89E3028
:10D2D00084F89FC0EB6A84F8A07084F8A16084F899
:10D2E000A20084F8A31084F8A42035D140F6B83CFD
:10D2F0006345D4BF0023012394F8A6C0BC4518BFE2
:10D30000012394F8A770B74218BF012394F8A860CE
:10D31000864218BF012394F8A900884218BF012350
:10D3200094F8AA10914200D19BB1FEF7D9FD94F870
:10D330009F2084F8A5200023B4F8A020EB62A4F875
:10D34000A62094F8A430B4F8A220A4F8A82084F869
:10D35000AA30012003B0F0BD0123CDE7E83F002053
:10D360005B1903001806030040060300A61C030017
:10D37000821C0300CA1C0300A03F00207040002054
:10D38000F7B504464D494E4E0830FFF71DFF4D4896
:10D390004D4B4E491B1ADB081B0443F0050001905E
:10D3A000F9F712FB0198651E173415F8012F01904B
:10D3B0003146F9F70DFBA5420198F6D144493F4D9E
:10D3C0003F4EF9F701FB01984249F9F7FDFA019840
:10D3D000102415F8012B01903146013CF9F7F8FAB9
:10D3E00014F0FF040198F4D13B4C39493B4DF9F757
:10D3F000EBFA94F8483094F84CC094F8A5E084F81F
:10D400009B3094F8493084F89C3094F84A3094F872
:10D410004D7094F84E6094F84F0094F8501094F8C2
:10D42000512084F89D30E64594F84B3084F89E30C6
:10D4300084F89FC0EB6A84F8A07084F8A16084F837
:10D44000A20084F8A31084F8A42035D140F6B83C9B
:10D450006345D4BF0023012394F8A6C0BC4518BF80
:10D46000012394F8A770B74218BF012394F8A8606D
:10D47000864218BF012394F8A900884218BF0123EF
:10D4800094F8AA10914200D19BB1FEF729FD94F8BF
:10D490009F2084F8A5200023B4F8A020EB62A4F814
:10D4A000A62094F8A430B4F8A220A4F8A82084F808
:10D4B000AA30012003B0F0BD0123CDE7E83F0020F2
:10D4C0005B1903001806030040060300E51C030077
:10D4D000821C0300051D0300A03F002070400020B7
:10D4E000274B284A1B6873B503F110011878107098
:10D4F0005878507098789070D878D07004338B42F8
:10D5000002F10402F2D1204B2048214C04211A6878
:10D5100001928D0714D1C2F30746C2F30725865D39
:10D520008DF80560160ED2B2455D825C8DF807203D
:10D530008A08865DA25C8DF806606A408DF804203A
:10D5400013F80C2C9DF804506A401A719DF8055090
:10D5500013F80B2C6A405A719DF8065013F80A2CE8
:10D560006A409A719DF8075013F8092C01316A40FE
:10D570002C29DA7103F10403C9D102B070BD00BFD8
:10D58000544100205841002064410020A3200300A2
:10D59000A41E03000B4B1968F0B50B4E0A1D0001C9
:10D5A0001431131F35181C7815F8017B7C4003F8E3
:10D5B000014B9342F7D11A1D8A4200F10400F0D1C9
:10D5C000F0BD00BF0842002058410020084B094828
:10D5D0001B6810B5191D002213F82240045D03F8E2
:10D5E00022400132042AF7D101338B42F3D110BD1E
:10D5F00008420020A32003000D4B1B6859795A787C
:10D600005970597A5971597B5972997A5A739A7823
:10D610009970997B9A729A799971D97B9A73DA7811
:10D62000D970D97AD973D979D972DA71704700BFB4
:10D6300008420020C30903EB430303EBC30383EA5F
:10D640004000C0B270470000084B09481B6810B585
:10D65000191D002213F82240045D03F82240013214
:10D66000042AF7D101338B42F3D110BD08420020C8
:10D67000A31F03000D4B1B68597A5A7B59735979C4
:10D68000597259785971997A5A709A789970997B28
:10D690009A729A799971D9799A73DA78D970D97A14
:10D6A000D971D97BD972DA73704700BF0842002064
:10D6B0002DE9F84F0020FFF76DFF214F0124FFF700
:10D6C00085FFFFF799FF3A6802F1100A92F800907F
:10D6D0005578917892F8038089EA050081EA080B71
:10D6E0008BEA0006FFF7A6FF89EA00007040107081
:10D6F00085EA0100FFF79EFF684070405070584671
:10D70000FFF798FF48407040907089EA0800FFF7E3
:10D7100091FF88EA00004640D67004329245D5D188
:10D7200020460134E4B2FFF735FF0A2CC7D1FFF7DA
:10D730004DFFFFF761FF2046BDE8F84FFFF72ABF16
:10D74000084200202DE9F04F0A2089B0FFF722FFA0
:10D750000926FFF78FFFFFF777FF3046FFF71AFF25
:10D760004E4B196801F11003069391F8009091F85F
:10D7700001808F7891F803A04846FFF75BFF009087
:10D78000FFF758FF0190FFF755FF83464046FFF72C
:10D7900051FF0246FFF74EFF0290FFF74BFF054691
:10D7A0003846FFF747FF0390FFF744FF0790FFF766
:10D7B00041FF04465046FFF73DFF0490FFF73AFF54
:10D7C0000590FFF737FF009BDDF81CE09C46019BAE
:10D7D0008CEA030C8BEA0C0C029B82EA0C0C8BEAA1
:10D7E00002025A40039B6A405A40059B62405A40DD
:10D7F000424089EA0202019B7A408AEA02024A70A8
:10D8000083EA0B02039B6A405A4082EA0E02049BA1
:10D8100062405A40424089EA020288EA02028AEAE9
:10D8200002038B70009B83EA0B0B029B85EA0C0CB6
:10D8300083EA0B0B8EEA0C0C049B84EA0C0C85EA41
:10D840000B0580EA0C0C6C4088EA0C0C5C40059BD4
:10D8500087EA0C0C8AEA0C0C83EA040A80EA0A00C4
:10D8600089EA000988EA090887EA080781F800C000
:10D87000CF70069B04318B427FF477AF013E16F0E8
:10D88000FF067FF466AFFFF7F5FEFFF7DDFE3046DB
:10D8900009B0BDE8F04FFFF77DBE00BF0842002091
:10D8A0004B1E01380F3113F8012F00F8012F8B4266
:10D8B000F9D17047074A10B51268431E013A0F307C
:10D8C00013F8011F12F8014F834281EA0401197015
:10D8D000F6D110BD5041002038B50D460146104626
:10D8E0001446FFF7DDFF054B1C60054B1D60FFF77D
:10D8F000F7FDBDE83840FFF7DBBE00BF084200205F
:10D900005441002038B50D46014610461446FFF735
:10D91000C7FF054B1C60054B1D60FFF7E1FDBDE82F
:10D920003840FFF70FBF00BF0842002054410020DD
:10D930002DE9F74FDFF890800C9D07461C4689467D
:10D94000164602F00F0AFFF7ABFFC8F800701CB1D3
:10D950001B4B1C60FFF7C4FD0DB11A4B1D60DFF8B7
:10D9600064B00025B54209EB050107EB050413D3AC
:10D97000BAF1000F20D02046FFF792FFCAF1100243
:10D98000002104EB0A0002F09BFAC8F8004003B043
:10D99000BDE8F04FFFF7D6BE20460191FFF780FFAC
:10D9A000C8F80040FFF7CEFE2046FFF783FF01993D
:10D9B000CBF800101035D5E703B0BDE8F08F00BFFD
:10D9C0005441002050410020084200200369C268F1
:10D9D00093429CBF80681B18013B981A70472DE941
:10D9E000F843D0E902940546A9EB04084068904545
:10D9F00020440F46144404D902F039FAEC60BDE823
:10DA0000F8834246A4EB090402F031FA6868224622
:10DA100007EB0801F0E72DE9F843C568064689469B
:10DA200017464FF000083469B3687068A54228BFF4
:10DA3000E418013C621B5C1BBC4228BF3C4694427C
:10DA400028BF144649462844224602F010FAB3681B
:10DA50002544AB4208BF00253F1BA044A144F5600C
:10DA6000E1D14046BDE8F88310B5114C114AA261DE
:10DA70000223C4E90433104BE361A2644FF4007342
:10DA80000E4A0F492362E26400231022E01DA362C4
:10DA90006362E362A3656365E365226502F043FAAE
:10DAA0000849204602F03FFA2023A37110BD00BFB1
:10DAB0000C420020A3210300944200208442002055
:10DAC000AC210300B021030070B5164B182400FBF5
:10DAD00004451D4404FB00331646DC6A012C0ED0BD
:10DAE000022C18D0E4B92846FFF770FF864204D80C
:10DAF00032462846FFF773FF3446204670BD28465D
:10DB0000FFF764FF8642344628BF04462246284673
:10DB1000FFF765FFF1E72846BDE87040FFF77BBFE0
:10DB20000024EAE70C420020FFF79EBF30B50B4B04
:10DB300019680B4B0022914201D1002009E09D7829
:10DB40008478A54206D11D880488A54202D1054BE0
:10DB5000186830BD01320433EDE700BF9C4400205B
:10DB6000A0440020944400202DE9F84F90F8C6A26C
:10DB70004FF0760B04460AFB0B0088469146FFF7F0
:10DB8000D5FF074668B3D4F8CC52052D29D804EB4D
:10DB9000C5165A46A6F8D2920BFB0A4106F5357017
:10DBA00002F065F9B8F1000FC6F84C730E4F14BFC0
:10DBB0000023022386F8D0323B6801359D42C4F829
:10DBC000CC520ED104F534750026EB6F28469847E9
:10DBD0003B6801369E4205F18005F6D30023C4F868
:10DBE000CC32BDE8F88F00BF9C44002030B5A1B016
:10DBF00004460D467C22002101A802F061F90323AE
:10DC00008DF80430044BADF806501B6802940BB13C
:10DC100001A8984721B030BD944400202DE9F0417F
:10DC2000074691F8C60276234FF00008A0B081F8AD
:10DC3000C88200FB03100C461546FFF777FF064627
:10DC400060B17C22414601A802F03AF901238DF827
:10DC50000430ADF80650029701A8B0472946204687
:10DC600020B0BDE8F041FFF7C1BF000030B5044669
:10DC70008BB00D462022002102A802F021F994F871
:10DC8000C53294F8C61213B3013BDAB276234B4384
:10DC9000122000FB023323445B8A01339BB2ADF8B0
:10DCA0000430762303FB01412A460B89ADF8063088
:10DCB00003238DF80830019BCDE90543064B0493FF
:10DCC000064B02A9186800F0FBFC0BB030BD7623B0
:10DCD00003FB0143DB88E2E71DDC0200B8440020BF
:10DCE000F0B5044689B020220D466846002102F0B6
:10DCF000E7F894F8C7321E4A01331268DBB2934248
:10DD000084F8C7324FF000022AD294F8C632194F75
:10DD100084F8C5220133DBB2762113FB01F057F8FA
:10DD2000237084F8C632261827504B433271E358CB
:10DD3000CDF81230104B02930222104B8DF80020C8
:10DD40000122ADF81020186803942A46694600F0B5
:10DD5000B7FC18B12A462146FFF760FF09B0F0BDB5
:10DD600084F8C82229462046FFF740FFF6E700BFA7
:10DD70009C440020A04400201DDC0200B844002088
:10DD80002DE9F047044688B00D46164600212022B2
:10DD9000684602F095F894F8C6C294F8C512762346
:10DDA0001CFB03F2A0184FF0120E07791EFB012393
:10DDB00001F1010C0A33BC4523441CD004F11C0CB6
:10DDC00000F1220807F1FF399444CAB2974216D9EC
:10DDD00089451B8919D00EFB01FA013338F80A2056
:10DDE00093422AD10CEB0A0394F8C522013284F83D
:10DDF000C5220131E9E71B890289934208D1012339
:10DE00002B70002008B0BDE8F0870289934218D03B
:10DE100001339BB2ADF810300B4B029300210B4B3A
:10DE2000297004218DF80010ADF8122018680394B1
:10DE30003246694600F044FCE4E7013A9BB292B2F4
:10DE4000E8E70023D0E700BF1DDC0200B844002053
:10DE500010B570B1026862B1436853B10649002041
:10DE60000860064901240C7005490A60054A1360E0
:10DE700010BD0E20FCE700BF9C4400209844002009
:10DE800094440020B844002010B5044680B10C4BE7
:10DE90001B787BB1FFF74AFE70B90A4A1368052B5D
:10DEA0000CD80949246841F823400133136010BDA0
:10DEB0000E20FCE70820FAE70020F8E70420F6E748
:10DEC000984400209C440020A0440020F0B50D465A
:10DED0008BB0044600283BD0204B1B78002B39D058
:10DEE0001F4B1B68002B35D090F8C812002933D186
:10DEF0004FF4BA621B4F019101F0E2FF0199202219
:10DF000002A801F0DDFF3868294600F079FCE8B985
:10DF1000154BC4F8CC0284F8C502A4F8C6021868F0
:10DF2000206002238DF808300126104BCDF81A002E
:10DF3000A4F8CA523868ADF818602A4602A90594B8
:10DF4000049300F0BDFB08B984F8C8620BB0F0BDC3
:10DF50000E20FBE70820F9E71120F7E7984400209E
:10DF60009C440020B8440020A04400201DDC020096
:10DF70002DE9FF410C46054660B159B1974B1B781E
:10DF800043B10388322B67D007D8112B00F01881DA
:10DF9000302B1FD004B0BDE8F081332BFAD182883A
:10DFA000B1F8CA329342F5D1C08891F8C6C291F84F
:10DFB000C562002800F0C080762101FB0C410023DF
:10DFC00009798DF80F30731C8B4200F0E68084F8DD
:10DFD000C532A5E08388B1F8CA229A42DAD1C38853
:10DFE0007BBB91F8C632762202FB03130269C3F8A9
:10DFF000062091F8C432827A1344062B0EDC81F895
:10E00000C432A9882046FFF731FE0028C2D0AA8872
:10E01000214604B0BDE8F041FFF700BE062381F8B9
:10E02000C4326F486F4B7049C01AC008000440F0FA
:10E0300002000190F8F7C8FC6C490198F8F7C4FC9D
:10E04000DFE720460021FFF78FFDA988204604B0B6
:10E05000BDE8F041FFF744BE8288B1F8CA329A4267
:10E0600098D1C388002B57D191F8C672762317FB3D
:10E0700003F701EB0708837A98F804603344062B12
:10E0800025DC88F80430122212FB0672334605F1B3
:10E090000C012244002098F80460B34201F10A0107
:10E0A00002F1120227D31222013B02FB034394F830
:10E0B000C62276213B4401FB0242598A13899942C8
:10E0C0002AD2062E28D0A98884F8C5629AE70623AA
:10E0D00088F804304248434BCA5B4549C01AC0081F
:10E0E000000440F002000190F8F772FC41490198E9
:10E0F000F8F76AFCC7E751F80A6C42F8086C51F867
:10E10000066C42F8046C31F8026C168050809080E6
:10E11000D08010810133BEE7002384F8C532AA887D
:10E120000DF10F012046FFF72BFE002842D0AA88F0
:10E130002146FFF773FD2DE7762303FB0CF312272F
:10E1400007FB0633B5F80AE0294623447045BFF4BF
:10E1500033AFCF89A7F52457082F08D8DFE807F099
:10E1600014170507070707071A008F899F829F8AE0
:10E170003FB1DF8A2FB11F8B1FB15F8B002F7FF460
:10E180001BAF01300631E1E78F89DF82EFE78F892E
:10E190001F83ECE78F895F83E9E701238DF80F3058
:10E1A0002046AA880121FFF7DFFCA9882046FFF757
:10E1B00097FDEFE69DF80F30002B3FF4EBAEEFE755
:10E1C000B1F8CA3282889A4201BF002381F8C8326E
:10E1D0004FF6FF73A1F8CA32DCE600BF9844002076
:10E1E0005806030018060300B7210300D6210300D8
:10E1F0001B2203006122030090DF7047A5DF7047F8
:10E20000B5DF70477FB50023ADF80810ADF80A10F0
:10E210006A4602A90646ADF80C30ADF80E30009300
:10E22000ADF80430FFF7E8FF054600B3114B124C80
:10E23000E41AE408FAF7AEF8240444F001040346B3
:10E240000E4932462046F8F7CCFBBDF80020BDF859
:10E25000023052EA030103D009492046F8F7C1FB16
:10E26000BDF804201AB107492046F8F7B1FB28464B
:10E2700004B070BD1806030078060300C72203002F
:10E28000112303005023030080B14FF0F713036004
:10E29000FB230371F723C3801723038141F6FB326D
:10E2A0000023016143818281184670470E20704728
:10E2B00030B1A1F11703E02B04D841800020704752
:10E2C0000E2070470720704713B5034680880C4620
:10E2D000B8B91A88242A00F09C8014D8112A74D066
:10E2E000232A00F0A780102A3ED0A37A4BB1E18800
:10E2F0000020FFF783FF002840F0A2804FF48073D6
:10E30000638102B010BD3A2A68D0552AEDD1DB886E
:10E31000C988A072172B38BF17238B4228BF0B4622
:10E320002381FFF76DFF60B1FAF734F84E4B4F4988
:10E3300002464F481B1ADB081B0443F00100F8F7A4
:10E3400047FBE27A002AD0D12369002BCDD040F6DA
:10E350007721ADF802202289ADF80010ADF8042035
:10E36000694620469847C0E7DB7B0A790A73012B90
:10E3700013D0022B14D0E18823898B4205D20020D0
:10E38000FFF73CFF70B90123E372217B637B8B4273
:10E39000ABD20020FFF736FFA7E70B88E380EAE760
:10E3A0004B88FBE7112802D10123A372EDE7F9F7AF
:10E3B000F1FF2D4B2F4902462D481B1ADB081B0489
:10E3C00043F00100F8F704FBDFE7F723CB801723C6
:10E3D0000B8141F6FB3348818B8186E75B89CA88D4
:10E3E000934228BF1346172B0A6938BF17230B81A6
:10E3F00062B1C97A51B140F67721ADF80010ADF89D
:10E400000200ADF80430694620469047002363813E
:10E410006BE71A7A0B694A73002B3FF466AF4DF62F
:10E420007A218DF80500ADF80010ADF802008DF8E6
:10E43000042095E7197A237B994228BF1946A9E75A
:10E4400011283FF45EAFF9F7A5FF074B09490246D3
:10E4500007481B1ADB081B0443F0010002B0BDE8AB
:10E460001040F8F7B5BA00BF78060300D7230300C1
:10E4700018060300A62303009BDF70479DDF70474B
:10E480009EDF7047A1DF7047A3DF7047AEDF7047A4
:10E4900030B5048800239AB2944206D9456835F80D
:10E4A00013508D4203F10103F5D1104630BD8B6945
:10E4B00010B50C461988102913D8023189B2F9F722
:10E4C000B8FD606078B1A16900230222F9F7F2FD7E
:10E4D000A26960681288E1690223F9F7EBFD002068
:10E4E00010BD0920FCE70420FAE710B50C46C98AE4
:10E4F00010290AD8F9F79DFD606040B1E28AA16950
:10E500000023F9F7D7FD002010BD0920FCE7042007
:10E51000FAE70000F0B58BB004460022C068124E46
:10E520000DF10601F9F78EFE142508B10BB0F0BD10
:10E53000BDF80630A76805FB0377002202A938461C
:10E54000F9F780FE30B1E06800220DF10601F9F71D
:10E5500079FEEAE79DF8083056F82330002BECD01E
:10E560000398F9F750FDE8E784240300F7B5054662
:10E570000C4C0D480092241AE40824040B460F4664
:10E5800016460A492A7844F00100F8F734FAAB68D5
:10E5900033B1E9683A46304603B0BDE8F040184769
:10E5A00003B0F0BD80060300180603001324030027
:10E5B000F0B58FB00D46012206A90646F9F742FED6
:10E5C000044690B99DF81830052B65D8DFE803F0B4
:10E5D000030F1C24292EBDF82A20BDF82810284638
:10E5E000FFF750FF0446112C40D10FB0F0BD02A937
:10E5F0000798BDF82E200C910023F9F765FD0AA9B4
:10E600002846FFF741FFEDE7BDF828100DF12A027B
:10E610002846FFF731FFE5E70AA92846FFF72EFF56
:10E62000E0E70AA92846FFF72BFFDBE70DF1060418
:10E6300002AB214607980D9302220023F9F744FD0F
:10E64000BDF806200D9907980C940223F9F73CFDBC
:10E650000AA92846BDF80670FFF718FF04460028EF
:10E66000C1D1BDF80630BB4218BF0C249DF818205C
:10E670000F4B53F8223013B10798F9F7C4FC00226E
:10E6800006A93046F9F7DEFD002CAED02246294619
:10E6900006A8FFF76BFFA8E70648074B07491B1AB8
:10E6A000DB081B0443F00200F8F78EF9DEE700BF39
:10E6B0008424030018060300800603005D24030081
:10E6C0002DE9F8430F461446054620B94FF00E08D1
:10E6D0004046BDE8F8830029F8D0FFF71BFF3B78E0
:10E6E000052B6AD821462846FFF7D2FE2B888342A5
:10E6F00063D014264643A8683044F9F79CFD0028EF
:10E7000060D03B78052B3BD8DFE803F00311171EE0
:10E71000242A7A8A398A2046FFF7B4FE112851D07C
:10E7200058B3024621463846FFF720FF25E007F19F
:10E7300010012046FFF7A8FEF0E7398A07F1120220
:10E740002046FFF799FEE9E707F110012046FFF7A1
:10E7500095FEE3E707F110012046FFF791FEDDE7A4
:10E76000BB6907F110012046B3F80080FFF78EFE69
:10E7700030BBBB691B8843450DD14FF00008A7E7AC
:10E780001B4B1C481C49C01AC008000440F0020082
:10E79000F8F71AF9F1E70C20C3E72869002895D0AB
:10E7A000394698478046A0B192E73B7859F8233024
:10E7B000BBB17868F9F727FC13E04FF0070887E74B
:10E7C0001128AED1DFF834903B7859F82330002B74
:10E7D000E3D1A86839463044F9F7D8FC80460028D0
:10E7E000E3D1A86821463044FFF7E2FE70E700BF9E
:10E7F00018060300800603005D2403008424030040
:10E80000F8B50D46044678B3FFF784FE2946204646
:10E81000FFF73EFE2288824211D00020F8BD6168D9
:10E8200031F81310814203F101030BD0208800233B
:10E830004FF6FF769AB282420BD30420EEE7002314
:10E840004FF6FF7099B28A42E9D82069F9F7D9FBEF
:10E85000ECE761685A0001EB43078A5AB24203F1C0
:10E860000103E7D13D80D8E70E20D7E737B50C4646
:10E8700008B301B30588112D15D181882046FFF713
:10E8800007FE2388ADF80600834214D0112D14D161
:10E8900063684FF6FF7223F810200DF10601E0685F
:10E8A000F9F774FC07E0A5F130031F2BE5D9A5F1BA
:10E8B00050031F2BE1D903B030BDA368142202FB23
:10E8C0000030FFF775FEF6E78ADF70478BDF704791
:10E8D0008CDF704730B590F82C3089B004460D4677
:10E8E000D3B190F836300193FFF7F0FF14220021E6
:10E8F00003A801F0E5FA019B04F12E0204F13801AE
:10E90000A81CFFF7E5FF05238DF80C30049018B123
:10E91000A36C0BB103A8984709B030BD30B5B8B1AE
:10E92000B2B1032916D190F82810092914D81488F7
:10E93000002330F82350A54208D001330A2BF8D128
:10E940004B1C80F82830136840F82130002000E08C
:10E950000E2030BD0720FCE70420FAE768B1CB06A3
:10E960000DD011F0040116BF012380F8291080F8A2
:10E97000293080F82A20002070470E207047072099
:10E98000704700002DE9F3474378FF2B044613D06E
:10E99000654E057835614378092B0DD1811C042221
:10E9A0006248F160019101F0D0F9019940B9B36971
:10E9B000002B01DC0123B372002002B0BDE8F08718
:10E9C0005B480191062201F0C0F9019908BB594B3F
:10E9D00059485A49C01AC008000440F00500019087
:10E9E000F7F7F2FFB3690198002B03DD5449F7F7FD
:10E9F000EBFFE1E704F1080052497063062201F0E1
:10EA000047F90028D8D10223B372012386F8993040
:10EA1000D2E74D480191062201F097F90199C8B952
:10EA2000444B45484949C01AC008000440F005005D
:10EA3000F7F7CAFFB369002BBEDA04F108004149B9
:10EA40007063062201F024F90028B5D10323B372C4
:10EA50000223DBE73E480191062201F076F9019995
:10EA6000D8B9344B34483B493B4FC01AC008000466
:10EA700040F005000190F7F7A7FF2544AC4201984C
:10EA800004D13649F7F7A0FF082394E714F8012BC7
:10EA900001903946F7F79CFFF0E73148062201F074
:10EAA00054F9002888D1234B234D2E49DFF8A8A024
:10EAB000ED1AED082D0445F005052846F7F784FF0B
:10EAC000671E04F11009B84618F8012F5146284670
:10EAD000F7F77EFFC845F7D120492846F7F774FFBE
:10EAE000B369002B02DA1649284680E704F10800D2
:10EAF00014497063062201F0CBF890B9164C17F850
:10EB0000012F21462846F7F763FF4F45F7D11349F8
:10EB10002846F7F759FF09231349B3722846F7F738
:10EB200053FF032372E700BFA03F00209C24030093
:10EB3000A12403001806030068060300A8240300AC
:10EB4000B0240300C53C0020C8240300CF240300E8
:10EB5000D7240300DE240300EC240300821C0300FE
:10EB6000F3240300FA2403000825030090F838007A
:10EB7000C0F3C0007047F8B50D460446002855D0D4
:10EB8000826400212C2201F09BF9002D3AD02B79D0
:10EB900084F82C302B7B84F836302B68FBB104F1E1
:10EBA000380203F1080718685968164603C6083387
:10EBB000BB423246F7D1186830609B88B380AA68A0
:10EBC000C2B11368C4F82E305368C4F8323004F16F
:10EBD0004C03E3661F23A4F870300020F8BDA36B3C
:10EBE00003F0E30343F4200343F48273A36350234D
:10EBF000E363E4E70623E385182323634FF4C87334
:10EC0000A386E4E7A36B84F82C5003F0E30343F4FA
:10EC1000200343F48273A3635023E3630623E38555
:10EC2000182323634FF4C873A386D0E70E20D5E7DB
:10EC300010B5044686B048B31422002101A801F0A3
:10EC40003FF9FFF743FE2046FFF790FF30B1A36C7A
:10EC500023B101228DF8042001A8984704F16C012A
:10EC600004F13800FFF730FE044630F008000BD006
:10EC70000748084B08491B1ADB081B0443F0010036
:10EC80002246F7F7A5FE204606B010BD0E20FBE792
:10EC90001806030068060300182503002DE9F04755
:10ECA00080468CB038F8083B103B06460D46162BC4
:10ECB00000F2C681DFE813F03202170024002B00B7
:10ECC00032003900400047004E0055005C0013023E
:10ECD0006300A9006A007100A20078007F0086002E
:10ECE0008D0094009B00A048A04BA149C01AC00809
:10ECF000000440F005000CB0BDE8F047F7F764BE33
:10ED000099489A4B9B49C01AC0080004F1E79648FD
:10ED1000964B9949C01AC0080004EAE79248934B01
:10ED20009649C01AC0080004E3E78F488F4B944906
:10ED3000C01AC0080004DCE78B488C4B9149C01A0C
:10ED4000C0080004D5E78848884B8F49C01AC0081E
:10ED50000004CEE78448854B8C49C01AC0080004E3
:10ED6000C7E78148814B8A49C01AC0080004C0E740
:10ED70007D487E4B8749C01AC0080004B9E77A482D
:10ED80007A4B8549C01AC0080004B2E77648774B31
:10ED90008249C01AC0080004ABE77348734B80492E
:10EDA000C01AC0080004A4E76F48704B7D49C01A20
:10EDB000C00800049DE76C486C4B7B49C01AC00832
:10EDC000000496E76848694B7849C01AC0080004F7
:10EDD0008FE76548654B7649C01AC008000488E78C
:10EDE0006148624B7349C01AC008000481E75E485D
:10EDF0005E4B7149C01AC00800047AE75A485B4B61
:10EE00006E49C01AC008000473E76D4CDFF8CC915E
:10EE10000021102207A8A17201F052F805F1380371
:10EE20000B93684B376A1F60D9F82C30B3F57A7FA3
:10EE300014DBFB78192B1CD13B79FF2B2BD17B7971
:10EE4000312B28D1BB79012B25D1FB79022B22D183
:10EE50003B7AEE2B1FD13846FEF7E2F903238DF8FB
:10EE60001C30CDF8208005F16C010020FFF72CFD4F
:10EE7000E6E0022B0FD13B790A2B0CD17B790C2BCE
:10EE800009D1BB79112B06D1FB79072B03D1384669
:10EE9000FEF776FAE2E7B6F824A03846FFF772FDEF
:10EEA0003B780133AAEB030ABAF1000F01DD1F44DE
:10EEB000F3E7A37A002BD1D0434F0F22002138462D
:10EEC00000F0FEFF337C0393F37B0293B37B01934B
:10EED000737B0093337BF27A3C49384600F020FF85
:10EEE000E762F37A6377337BA377737BE377B37B54
:10EEF00084F82030F37B84F82130337C84F822308E
:10EF0000A37A012B02D10023A372A7E79A1E012A3C
:10EF100066D8A369002B7CD0D9F8242041F288332D
:10EF20009A4276DD114B104822692949294FC01AAF
:10EF3000C0080004002640F00500C9F82460A6724D
:10EF40000590F7F745FD236905989E4203DB2249AA
:10EF5000F7F73AFD5DE0E36805909A5D3946F7F70B
:10EF600037FD0136EFE700BF68060300180603000F
:10EF70003C25030080250300A0250300C1250300D4
:10EF8000E0250300FE2503001826030037260300B2
:10EF9000582603007226030090260300AB260300C8
:10EFA000C5260300ED2603000E27030027270300D4
:10EFB000502703007127030099270300BA27030095
:10EFC000A03F0020CC440020BC440020AB13030031
:10EFD000D82703005B190300821C03007040002047
:10EFE000082B37D15C4B5D485D49C01AC00800044E
:10EFF00040F005000590F7F7E7FC0023A372237F9C
:10F000000598012B1FD15749F7F7DEFC042384F83C
:10F0100099302846FFF7AAFD05F16C0400283BD083
:10F0200002238DF81C3007A8AB6CCDF820809847E0
:10F0300021460020FFF748FC41462846FFF74AFCDE
:10F040000CB0BDE8F0873846FDF7DCFF01287FF4FF
:10F0500005AFDEE7092B7FF401AF3F4B3F48424944
:10F06000424FC01AC008000440F005000590F7F7B1
:10F07000ABFC22693E490598F7F7AAFC00262369F4
:10F0800005989E42BFF663AFE36805909A5D3946E6
:10F09000F7F79EFC0136F2E795F8291095F82A203B
:10F0A00029B19DF8243043F004038DF82430CDF8C5
:10F0B000208062B100238DF81C3041462846FFF7BE
:10F0C00009FCAB6C0BB107A898472146CDE611B1FE
:10F0D0008DF81C20F1E703238DF81C30F1E71E4B5F
:10F0E0001E482449C01AC008000440F00500F7F784
:10F0F0006BFC1422002107A800F0E2FE327A012AFC
:10F100009ED1AB6C002B9BD0042138358DF81C10A0
:10F110000B958DF8202007A8984791E70E4B0F48D4
:10F120001549C01AC008000440F00500F7F74CFC70
:10F130001022002107A800F0C3FE06238DF81C3022
:10F14000B388ADF8243005F138030B93AB6CCDF8E0
:10F150002080002BDFD173E7180603006806030048
:10F16000E827030008280300222803005B19030096
:10F17000D8270300432803005928030062DF7047A3
:10F180000B6903B1184770472DE9F0410C4686B072
:10F1900005461422002101A800F092FE237813BB3B
:10F1A000A288012A1FD1A1792A7891421BD194F813
:10F1B000088022461E4618469C461F46194688452A
:10F1C00014D8BCF1000F01D0ADF816701EB1ADF827
:10F1D0001200ADF81430EB682BB16288ADF8062050
:10F1E00001A92846984706B0BDE8F081B2F80EE0C4
:10F1F000BEF1020F05D0BEF1030F06D0013112326D
:10F20000DDE7D78A4FF0010CF8E7D08A138B01268F
:10F21000F4E70000F0B5184B87B002AA04460D468B
:10F2200003F1100C174618685968164603C60833D0
:10F2300063453246F7D1ECB1E5B1AB68D3B12146B5
:10F240003846FFF79BFF98B923788DF806300123E5
:10F25000ADF804304FF6FF7363802B68E3606B6892
:10F260002361AB68A0802081636101A8FEF70CFEDA
:10F2700007B0F0BD0E20FBE7DF28030010B5034602
:10F2800086B00846F9B1F3B149884FF6FF72914252
:10F2900019D09C888C4216D11988112915D039298A
:10F2A00011D182887AB1598991420CD1C26852B188
:10F2B00001218DF8041003F11001DB890391ADF8F1
:10F2C000103001A9904706B010BDC368002BFAD0DA
:10F2D00002218DF80410428001A99847F3E700004D
:10F2E00070B504468AB040B345884FF6FF739D421F
:10F2F00025D0C6881EB32022002102A800F0E0FD20
:10F3000001238DF804308DF808300E4B6069ADF89C
:10F310001A60CDE9043402230022ADF81E3001AB9F
:10F320008DF8052008932A4640F2011302A9ADF892
:10F330001830FFF7C5F90AB070BD0E20FBE70820B2
:10F34000F9E700BF81F1020070B50E4688B015469E
:10F350000446002839D020220021684600F0B0FD84
:10F36000F42D0CD91A4B1B481B49C01AC0080004C5
:10F3700040F00200F7F728FB072008B070BD628854
:10F380004FF6FF739A420BD1114B12481349C01A22
:10F39000C008000440F00200F7F716FB0820ECE775
:10F3A00001238DF800300E4B6069ADF81650CDE9A1
:10F3B00002342389ADF8123069464FF48173069602
:10F3C000ADF81030FFF77CF9D7E70E20D5E700BF86
:10F3D0001806030060060300A8280300BA280300EB
:10F3E00081F1020050B141802AB15388C380138853
:10F3F0008380938803814069FFF702BA0E2070472B
:10F4000010DF704711DF704713B50446094968469D
:10F41000F8F766FF019808B902B010BDD0E90021E5
:10F420002046904718B16846F8F764FFF2E71120CC
:10F43000F2E700BFE829030013B504460749684610
:10F44000F8F74EFF019B0BB902B010BD2046D3E97F
:10F45000002190476846F8F74DFFF3E7002A0300C4
:10F46000084B9A6822B11A6822F480021A60704729
:10F47000054B4FF48002C3F88020BFF34F8FBFF3DA
:10F480006F8F70473037002000E100E00B4991F8A2
:10F4900016335A09EC231341DB0706D5084B9A684B
:10F4A0003AB94FF480030B60704742F20200F7F75D
:10F4B0009BBD1A6842F480021A60704700E100E0C8
:10F4C000303700202DE9F341254B264DDFF8B4807D
:10F4D000ED1AED0898F800402D0445F0050544B1FB
:10F4E00021492846F7F770FA0824204602B0BDE803
:10F4F000F0811E4F012620463E70FFF785FF112840
:10F5000004D11B492846F7F75FFAEEE72046FFF7DC
:10F5100093FF18492846F7F757FA174B8DF8034021
:10F52000186801900DF10300F8F780F8134901A85D
:10F53000FFF766FF0446B0FA80F0400988F8000043
:10F540009DF80300F8F796F8002CCED10C4B3C70D8
:10F550001C70FFF79BFF3046FFF76EFFC5E700BF4B
:10F560001806030090060300EF280300D044002093
:10F570002229030049290300E22903000570020043
:10F58000D2440020D1440020F7B51F4E33786BB928
:10F590001E4B1F481F49C01AC008000440F0050058
:10F5A000F7F712FA0824204603B0F0BD1A4D0120E7
:10F5B0002870FFF729FF11280BD1144B1448174965
:10F5C000C01AC008000440F00500F7F7FDF9002458
:10F5D000E9E70220FFF730FF00270DF107008DF863
:10F5E0000770F8F723F8FFF70DFF04469DF80700B2
:10F5F0003770F8F73FF8002CD5D103202C70FFF7B7
:10F600002FFFFFF719FFCEE7D144002018060300B3
:10F61000900603007E290300D0440020B229030095
:10F62000054B1B7833B1054B1B780BB1FFF7ACBF13
:10F63000FFF748BF08207047D0440020D144002085
:10F64000014B1878704700BFD144002007B5084926
:10F650006846F8F745FE019B13B903B05DF804FB5B
:10F66000D3E9002090476846F8F744FEF3E700BF6F
:10F67000F4290300FFF7EABF60DF704769DF7047D6
:10F6800061DF704730B5134DADF5017D4FF4FA746D
:10F690000DF1020103A8ADF80240FFF7F1FF70B9C8
:10F6A000294601A8F8F71CFE029B002BF0D003A806
:10F6B000D3E90021904701A8F8F71CFEF4E70528DC
:10F6C00005D00DF5017DBDE83040F7F78DBC0DF597
:10F6D000017D30BD882C0300024B1B780BB1FFF776
:10F6E000D1BF7047D344002030B5054685B00C46E5
:10F6F000002900F0A5800023CDE90133514A03938E
:10F7000001230A608DF804008DF8063001A9062354
:10F710002020ADF80830FFF7B1FF60B1F8F73AFEEE
:10F72000494B4A4902464A481B1ADB081B0443F06E
:10F730000100F7F74DF90023CDE901330393226867
:10F7400040F2011301A94020ADF80630FFF796FF03
:10F7500060B1F8F71FFE3C4B3E4902463C481B1A7D
:10F76000DB081B0443F00100F7F732F90023CDE971
:10F770000133039322688DF80450F72301A9232055
:10F78000ADF80630FFF77AFF60B1F8F703FE2E4BB5
:10F79000314902462E481B1ADB081B0443F00100C6
:10F7A000F7F716F9002301202268039301A9CDE998
:10F7B00001338DF80400FFF761FF60B1F8F7EAFD4F
:10F7C000214B2649024622481B1ADB081B0443F042
:10F7D0000100F7F7FDF80023CDE9023322684FF46A
:10F7E000B06301A9A1200193FFF748FF60B1F8F7CA
:10F7F000D1FD154B1A49024615481B1ADB081B049C
:10F8000043F00100F7F7E4F800252268039501A909
:10F81000A020CDE90155FFF731FF034668B1F8F7A5
:10F82000B9FD094B0F49024609481B1ADB081B04A6
:10F8300043F00100F7F7CCF82B46184605B030BD71
:10F840000E23FAE7282A0020980603000C2A03005A
:10F8500018060300522A03009E2A0300E52A03002B
:10F86000312B0300822B030073B505460668FFF7B2
:10F8700003FF2B68B34204461DD91A481A4B1B4993
:10F880001B1ADB081B0443F002000190F7F79CF8F9
:10F890002B68174901983246F7F7A3F84FF08053C9
:10F8A0002A68D3F80C31134901989B0203F10053E5
:10F8B0009A1AF7F78DF82CB90F4B01221A702046CF
:10F8C00002B070BD2046F8F765FD074B0B490246B4
:10F8D00004481B1ADB081B0443F00100F7F778F813
:10F8E000EDE700BF1806030098060300D52B0300C0
:10F8F000042C0300352C0300D34400205F2C0300AC
:10F900004BDF70471FB50E4C01A8FFF7F9FF70B928
:10F91000214602A8F8F7E4FC039B002BF4D00198E1
:10F92000D3E90021904702A8F8F7E4FCF4E70528A2
:10F9300004D004B0BDE81040F7F756BB04B010BDCA
:10F94000A02C030053EA020C61D02DE9F04BB3FA6E
:10F9500083F51E0007BFB2FA82F502FA05F403FA36
:10F9600005F41646C5F120051EBF22FA05F73C43F3
:10F97000203556EA044C4FEA144418BF0134A3461C
:10F980004FF00009C846904271EB030C39D309428D
:10F9900007BFB0FA80F700FA07F6B1FA81F701FA6B
:10F9A00007F6C7F120071EBF20FA07FC46EA0C063F
:10F9B0002037B6FBFBFC7F1B103F07F01F04C4F190
:10F9C00020060CFA04F42CFA06F644BF344600264E
:10F9D000202FA4BF2646002454EA060C08BF0124A9
:10F9E00018EB040849EB0609A4FB027CC01B06FBCC
:10F9F00002CC04FB03CC71EB0C01904271EB030CC5
:10FA0000C5D20B46024649464046BDE8F08BB2FBE4
:10FA1000F3F200007F2805D8034B185C034B5B5CB6
:10FA20001840704700207047B82C0300382D0300A1
:10FA3000A0F16103192B98BF20387047A0F1410352
:10FA4000192B98BF203070477F2805D8034B185CCE
:10FA5000034B5B5C1840704700207047B82C0300D4
:10FA6000382D0300A0F16103192B98BF203870478F
:10FA7000A0F14103192B98BF203070477F299ABF0E
:10FA8000017001206FF02E0070475AB10A787F2A6A
:10FA90000AD800B10260002119605960501A18BFDD
:10FAA00001207047002070476FF02E00704710B59E
:10FAB00004460846A2684AB12368616803F1010C54
:10FAC0008C4508BF00208B4208D2D054E3682BB18C
:10FAD00021686268914201D2214698472368013328
:10FAE000236010BD70B54C1E09D41646C5B2294618
:10FAF0003046FFF7DCFF013CB4F1FF3FF7D170BDAA
:10FB000010F0100F08D108B510F4007F14BF30209A
:10FB10002020FFF7E7FF08BD7047000008B5034B42
:10FB20005B689B681B68984708BD00BF5430002085
:10FB300008B50721FFF7F2FF08BD08B50621FFF75A
:10FB4000EDFF08BD08B50421FFF7E8FF08BD38B593
:10FB500004460D46FFF7F6FF30B1A4F13000A8428D
:10FB6000A8BF4FF0FF3038BD2046FFF7E6FF10B1C9
:10FB7000A4F15700F3E72046FFF7DAFF10B1A4F134
:10FB80003700ECE74FF0FF30E9E708B50821FFF751
:10FB9000C5FF08BD08B50921FFF7C0FF08BD00007B
:10FBA00000B5F6F715FC024B18445DF804FB00BFE6
:10FBB000080000002DE9F04F83B001908B4692467B
:10FBC0000446264614F8015BE5B12846FFF7DDFF41
:10FBD0000028F6D1302D15D1B31C257805F0DF02B1
:10FBE000582A06D0BAF1000F4ED14FF0010A08266C
:10FBF00006E03AF0100243D1A31C65789246102625
:10FC00001C4603E0BAF1000F1CD10A264FF0000891
:10FC10004746C14631462846FFF799FF002815DBC5
:10FC200008FB06084FEA184307FB06371FFA88F857
:10FC3000B7F5803F28BF4FF0010914F8015B4FF082
:10FC4000010AE7E756464FF0000ADFE7BBF1000F75
:10FC500007D0BAF1000F01D0631E0193019BCBF8CE
:10FC60000030B9F1000F04D148EA074003B0BDE805
:10FC7000F08FFFF795FF222303604FF0FF30F5E789
:10FC800056464FF0010ABBE756464FF0010AB7E768
:10FC90009AB330B594460F2A18D902460B4640EA6B
:10FCA000010414F0030F02D00CF1FF3C11E01946DF
:10FCB0001046043204330C680568A54206D110468C
:10FCC0001946ACF1040CBCF1040FF0D8BCF1010CE6
:10FCD0000FD00A46034684441146184601330132C8
:10FCE000047891F800E0744503D118461146634545
:10FCF000F2D100780B78C01A30BD002070470000A8
:10FD0000054B1A68054943F2390001FB02001860EF
:10FD1000C0F30E40704700BF683000206D4EC641F2
:10FD20000EB400B586B007AA52F8041B05920390E2
:10FD3000002304936FF00043029301A800F046F9FA
:10FD400006B05DF804EB03B07047D2B110B51446AD
:10FD5000012A12D00A460346204400F1FF3E114614
:10FD6000184613F8014B44B1013291F800C0A44584
:10FD700003D1184611469E45F1D100780B78C01A80
:10FD800010BD00207047BAB100B594460139034652
:10FD90009E4611F8012F03F8012B22B1BCF1010C92
:10FDA000F6D15DF804FBBCF1010FFAD9F44403F875
:10FDB000012B6345FBD1F4E77047037853B159B188
:10FDC0000144034613F8012F12B18B42FAD10B46BE
:10FDD000181A70470346FBE70346F9E72DE9F04F91
:10FDE00083B0814688469246FFF7DAFED0F800B02D
:10FDF0004C46274614F8015B7DB32846FFF7C5FE45
:10FE000006460028F5D12B2D03D02D2D08BF012645
:10FE100023D1FFF7C5FE00230360524601A9204607
:10FE2000FFF7C8FE0546B8F1000F05D0019BA342BD
:10FE300008BF4B46C8F80030FFF7B2FE0368222B1C
:10FE400007D0FFF7ADFEC0F800B016B1002D07DBFC
:10FE50006D42284603B0BDE8F08F3C460026D8E747
:10FE6000FFF79EFE222303604FF0FF35F1E7844643
:10FE700040EA010313F0030F18D18446202A0BD364
:10FE80002DE9F007B1E8F807A0E8F807A2F1200291
:10FE9000202AF7D2BDE8F007042A07D351F8043B23
:10FEA00040F8043BA2F10402042AF7D2002A05D04C
:10FEB00011F8013B00F8013B013AF9D16046704767
:10FEC0008446002A2DD010F0030F04D000F8011B47
:10FED000013A26D0F7E7C9B241EA012141EA0141DE
:10FEE000202A12D3A2F120022DE9F0030B460C4682
:10FEF0000D460E460F4688468946A0E8FA03203A8A
:10FF0000FBD2BDE8F00320320BD0042A05D340F821
:10FF1000041B043A05D0042AF9D200F8011B013A67
:10FF2000FBD160467047024610F0030F16D111F066
:10FF3000030F13D12DE9F0004FF001374FF080335C
:10FF400051F8044BA4EB070525EA04051D4002D136
:10FF500042F8044BF4E7A1F10401F0BC11F8013BB5
:10FF600002F8013B002BF9D1704700F1010110F0BC
:10FF7000030F11D010F8012B002A23D010F0030F2B
:10FF80000AD010F8012B002A1CD010F0030F03D068
:10FF900010F8012B002A15D02DE970004FF0013226
:10FFA0004FF0803350F8044BA4EB020525EA04051A
:10FFB0001D4000D1F6E7A0F1040070BC10F8012B41
:10FFC000002AFBD1A0EB0100704700002DE9F04FA3
:10FFD00089B007460392002303600C4614F8011B06
:10FFE000002900F0FC82DFF818B5EBE2002507E0FD
:10FFF0005E2868D145F4805501E045F040051C4677
:020000023000CC
:10000000234613F8010B3028F2D81F2837D9A0F166
:100010002002102A33D801A151F822F0FBFF020080
:100020007F0003007F000300610003007F000300E6
:100030007F0003007F000300670003007F000300D0
:100040007F0003007F0003006D0003007F000300BA
:10005000730003007F0003007F00030079000300AA
:1000600045F08005CBE745F40045C8E745F020059D
:10007000C5E745F01005C2E745F40075BFE72A283B
:1000800021D1039A111D0391D2F800A0BAF1000FFB
:10009000BCBFCAF1000A45F010051878A31C2AEA73
:1000A000EA7A2E2826D00021742847D07A2845D015
:1000B0006C2800F0A8804C2800F0AB80682800F085
:1000C000B8801C463DE0A0F13002D2B2092A88BFB8
:1000D0004FF0000AE3D84FF0000A0AEB8A0A3038E2
:1000E00000EB4A0A13F8010BA0F13002D2B2092A40
:1000F000F3D9D4E718782A280AD1039A111D03915D
:100100001168587802330029CEDB45F48075CBE7BF
:100110000133A0F13002D2B2092A88BF0021F4D8FD
:10012000002101EB8101303800EB410113F8010B94
:10013000A0F13002D2B2092AF3D9E4E71C4614F840
:10014000010B002800F05782A0F12503DBB2532BEE
:1001500062D8A0F12503532B5ED8DFE813F07600B8
:100160005D005D005D005D005D005D005D005D00A7
:100170005D005D005D005D005D005D005D005D0097
:100180005D005D005D005D005D005D005D005D0087
:100190005D005D005D005D005D005D005D005D0077
:1001A0005D005D005D005D005D005D005D005D0067
:1001B0005D005D005D005D005D005D005D005D0057
:1001C0005D005D00EC005D005D005D005D005D00B8
:1001D0005D005D005D005D005D007B0021015D0054
:1001E0005D005D005D0021015D005D005D005D0062
:1001F00095000F01D2005D005D00A6005D001A01B0
:100200005D005D00EE001C4614F8010B45F0010591
:1002100097E745F001051C46B54B1E68002E00F01F
:10022000CE8103AB0193009153462A463946B0472D
:10023000C5E11878682803D05C1C45F0040580E708
:1002400045F008059C1C58787BE725213846FFF7C8
:100250002EFCB4E1039B1A1D03921E780AF1FF3AAB
:100260003A4651462846FFF74BFC31463846FFF7E1
:100270001EFCA94619F0100F00F0A1813A46514624
:100280002020FFF72FFC9AE115F0080F06D03A68FE
:10029000039B191D03911B681A7090E1039B1A1DA3
:1002A00003921B683A681A6089E1039B1A1D039246
:1002B000D3F800808F4BB8F1000F08BF9846464630
:1002C00025F4007915F4807F16D04046FFF775FDC0
:1002D0000546AAEB050A3A4651464846FFF710FC88
:1002E000002DC7D016F8011B3846FFF7E0FBA8EB3E
:1002F0000603EB42F6D1BDE74046FFF736FE054662
:10030000E7E7039B1A1D03921B6815F0800F0CBFD3
:100310000026232645F4807508211A46002B00F09C
:100320002A8105AB4FF0000805F4005CA646604644
:100330008C460146D2E045F4005515F0800F1BD0E5
:1003400043F2780643F25803782818BF1E4615F486
:10035000807F01D025F4007515F4804F32D0039BC7
:100360001A1D03921B6815F0040F1FD01BB2002B3F
:1003700020DA5B422D262DE00026E8E715F0800FFD
:100380000CBF0026302615F4807FE5D025F40075DB
:10039000E2E715F4807F07D025F400750026DBE73F
:1003A00045F480450026D7E70026D5E715F0080F6D
:1003B000DDD0DBB215F0200F61D115F0400F18BF72
:1003C000202607E0039B1A1D03921B6815F0040FFB
:1003D00050D09BB215F4807F14BF25F40075012125
:1003E0005838202800F2AF8001A252F820F000BF58
:1003F0001B030300470503004705030047050300EF
:1004000047050300470503004705030047050300B0
:1004100047050300470503004705030047050300A0
:10042000AB0403004705030047050300470503002D
:1004300047050300AB04030047050300470503001D
:100440004705030047050300470503008304030035
:100450001B0303004705030047050300470503008E
:1004600047050300AB0403004705030047050300ED
:100470001B03030015F0080FACD0DBB2AAE72B2654
:10048000A8E71A464FF00008002B5ED005A84FF0F1
:10049000000803F00703303300F8013B08F10108BE
:1004A000D2081346002AF4D14FE018464FF0000856
:1004B000002B4AD04FF0000805F4004E4FF02C09F5
:1004C00073468E4619462FE002F00F000A4C205C5E
:1004D00003F8010B08F10108120906D00029F3D036
:1004E00002F00F00054C205CF2E7744661462CE0F8
:1004F000D44400200C2F0300EC2E0300FC2E03003C
:10050000CDCCCCCC08AB03EB080CABFB0032D20853
:1005100002EB8203A0EB430330330CF80C3C08F1F0
:10052000010809280DD910460029EBD008F0030373
:10053000032BE7D108AB434403F80C9C08F10108F6
:10054000E0E7714601E04FF00008A1EB080121EA65
:10055000E179AAEB090AAAEB080AFF2E0ED9AAF143
:10056000020AC6F307213846FFF7A1FAF1B238466E
:10057000FFF79DFA04E04FF00008E6E7002E3DD1BA
:100580003A4651462846FFF7BBFA3A4649463020DC
:10059000FFF7A8FAB8F1000F0EDD0DF1140908F10C
:1005A000FF38C84498F8001046463846FFF77FFAEF
:1005B000C14508F1FF38F5D115F0100F09D114F835
:1005C000011B61B125293FF411AD3846FFF76FFAE1
:1005D000F5E73A4651462020FFF784FAEFE7BB687B
:1005E0002BB13A6879688A423CBF00219954386837
:1005F00009B0BDE8F08F4FF0FF30F9E70AF1FF3A9C
:04060000B4E700BF9C
:10060400F595020000000000A19A0200000000001D
:04061400A9B7020080
:1006180086100300000000008C100300000000009A
:100628009310030000000000971003000000000072
:100638009C10030000000000B5070300000003033E
:100648008C08030000000000B5080300000000004B
:10065800BB22030000000303D528030000000303A6
:100668009F2803000000030380100300000000001F
:10067800062403000000030378240300000003039A
:10068800F90F030000000303DA2903000000030345
:100698007C2C030000000303942C030000000303D8
:1006A80046090300000000005C0903000000000088
:1006B800B03000207831002080310020B830002090
:1006C80018000000703A0020383B0020403B002012
:0806D800783A00201800000030
:1006E000443B0020403B00200100000002000000CD
:0406F0000100000005
:0806F40039940200000000002F
:1006FC0001960200000000003D9B0200000000007B
:10070C00D9F602000000000005F90200000000000C
:10071C0099AD0200000000006DE802006C2A002078
:10072C009DEC0200503C002071DF0200842A002066
:10073C00C9E20200183C00207DF20200FC3B0020C4
:08074C0045B0020000000000AE
:100754008807030000000000940703003C2A0020DF
:1007640000000000000000009D8C0200000000005A
:040774000000000081
:1007780000000000000000000338FDD870470000AA
:10078800DD63020049640200D96302007274745F79
:100798006C6F675F6261636B656E64004261636B77
:1007A800656E647320666C7573686564006170704B
:1007B80000000000A03500207F0000002036002047
:1007C8001B5B313B33316D0025734C6F67732064BD
:1007D800726F70706564202825642925730D0A00DE
:1007E8001B5B306D002573003C25733E2025733A52
:1007F8002000202530327800202020007C0025634E
:10080800001B5B313B33306D001B5B313B33326D7A
:10081800001B5B313B33336D001B5B313B33346D65
:10082800001B5B313B33356D001B5B313B33366D51
:10083800001B5B313B33376D007761726E696E6701
:1008480000696E666F00646562756700E8070300FB
:1008580009080300C807030011080300190803006A
:1008680021080300290803003108030039080300A0
:1008780000000000A2080300410803004908030023
:100888004E0803006170705F627574746F6E0000CB
:1008980040360020466174616C206572726F720088
:1008A80053797374656D2072657365740061707037
:1008B8005F74696D657200000100060000000000A9
:1008C8007C360020C9700200FFFFFFFFFFFFFFFF1B
:1008D800FFFFFFFFFFFFFFFF000000000000000018
:1008E8000000D6010601000052544320696E73745B
:1008F800616E636520616C726561647920696E69F7
:100908007469616C697A65642E005254433A2069AF
:100918006E697469616C697A65642E000000000074
:1009280000000000000000000338FDD87047303197
:100938003233343536373839414243444546707787
:10094800725F6D676D7400001406030018060300DB
:1009580004000000736F72746C697374004E524621
:100968005F53554343455353004E52465F455252D9
:100978004F525F5356435F48414E444C45525F4D7A
:10098800495353494E47004E52465F4552524F52C3
:100998005F534F46544445564943455F4E4F545F55
:1009A800454E41424C4544004E52465F4552524FD7
:1009B800525F494E5445524E414C004E52465F4597
:1009C80052524F525F4E4F5F4D454D004E52465F5B
:1009D8004552524F525F4E4F545F464F554E44005A
:1009E8004E52465F4552524F525F4E4F545F5355D9
:1009F80050504F52544544004E52465F4552524F54
:100A0800525F494E56414C49445F504152414D0056
:100A18004E52465F4552524F525F494E56414C49DD
:100A2800445F5354415445004E52465F4552524F1D
:100A3800525F494E56414C49445F4C454E475448D5
:100A4800004E52465F4552524F525F494E56414CF6
:100A580049445F464C414753004E52465F45525207
:100A68004F525F494E56414C49445F4441544100FE
:100A78004E52465F4552524F525F444154415F5374
:100A8800495A45004E52465F4552524F525F5449AB
:100A98004D454F5554004E52465F4552524F525F96
:100AA8004E554C4C004E52465F4552524F525F468F
:100AB8004F5242494444454E004E52465F455252B9
:100AC8004F525F494E56414C49445F41444452009D
:100AD8004E52465F4552524F525F42555359004E4F
:100AE80052465F4552524F525F434F4E4E5F434FFF
:100AF800554E54004E52465F4552524F525F524532
:100B0800534F5552434553004E52465F4552524F3C
:100B1800525F4D4F44554C455F4E4F545F494E49C7
:100B28005449414C495A4544004E52465F45525239
:100B38004F525F4D555445585F494E49545F4641A1
:100B4800494C4544004E52465F4552524F525F4D04
:100B5800555445585F4C4F434B5F4641494C4544BB
:100B6800004E52465F4552524F525F4D55544558BC
:100B78005F554E4C4F434B5F4641494C4544004EF0
:100B880052465F4552524F525F4D555445585F4348
:100B98004F4E445F494E49545F4641494C454400D5
:100BA8004E52465F4552524F525F4D4F44554C4549
:100BB8005F414C52454144595F494E495449414C63
:100BC800495A4544004E52465F4552524F525F5370
:100BD800544F524147455F46554C4C004E52465F74
:100BE8004552524F525F4150495F4E4F545F494DF5
:100BF800504C454D454E544544004E52465F455273
:100C0800524F525F464541545552455F4E4F545FCF
:100C1800454E41424C4544004E52465F4552524F64
:100C2800525F494F5F50454E44494E47004E524629
:100C38005F4552524F525F4452565F5457495F4581
:100C480052525F4F56455252554E004E52465F45DE
:100C580052524F525F4452565F5457495F45525261
:100C68005F414E41434B004E52465F4552524F52F0
:100C78005F4452565F5457495F4552525F444E4154
:100C8800434B004E52465F4552524F525F424C45CD
:100C98005F495053505F52585F504B545F54525500
:100CA8004E4341544544004E52465F4552524F52BE
:100CB8005F424C455F495053505F4348414E4E4553
:100CC8004C5F414C52454144595F45584953545330
:100CD800004E52465F4552524F525F424C455F4963
:100CE8005053505F4C494E4B5F444953434F4E4E0F
:100CF8004543544544004E52465F4552524F525F59
:100D0800424C455F495053505F504545525F5245EC
:100D18004A454354454400556E6B6E6F776E2065A7
:100D280072726F7220636F6465000000000000003B
:100D380065090300010000007109030002000000BA
:100D48008F09030003000000B0090300040000003D
:100D5800C309030005000000D409030006000000D1
:100D6800E809030007000000000A0300080000006B
:100D7800180A030009000000300A03000A000000F6
:100D8800490A03000B000000610A03000C00000080
:100D9800780A03000D0000008C0A03000E00000012
:100DA8009E0A03000F000000AD0A030010000000B7
:100DB800C10A030011000000D80A03001200000055
:100DC800E70A030013000000FC0A0300800000008B
:100DD800100B030081000000310B030082000000AB
:100DE8004D0B030083000000690B03008400000022
:100DF800870B030085000000A80B03008600000095
:100E0800CD0B030090000000E40B030091000000EC
:100E1800020C030092000000200C03000082000076
:100E2800350C030001820000530C0300028200000D
:100E38006F0C0300008400008B0C03000184000089
:100E4800AF0C030002840000D90C030003840000E7
:100E5800FE0C03000000FFFFDEC0ADDEFE011EF148
:100E6800DEC0ADDEFF011EF1705F667300257320E2
:100E7800636865636B206661696C656420696E20D0
:100E88002573282920776974682076616C75652038
:100E9800307825782E00705F66732D3E705F617024
:100EA8006900705F64657374006C656E00616464EA
:100EB800725F69735F616C69676E6564333228734A
:100EC80072632900616464725F69735F776974682B
:100ED800696E5F626F756E647328705F66732C202D
:100EE8007372632C206C656E2900705F73726300E7
:100EF80021286C656E202520705F66732D3E705F1B
:100F0800666C6173685F696E666F2D3E70726F679D
:100F180072616D5F756E69742900616464725F69DE
:100F2800735F616C69676E656433322864657374D6
:100F38002900616464725F69735F616C69676E65DB
:100F4800643332282875696E7433325F7429705F90
:100F58007372632900616464725F69735F7769748F
:100F680068696E5F626F756E647328705F66732C54
:100F780020646573742C206C656E2900616464724A
:100F88005F69735F706167655F616C69676E6564EF
:100F980028705F66732C20706167655F6164647296
:100FA8002900616464725F69735F77697468696E48
:100FB8005F626F756E647328705F66732C20706152
:100FC80067655F616464722C20286C656E202A2036
:100FD800705F66732D3E705F666C6173685F696EE3
:100FE800666F2D3E65726173655F756E6974292938
:100FF800006E72665F6673746F72616765006E7209
:10100800665F6673746F726167655F657261736549
:10101800006E72665F6673746F726167655F777280
:10102800697465006E72665F6673746F7261676576
:101038005F696E6974000000001000000400000081
:10104800010000007D9402005D9402004D940200AE
:101058009196020041960200219402002594020014
:1010680029940200000001010000000101000000B5
:101078000B0C0D0E0F101112636C6F636B00434C59
:101088004F434B004750494F544500505253005569
:10109800415254005541525445004150505F55410A
:1010A80052545F4441544100436F6D6D756E6963DE
:1010B8006174696F6E206572726F72206F636375F9
:1010C80072726564207768696C652068616E646C0B
:1010D800696E6720554152542E004572726F722016
:1010E8006F6363757272656420696E204649464F66
:1010F800206D6F64756C6520757365642062792056
:10110800554152542E004576656E743A2025732059
:10111800726563656976656420284E52465F53554B
:10112800434345535329004576656E743A20257329
:1011380020726563656976656420282573290052E5
:1011480065636F72642049443A09307825303478F1
:101158000046696C652049443A093078253034786E
:10116800005265636F7264206B65793A093078259F
:1011780030347800424C455F4741505F4556545FD4
:101188005343414E5F5245515F5245504F525400B0
:10119800424C455F4741505F4556545F434F4E4E62
:1011A800454354454400446973636F6E6E656374C8
:1011B80065642E20636F6E6E5F68616E646C653A5D
:1011C80020307825782C20726561736F6E3A203054
:1011D80078257800436F6E6E656374696F6E205270
:1011E8006571756573742074696D6564206F7574B5
:1011F8002E00446973636F7665727920636F6D7032
:101208006C6574652E00436F6E6E6563746564204B
:10121800746F206465766963652077697468204E09
:101228006F72646963205541525420536572766920
:1012380063652E00547970652025780A0057455358
:1012480020005452414E5346455220535749544367
:1012580048202D2D2D2020456D657267656E6379B8
:1012680000446576696365205265676973747261C5
:1012780074696F6E2044697361626C6500545241F1
:101288004E5346455220535749544348202D2D2D3F
:10129800202054455354005452414E534645522041
:1012A800535749544348202D2D2D202044657669F5
:1012B800636520526567697374726174696F6E0043
:1012C80030782530327800526567204D61633D3EA5
:1012D80025730A0053656E642057455341434B00FC
:1012E8005452414E5346455220535749544348207F
:1012F8002D2D2D2020416C6976650042616E642099
:101308005061726B696E672025640A004E75732000
:1013180046697273742044617461203D3D3E004209
:10132800616E6420416C61726D2025640A004F6E05
:10133800652050617373204170702025640A004E47
:101348007573205365636F756E6420446174612002
:101358003D3D3D3E003D3D3D3D3D3D3D3D205365D0
:101368006E642043415241434B0A00446973636FE2
:101378006E6E6563746564202D2D2D2D2D2D2D2DFC
:101388002D2D2D2D2D2D2D2D2D2D2D2D0A00436F7D
:101398006E6E656374696E6720746F20746172671E
:1013A800657420253032782530327825303278251A
:1013B8003032782530327825303278005363616EC8
:1013C8002074696D6564206F75742E004154542033
:1013D8004D54552065786368616E676520636F6D4D
:1013E800706C657465642E00426C65204E55532000
:1013F8006D61782064617461206C656E6774682023
:1014080073657420746F2030782558282564290066
:1014180053656E6420627574746F6E2064617461C4
:101428000067705374733D25640D0A00505245538C
:101438005345440D0A0052656C65617365640D0A75
:101448000044656C6574696E67206E6578742072F7
:1014580065636F72642E004E6F207265636F7264ED
:1014680073206C65667420746F2064656C657465A0
:101478002E005F313030306D735F74696D65725F57
:1014880068616E646C652853595354454D5F454DEA
:10149800455247454E43595F534952454E29202DE1
:1014A8002D205B2564202F2025645D0A005F3130E4
:1014B80030306D735F74696D65725F68616E646CFE
:1014C800652853595354454D5F5345525645525F0D
:1014D800434F4D4D29202D2D205B2564202F20259D
:1014E800645D0A005F313030306D735F74696D651B
:1014F800725F68616E646C652853595354454D5F3B
:10150800524547495354455229202D2D205B2564C7
:10151800202F2025645D0A005F313030306D735F05
:1015280074696D65725F68616E646C6528535953A0
:1015380054454D5F5345525645525F434F4D4D5F9D
:1015480052455129202D2D205B2564202F2025640C
:101558005D0A000A3D3D3D3D3D3D3D3D3D3D3D3D36
:101568003D3D3D3D3D3D3D3D3D3D3D3D3D3D3D3DA3
:101578003D3D3D3D3D3D3D3D3D3D3D3D3D3D3D3D93
:101588003D3D3D3D3D3D3D3D3D3D3D3D3D3D3D0AB6
:101598000A004945532D36303052422043454E54B7
:1015A80052414C2050726F6772616D2053746172A2
:1015B80074202D2D2056657220312E313020203296
:1015C8003032322F30332F32300A00424C4520550A
:1015D8004152542063656E7472616C206578616D48
:1015E800706C6520737461727465642E0046445390
:1015F8005F4556545F494E4954004644535F45562B
:10160800545F5752495445004644535F4556545F0A
:10161800555044415445004644535F4556545F4431
:10162800454C5F5245434F5244004644535F45562C
:10163800545F44454C5F46494C45004644535F451A
:1016480056545F47430000000800000006000000F1
:1016580005000000070000000000000000502700FF
:1016680000000000000000000338FDD870470000AB
:10167800F515030002160300101603001F160300D9
:101688003216030043160300F03B0020503B0020B5
:10169800040000002000000001000000010002001A
:1016A800303C0020070B0C0D3D3D3D3D3D3D3D3D93
:1016B8003D3D3D3D3D3D3D3D3D3D3D3D3D3D3D3D52
:1016C8003D3D3E0A0A0053656E64546F4576656E6B
:1016D80074536572766572203D3D3E200025303298
:1016E8005820003D3D3D3E2053656E645061726B4D
:1016F800696E6741707028290A003D3D3D3E2053C0
:10170800656E64456D657267656E637942616E6486
:1017180028290A0053656E64456D657267656E63B6
:101728007942616E643D3D3D003D3D3D3E2053653F
:101738006E645061726B696E6742616E6428290A33
:101748000053656E645061726B696E6742616E64C6
:10175800203D3D3D003D3D3D3E20526553656E6454
:10176800456D657267656E637928290A005265536D
:10177800656E64456D657267656E6379203D3D3DB4
:10178800003D3D3D3E2053656E6441636B28290A48
:10179800003D3D3D3E2053656E64456D657267654D
:1017A8006E637928290A003D3D3D3E2053656E64ED
:1017B800416C69766528290A0053656E64416C6935
:1017C8007665203D3D3D003D3D3D3E2053656E64C0
:1017D80043757272656E7452656744657628290A86
:1017E800003D3D3D3E205365727665725F416E73E4
:1017F8007765725F5265675F4C697374202825644A
:10180800204541290A004465764C697374202530C7
:1018180032782530327825303278203D3D3D3D3DC7
:1018280020004465764C6973742025303278253061
:10183800327825303278203D3D3D3D3D3E200053F5
:1018480065727665725F416E737765725F43616C2E
:101858006C2829003D3D3D3E205365727665725FD8
:1018680056657273696F6E5F416E73776572283261
:1018780032290A003D3D3D3E205365727665725F10
:10188800416E737765725F55706772656164282968
:101898000A003D3D3D3D3D3D3D3D3D3D3D3D3D3DE0
:1018A8003D3D3D3D3D3D3D3D3D3D3D3D3D3D3D3D60
:1018B8003D3D3D3D3D3D3D3D3D3D3D3D3D3D3D3D50
:1018C8003D3D3D3D3D3D3D3D3D3D3D3D3D3D3D3D40
:1018D8003D3D3D3D3D3D3D3D3D3D3D3D3D3D3D3D30
:1018E8003D3D0A003D3D3D3D3D3D3D3D3D3D3D3D90
:1018F8003D3D3D3D3D3D3D3D3D3D3D3D20526562CB
:101908006F6F7420546F20426F6F744C6F61642046
:101918005374617274203D3D3D3D3D3D3D3D3D3D2F
:101928003D3D3D3D3D3D3D3D3D3D3D3D3D3D3D3DDF
:101938003D3D3D3D0A00534552564552203D3D3EF2
:1019480020524543455645522044415441203A20AF
:1019580000307825303278200052656376203A20AE
:101968004E6F726D616C0052656376203A20546147
:101978006C6B696E670052656376203A2044697320
:10198800636F6E6E6563740052656376203A204219
:101998007573790052656376203A204B656570202F
:1019A800416C6976650052656376203A206D6963FB
:1019B800206F6E2F6F6666006D6963206F6E00730F
:1019C8007065616B6572206F6666006D6963206F74
:1019D800666600737065616B6572206F6E00526594
:1019E8006376203A20434F4D5F545950455F535614
:1019F800525F524543565F5245475F524551005327
:101A0800595354454D2069732042555359203A2063
:101A18005B25645D0A0052656376203A20434F4D8A
:101A28005F545950455F5356525F524543565F497C
:101A38004E49545F5245510052656376203A20431F
:101A48004F4D5F545950455F5356525F5245435668
:101A58005F4C4953545F5245510052656376203AB2
:101A680020434F4D5F545950455F5356525F434191
:101A78004C4C5F5245510052656376203A20434FE3
:101A88004D5F545950455F5356525F5645525F5209
:101A980045510052656376203A20434F4D5F5459B3
:101AA80050455F5356525F555047524541445F5227
:101AB800455100566F696420416C697665546573B9
:101AC8007428290A000000000338FDD870477265A1
:101AD800632E206964090966696C652069640909CF
:101AE8007265632E206B6579096C656E6774680A88
:101AF800006572726F723A204352432063686563CF
:101B08006B206661696C6564210A006572726F7288
:101B18003A207265636F7264206E6F7420666F7509
:101B28006E64210A006572726F723A20756E65786C
:101B38007065637465206572726F722025732E0A52
:101B48000020307825303478090920307825303461
:101B5800780909203078253034780909202534752A
:101B6800206279746573090077726974696E6720F9
:101B78007265636F726420746F20666C6173682E7F
:101B88002E2E0A66696C653A20307825782C206BF1
:101B980065793A20307825782C20222573222C204C
:101BA8006C656E3A2025752062797465730A006544
:101BB80072726F723A206664735F7265636F7264E3
:101BC8005F777269746528292072657475726E650D
:101BD800642025732E0A000A7265632E2069640941
:101BE8000966696C6520696409097265632E206B52
:101BF8006579096C656E677468096D61630A004DE3
:101C0800616320506F6F6C204F7665720A00416CDB
:101C18006C72656164792052656769737472617466
:101C280065640A0056616C6964204D61630A004569
:101C3800434220656E63727970743A2025780A00F1
:101C4800536D61727442616E6450415254524F4EEA
:101C5800004341520102030405060708090A0B0C58
:101C68000D004543422041434B0A00434152414342
:101C78004B0102030405060708090A0031392D48FB
:101C880044432D49434F4E54524F4C53004844430C
:101C98002D49562D524E4443454E544552004170ED
:101CA80070205061726B20496E666F20416E6472BD
:101CB8006F6964204C6F772044617461203D3D3E1C
:101CC8002000417070205061726B20496E666F2051
:101CD800416E64726F6964203D3D3E200041707022
:101CE800205061726B20496E666F20694F53204CFB
:101CF8006F772044617461203D3D3E200041707043
:101D0800205061726B20496E666F20694F53203DE9
:101D18003D3E20004644535F4552525F4F50455266
:101D28004154494F4E5F54494D454F555400464420
:101D3800535F4552525F4E4F545F494E4954494193
:101D48004C495A4544004644535F4552525F554EEC
:101D5800414C49474E45445F414444520046445330
:101D68005F4552525F494E56414C49445F41524784
:101D7800004644535F4552525F4E554C4C5F4152AA
:101D880047004644535F4552525F4E4F5F4F5045A0
:101D98004E5F5245434F524453004644535F4552A9
:101DA800525F4E4F5F53504143455F494E5F464C2B
:101DB800415348004644535F4552525F4E4F5F536C
:101DC800504143455F494E5F51554555455300467F
:101DD80044535F4552525F5245434F52445F544FFC
:101DE8004F5F4C41524745004644535F4552525F4E
:101DF8004E4F545F464F554E44004644535F45523C
:101E0800525F4E4F5F5041474553004644535F452C
:101E180052525F555345525F4C494D49545F5245A4
:101E28004143484544004644535F4552525F43523C
:101E3800435F434845434B5F4641494C4544004650
:101E480044535F4552525F42555359004644535FCD
:101E58004552525F494E5445524E414C00000000D5
:101E68001C1D0300361D03004E1D0300651D0300E5
:101E7800791D03008A1D0300A21D0300BC1D030079
:101E8800D71D0300F01D0300021E0300131E0300EC
:101E98002E1E0300471E0300541E03008D0102047A
:101EA80008102040801B366CD8AB4D9A2F5EBC635F
:101EB800C697356AD4B37DFAEFC5913972E4D3BDBC
:101EC80061C29F254A943366CC831D3A74E8CB8D52
:101ED80001020408102040801B366CD8AB4D9A2FA5
:101EE8005EBC63C697356AD4B37DFAEFC591397283
:101EF800E4D3BD61C29F254A943366CC831D3A74EE
:101F0800E8CB8D01020408102040801B366CD8AB4A
:101F18004D9A2F5EBC63C697356AD4B37DFAEFC578
:101F2800913972E4D3BD61C29F254A943366CC834C
:101F38001D3A74E8CB8D01020408102040801B363E
:101F48006CD8AB4D9A2F5EBC63C697356AD4B37D07
:101F5800FAEFC5913972E4D3BD61C29F254A943323
:101F680066CC831D3A74E8CB8D010204081020402A
:101F7800801B366CD8AB4D9A2F5EBC63C697356A0A
:101F8800D4B37DFAEFC5913972E4D3BD61C29F2500
:101F98004A943366CC831D3A74E8CB52096AD5302B
:101FA80036A538BF40A39E81F3D7FB7CE339829BDB
:101FB8002FFF87348E4344C4DEE9CB547B9432A68A
:101FC800C2233DEE4C950B42FAC34E082EA166285B
:101FD800D924B2765BA2496D8BD12572F8F6648656
:101FE800689816D4A45CCC5D65B6926C704850FDB8
:101FF800EDB9DA5E154657A78D9D8490D8AB008C55
:10200800BCD30AF7E45805B8B34506D02C1E8FCACE
:102018003F0F02C1AFBD0301138A6B3A9111414FC3
:1020280067DCEA97F2CFCEF0B4E67396AC7422E799
:10203800AD3585E2F937E81C75DF6E47F11A711D79
:1020480029C5896FB7620EAA18BE1BFC563E4BC63F
:10205800D279209ADBC0FE78CD5AF41FDDA83388E8
:1020680007C731B11210592780EC5F60517FA91959
:10207800B54A0D2DE57A9F93C99CEFA0E03B4DAE84
:102088002AF5B0C8EBBB3C83539961172B047EBA81
:1020980077D626E169146355210C7D637C777BF242
:1020A8006B6FC53001672BFED7AB76CA82C97DFA44
:1020B8005947F0ADD4A2AF9CA472C0B7FD932636A1
:1020C8003FF7CC34A5E5F171D8311504C723C318FF
:1020D80096059A071280E2EB27B27509832C1A1B22
:1020E8006E5AA0523BD6B329E32F8453D100ED207A
:1020F800FCB15B6ACBBE394A4C58CFD0EFAAFB4340
:102108004D338545F9027F503C9FA851A3408F92DB
:102118009D38F5BCB6DA2110FFF3D2CD0C13EC5F75
:10212800974417C4A77E3D645D197360814FDC2214
:102138002A908846EEB814DE5E0BDBE0323A0A4994
:1021480006245CC2D3AC629195E479E7C8376D8DFB
:10215800D54EA96C56F4EA657AAE08BA78252E1CD5
:10216800A6B4C6E8DD741F4BBD8B8A703EB56648C1
:1021780003F60E613557B986C11D9EE1F8981169BD
:10218800D98E949B1E87E9CE5528DF8CA1890DBF77
:10219800E6426841992D0FB054BB165465726D69BB
:1021A8006E616C0052545400534547474552004EE7
:1021B8006F7420656E6F7567682073706163652042
:1021C800666F722073657276696365732E00496E57
:1021D80063726561736520424C455F44425F4449C0
:1021E80053434F564552595F4D41585F53525620FD
:1021F800746F2062652061626C6520746F2073744F
:102208006F7265206D6F726520736572766963659C
:102218007321004E6F7420656E6F75676820737048
:1022280061636520666F72206368617261637465BB
:1022380072697374696373206173736F636961741E
:1022480065642077697468207365727669636520B0
:10225800307825303458202100496E6372656173E7
:102268006520424C455F474154545F44425F4D41AD
:10227800585F434841525320746F20626520616261
:102288006C6520746F2073746F7265206D6F726552
:1022980020636861726163746572697374696373DA
:1022A80020666F7220656163682073657276696362
:1022B800652100626C655F64625F646973630073C3
:1022C800645F626C655F6761705F646174615F6CB5
:1022D800656E6774685F7570646174652829202865
:1022E8007265717565737429206F6E20636F6E6EE9
:1022F800656374696F6E203078257820726574750F
:10230800726E65642025732E0054686520726571AD
:102318007565737465642054582F52582070616332
:102328006B6574206C656E67746820697320746FC0
:102338006F206C6F6E672062792025752F257520B8
:102348006F63746574732E005468652072657175C7
:10235800657374656420636F6D62696E6174696F1B
:102368006E206F6620545820616E64205258207089
:1023780061636B6574206C656E677468732069733C
:1023880020746F6F206C6F6E67206279202575202E
:102398006D6963726F7365636F6E64732E00736427
:1023A8005F626C655F67617474635F6578636861B9
:1023B8006E67655F6D74755F726571756573742896
:1023C800292072657475726E65642025732E0073FA
:1023D800645F626C655F67617474735F6578636876
:1023E800616E67655F6D74755F7265706C792829B9
:1023F8002072657475726E65642025732E006E7286
:10240800665F626C655F676174740053442047417E
:1024180054542070726F6365647572652028256452
:1024280029206661696C6564206F6E20636F6E6E2B
:10243800656374696F6E2068616E646C65202564DD
:102448002077697468206572726F723A2030782537
:102458003038582E00556E696D706C656D656E74F8
:102468006564204741545420526571756573740042
:102478006E72665F626C655F677100000000000045
:10248800EBE4020000000000000000000000000073
:10249800AFE40200494353420049435343415200C9
:1024A8004943534341520A00203C3C202054726166
:1024B8006E73666572204275737920203E3E0A006D
:1024C800494353454D4700494353454D470A004941
:1024D8004353574553003D3D3E20494353574553C9
:1024E800203A2000253032582C20004943535043CD
:1024F80041003D3D3E20494353504341203A20008E
:102508003D3D3E204943535043415F4D41430A00FE
:1025180073645F626C655F6761705F7363616E5F50
:1025280073746172742072657475726E656420309C
:10253800782578003C2D2D2D2D2D2D2D2D2D2D2D53
:102548002D2D2D2D2D2D2D2D20424C455F474150F1
:102558005F4556545F444953434F4E4E4543544597
:1025680044202D2D2D2D2D2D2D2D2D2D2D2D2D2D89
:102578002D2D2D2D2D3E0A00424C455F4741505FC1
:102588004556545F434F4E4E5F504152414D5F5543
:102598005044415445200A00424C455F4741505F32
:1025A8004556545F5345435F504152414D535F5226
:1025B800455155455354200A00424C455F47415008
:1025C8005F4556545F5345435F494E464F5F5245FA
:1025D8005155455354200A00424C455F4741505FCE
:1025E8004556545F504153534B45595F44495350E6
:1025F8004C4159200A00424C455F4741505F4556BF
:10260800545F4B45595F50524553534544200A0087
:10261800424C455F4741505F4556545F41555448C9
:102628005F4B45595F52455155455354200A004266
:102638004C455F4741505F4556545F4C4553435F97
:1026480044484B45595F52455155455354200A005B
:10265800424C455F4741505F4556545F4155544889
:102668005F535441545553200A00424C455F47413B
:10267800505F4556545F434F4E4E5F5345435F5539
:102688005044415445200A00424C455F4741505F41
:102698004556545F525353495F4348414E4745445A
:1026A800200A00424C455F4741505F4556545F53EE
:1026B80045435F52455155455354200A00424C4505
:1026C8005F4741505F4556545F434F4E4E5F504100
:1026D80052414D5F5550444154455F52455155450F
:1026E8005354200A00424C455F4741505F455654B9
:1026F8005F5048595F5550444154455F52455155C4
:10270800455354200A00424C455F4741505F4556A7
:10271800545F5048595F555044415445200A00427F
:102728004C455F4741505F4556545F444154415FB3
:102738004C454E4754485F5550444154455F5245B7
:102748005155455354200A00424C455F4741505F5C
:102758004556545F444154415F4C454E4754485F89
:10276800555044415445200A00424C455F4741506A
:102778005F4556545F514F535F4348414E4E454C59
:102788005F5355525645595F5245504F5254200A8F
:1027980000424C455F4741505F4556545F4144569F
:1027A8005F5345545F5445524D494E41544544206A
:1027B8000A00424C455F4741505F4556545F5343BA
:1027C800414E5F5245515F5245504F5254200A00C6
:1027D8006E616D65206C656E20697320256420002C
:1027E8003D3D3D3D3D3D3D3D3D3D3D3D3D3D3D3D11
:1027F8003D20204445565F5745535F4144560A00E3
:1028080052656369766572204D6F6465206973202F
:1028180052656769737465720A003D3D3D3D3D3DF3
:102828003D3D3D3D3D3D3D3D3D3D3D2020444556E2
:102838005F494F535F5041524B0A00424C455F4736
:1028480041505F4556545F54494D454F5554200AF1
:10285800003C2D2D2D2D2D2D2D2D2D2D2D2D2D2DBE
:102868002D2D2D2D2D2D2D20424C455F4741505F9C
:102878004556545F434F4E4E4543544544202D2DF5
:102888002D2D2D2D2D2D2D2D2D2D2D2D2D2D2D2D70
:102898002D2D2D3E200A00626C655F7363616E000A
:1028A800436F6E74656E7420746F6F206C6F6E6703
:1028B8002E00436F6E6E656374696F6E2068616E7B
:1028C800646C6520696E76616C69642E00626C6563
:1028D8005F6E75735F63009ECADC240EE5A9E09302
:1028E800F3A3B50000406E6E72665F7364685F653F
:1028F8006E61626C655F72657175657374202D2DEC
:10290800204E52465F4552524F525F494E56414CF7
:1029180049445F53544154450A006E72665F7364BC
:10292800685F656E61626C655F7265717565737409
:10293800202D2D204E52465F535543434553530A8D
:10294800006E72665F7364685F656E61626C655F76
:1029580072657175657374202D2D207364685F73BB
:10296800746174655F6F627365727665725F6E6FAE
:10297800746966790A006E72665F7364685F646979
:102988007361626C655F72657175657374202D2D56
:10299800204E52465F4552524F525F494E56414C67
:1029A80049445F53544154450A006E72665F73642C
:1029B800685F64697361626C655F72657175657380
:1029C80074202D2D204E52465F5355434345535393
:1029D8000A006E72665F73646800010000070000F9
:1029E800F4060300FC060300080000000C070300BF
:1029F8001C07030008000000FC0603000C07030086
:102A08000800000073645F626C655F6366675F73EC
:102A1800657428292072657475726E656420257343
:102A2800207768656E20617474656D7074696E676F
:102A380020746F2073657420424C455F434F4E4E9F
:102A48005F4346475F4741502E0073645F626C6581
:102A58005F6366675F736574282920726574757291
:102A68006E6564202573207768656E2061747465CF
:102A78006D7074696E6720746F2073657420424CA2
:102A8800455F4741505F4346475F524F4C455F4360
:102A98004F554E542E0073645F626C655F636667C2
:102AA8005F73657428292072657475726E65642079
:102AB8002573207768656E20617474656D7074691C
:102AC8006E6720746F2073657420424C455F434FD6
:102AD8004E4E5F4346475F474154542E0073645F30
:102AE800626C655F6366675F736574282920726529
:102AF8007475726E6564202573207768656E206131
:102B08007474656D7074696E6720746F2073657472
:102B180020424C455F434F4D4D4F4E5F4346475F04
:102B280056535F555549442E0073645F626C655F68
:102B38006366675F73657428292072657475726EA1
:102B48006564202573207768656E20617474656DEF
:102B58007074696E6720746F2073657420424C45E9
:102B68005F47415454535F4346475F415454525F53
:102B78005441425F53495A452E0073645F626C6545
:102B88005F6366675F736574282920726574757260
:102B98006E6564202573207768656E20617474659E
:102BA8006D7074696E6720746F2073657420424C71
:102BB800455F47415454535F4346475F5345525618
:102BC8004943455F4348414E4745442E00496E738B
:102BD800756666696369656E742052414D20616C43
:102BE8006C6F636174656420666F72207468652019
:102BF800536F66744465766963652E004368616E39
:102C08006765207468652052414D20737461727441
:102C1800206C6F636174696F6E2066726F6D20300F
:102C280078257820746F20307825782E004D6178CB
:102C3800696D756D2052414D2073697A6520666F04
:102C480072206170706C69636174696F6E2069735A
:102C580020307825782E0073645F626C655F656E3E
:102C680061626C6528292072657475726E656420CE
:102C780025732E006E72665F7364685F626C650010
:102C88001C07030054070300080000006E72665F0B
:102C98007364685F736F630004060300140603001F
:102CA8000800000043000000504F5349580000003E
:102CB80020202020202020202068282828282020A4
:102CC80020202020202020202020202020202020FC
:102CD80048101010101010101010101010101010B4
:102CE8008484848484848484848410101010101054
:102CF80010818181818181010101010101010101AD
:102D08000101010101010101010101101010101060
:102D1800108282828282820202020202020202027D
:102D28000202020202020202020202101010102025
:102D38000007032004170201085710408000000014
:102D4800AC2C0300B02D0300C42E030053756E0095
:102D58004D6F6E00547565005765640054687500C2
:102D68004672690053617400000000004A616E00F9
:102D7800466562004D617200417072004D617900D4
:102D88004A756E004A756C0041756700536570009E
:102D98004F6374004E6F76004465630000000000C6
:102DA800414D00504D000000E82E0300E42E0300C2
:102DB800E42E0300E42E0300E42E0300E42E0300B7
:102DC800E42E0300E42E0300E42E0300E42E0300A7
:102DD800FFFFFFFFFFFFFFFFFFFFFFFFFFFF0000F9
:102DE800242E0300542D0300602E0300742D0300CD
:102DF800A82D0300082E0300B82E0300142E03008C
:102E0800256D2F25642F25790000000025612025D8
:102E180062202565202554202559000053756E64CD
:102E28006179004D6F6E64617900547565736461F2
:102E380079005765646E65736461790054687572CA
:102E480073646179004672696461790053617475CD
:102E580072646179000000004A616E7561727900E0
:102E68004665627275617279004D617263680041EE
:102E78007072696C004D6179004A756E65004A751B
:102E88006C79004175677573740053657074656D6E
:102E9800626572004F63746F626572004E6F76658B
:102EA8006D62657200446563656D6265720000005D
:102EB80025483A254D3A25530000000015FA02002E
:102EC80031FA02003DFA020049FA020065FA0200EE
:102ED80071FA02007DFA02008BFA0200000000007D
:102EE8002E000000303132333435363738396162DC
:102EF80063646566303132333435363738394142A8
:0B2F080043444546286E756C6C2900A0
:102F140000000000FF000000001001401100040048
:102F240000000000002000400000000000200040DD
:102F3400000000000090D0030B00030019B8020049
:102F440001000000802A002090160300E006030020
:102F5400CC060300FFFF000000000000000000009A
:102F6400000000000000000000000000000000005D
:102F7400000000000000000000000000000000004D
:102F8400000000000000000000000000000000003D
:102F9400000000000000000000000000000000002D
:103224000000FFFF0000000000000000000000009C
:10323400000000000000000000000000000000008A
:10324400000000000000000000000000000000007A
:10325400000000000000000000000000000000006A
:10326400000000000000000000000000000000005A
:103524000000000000000000482D0300482D0300A7
:10353400482D0300482D0300482D0300010000001E
:040000032000637501
:00000001FF
